:020000041000EA
:1000000000B5324B212058609868022188439860DF
:10001000D860186158612E4B002199600221596106
:100020000121F02299502B49196001219960352056
:1000300000F044F80222904214D00621196600F024
:1000400034F8196E01211966002018661A6600F04E
:100050002CF8196E196E196E052000F02FF8012189
:100060000842F9D1002199601B49196000215960AB
:100070001A491B48016001219960EB211966A021F2
:10008000196600F012F800219960164914480160C1
:100090000121996001BC002800D000471248134993
:1000A000086003C880F30888084703B5996A0420EC
:1000B0000142FBD001200142F8D103BD02B5186610
:1000C0001866FFF7F2FF186E186E02BD00000240BE
:1000D000000000180000070000035F00212200005C
:1000E000F4000018222000A00001001008ED00E03C
:1000F00000000000000000000000000074B24E7A12
:1001000000200420F7010010C3010010C5010010F9
:10011000C1010010C1010010C1010010C101001097
:10012000C1010010C1010010C1010010C701001081
:10013000C1010010C1010010C9010010CB01001065
:10014000CD010010CD010010CD010010CD01001037
:10015000CD010010CD010010CD010010CD01001027
:10016000CD010010CD010010CD010010CD01001017
:10017000CD010010CD010010CD010010CD01001007
:10018000CD010010CD010010CD010010CD010010F7
:10019000CD010010CD010010CD010010CD010010E7
:1001A000CD010010CD010010CD010010CD010010D7
:1001B000CD010010CD010010CD010010CD010010C7
:1001C00000BE00BE00BE00BE00BE00BE00F04BF888
:1001D000103800BEF2EB887160D3001088D3001095
:1001E0003402001090A31AE700202149086006C8D5
:1001F00081F3088810471F48006800282FD10DA4FC
:100200000ECC002902D000F012F8F9E71A491B4A77
:10021000002000E001C19142FCD1194988471949E9
:1002200088471949884700BEFDE701C901C29A42C3
:10023000FBD3704788D30010C0000020281E002088
:10024000F0F000100000042000000420F0F0001086
:1002500000100420001004200000000070470B482C
:1002600006F00CFA0047EFF30580C0B270470000BB
:1002700008ED00E0000000D0281E0020202F002004
:1002800019370010FD0E00104538001057560000B9
:1002900006005250ABB3605344CE001006005250DB
:1002A000861C030254CE0010060052505422A29D18
:1002B0005CCE001005005250DE65F468F0F00010CE
:1002C000F8B5C0460448054B10B5834203D0044B33
:1002D000002B00D0984710BD281E0020281E0020AB
:1002E0000000000006480749091A8910CB0F591869
:1002F00010B5491003D0044B002B00D0984710BD17
:10030000281E0020281E00200000000010B5074C09
:100310002378002B09D1FFF7D5FF054B002B02D026
:10032000044800E000BF0123237010BD301F0020EF
:100330000000000008C80010054B10B5002B03D0CA
:100340000449054800E000BFFFF7CCFF10BDC046E0
:1003500000000000341F002008C80010F8B5254D2B
:100360002B681B785A2B41D0234807F07DF9234C8A
:10037000B9220021200007F04FF8EFF3108772B682
:100380001F4807F04DFA80218020490100030CF03E
:100390000BFA1C4E300007F067F91B4807F040FAD3
:1003A0002100802280204739520000030CF0E4F93C
:1003B000300007F059F987F310888022134C52005F
:1003C0002968200007F02EF8114807F04DF9611C4C
:1003D000104807F025FA21000F480B3107F020FAEA
:1003E00021000E48333107F01BFAF8BD0C4807F026
:1003F0003BF9E2E7C414002048CA0010C71F0020E0
:1004000070CA001088CA001090CA0010801F002017
:10041000DCCA0010ECCA0010FCCA001010CB00109F
:10042000B4CA0010F0B5D6464F4646462D48C0B572
:1004300007F01AF92C4C2D48216807F0F1F92C4EE1
:100440002C48316807F0ECF92B4B2C4819689A4678
:1004500007F0E6F92A4D2B48296807F0E1F92A4F01
:100460002A48396807F0DCF9294B2A481968984668
:1004700007F0D6F9284B29481968994607F0D0F9B2
:10048000274807F0CDF92168264C20000AF0CEF964
:10049000002803D1244807F0E7F8FEE75346200080
:1004A00019680BF071FB4B46200019680BF0CAF974
:1004B000434639681A6820000AF0B0FF316820000E
:1004C0000BF06AF8296820000BF00CFB20000BF001
:1004D000A3FB164807F0C8F81CBC90469946A246F4
:1004E000F0BDC046A8C80010D0140020B8C8001045
:1004F000D8140020D4C80010D4140020F0C8001074
:10050000CC1400200CC90010DC14002028C90010F5
:10051000C014002044C90010C814002060C9001095
:100520007CC900108020002090C90010A0C90010D4
:10053000F0B5C64600B507F07FF9FF2200211F483D
:1005400006F06AFFFF2200211D4806F065FF062025
:1005500001F024FF052001F021FF042001F01EFF1F
:10056000022001F01BFF032001F018FF0820D02417
:10057000402120220026042710238046114D240606
:1005800061626262636267626062A161F2302E70D2
:10059000A2616E706361AE70676102F071FB4346E9
:1005A000A7610948A361EE7002F06AFBFFF7D6FE6F
:1005B000FFF738FF04BC9046F0BDC046202A00205B
:1005C000402B0020AC20002088130000F0B5C64668
:1005D000CB4D00B58046FD222800002106F01CFF0F
:1005E000C423023D5B422B80C64EC533AB7073788B
:1005F000002B00D1AFE1EB70B378002B00D1B9E153
:100600002B71F378002B00D1B8E16B713379002B9B
:1006100000D1B5E1AB717379002B00D18CE1EB71A6
:10062000B379002B00D1ADE12B72F379002B00D10F
:10063000AAE16B72337A002B00D1A7E1AB72737A17
:10064000002B00D1A4E10C27EB727B1CBA1C1D000F
:1006500011003E24AC48C455777D002F3FD0C754CD
:10066000B57D5A1C92B2002D00D15FE18554F57D15
:10067000991C89B2002D00D15AE14554357EDA1C0F
:1006800092B2002D00D151E18554757E191D89B2B9
:10069000002D00D14CE14554B57E5A1D92B2002D7B
:1006A00000D143E18554F57E991D89B2002D00D11A
:1006B0003EE14554357FDA1D92B2002D00D135E17F
:1006C00019008554727F083189B2002A00D12FE1C8
:1006D00009339BB242545A1C92B21D001100F77F9D
:1006E000002F52D02C23202143558754531C775C74
:1006F000911C9BB289B21D008C46002F00D11FE1D6
:10070000C7542123F75CD31C9BB21D00002F00D1DE
:1007100027E147542221775C111D89B28C46002FB6
:1007200000D10DE1C7542323F75C531D9BB21D007C
:10073000002F00D115E147542421775C911D89B227
:100740008C46002F00D1FBE0C7542523F75CD31D56
:100750009BB21D00002F00D103E147542621775C96
:100760001100083189B28C46002F00D1E8E0C7544F
:100770002723F75C130009339BB21D00002F00D123
:10078000EFE00A3292B2475411002927F75D002F9B
:100790004DD02C232A2143558754531C775C911C40
:1007A0009BB289B21D008C46002F40D0C7542B232A
:1007B000F75CD31C9BB21D00002F00D1D6E047543C
:1007C0002C21775C111D89B28C46002F2FD0C75485
:1007D0002D23F75C531D9BB21D00002F00D1C5E0F7
:1007E00047542E21775C911D89B28C46002F1ED074
:1007F000C7542F23F75CD31D9BB21D00002F00D1DF
:10080000B4E047543021775C1100083189B28C463E
:10081000002F0CD0C7543123F75C130009339BB26F
:100820001D00002F00D1A1E00A32475491B23A22B4
:1008300042554254F57A9F1CBFB2002D00D181E091
:100840003C3AD31A00E017007A1C92B2D11889B250
:10085000C5557518ED7A002DF5D108293BD820250E
:1008600085544A1CBB1C92B29BB2092A00D183E07A
:100870000231033789B2BAB2C55409292BD02023DB
:100880004E1C551CB6B2ADB28354092E52D04355FE
:100890008D1C961CADB2B6B2092D4FD08355CE1C1F
:1008A000D51CB6B2ADB2092E44D043550D1D161D50
:1008B000ADB2B6B2092D41D083554E1D551DB6B20D
:1008C000ADB2092E36D0961DB6B24355032935D0A8
:1008D000073292B283553A23835443461978561C03
:1008E000B6B200291AD0FE2E18D8451CAD198319AE
:1008F000FD264446B21A92B20134AA180AE0C04654
:10090000422B0020801F0020402B002001330134A7
:10091000934203D0197021780029F7D101221D4B91
:100920001A7006F0A1FE04BC9046F0BD1300D2E69A
:100930000B00D0E62A00CEE7072786E63200CAE79A
:100940000A0022E720211A1D03339BB2C15592B23F
:10095000C1541E3993E705210522042504230327EA
:1009600077E61A000D00190063460EE70D00190026
:1009700063465CE7042768E61A00ACE7052764E6EF
:10098000062762E6082760E609275EE60A275CE696
:100990000B275AE6512C0020F0B5DE464546574657
:1009A0004E46E0B59C4C0A22A54404AC0021200030
:1009B00020AD06F031FDFF220021280006F02CFDBD
:1009C000FF22002160A806F027FDFF220021A0A839
:1009D00006F022FD6422002107A806F01DFDFF227B
:1009E0000021E0A806F018FD8C4B1A78002A41D0AF
:1009F00022703E2A00D1EAE05A78002A3AD062708A
:100A00003E2A00D1E6E09A78002A33D0A2703E2A2E
:100A10003DD0DA78002A2DD0E2703E2A00D1D0E015
:100A20001A79002A26D022713E2A00D1CCE05A79C8
:100A3000002A1FD062713E2A00D1CEE09A79002AA6
:100A400018D0A2713E2A00D1D9E0DA79002A11D05B
:100A5000E2713E2A00D1D5E01A7A002A0AD0227229
:100A60003E2A00D1D1E05A7A002A03D062723E2A8F
:100A700000D1CDE06A4806F0D3FE00252800694B7E
:100A80009D443CBC90469946A246AB46F0BD03212E
:100A900002220020A0545A5C002AEBD02A703A2A85
:100AA00000D18FE101220131585C17000028E1D00C
:100AB000A85401323A28F6D10022EA555A18507843
:100AC000002200280DD00132561EC027B4466E46C3
:100AD0007F00F6196746F0558818181840780028E6
:100AE000F1D1C02069460023400009188B542978B1
:100AF000002900D15DE10022002000279846994698
:100B0000431C9C46434607AEB2469B185B005344C9
:100B1000561C1954B2462C2962D060460137E95D53
:100B20000029EDD107AB9C46424452006244115467
:100B30003D482278C17A8A420BD1002A10D0002386
:100B400001E0002A0CD00133C118E25CC97A8A4264
:100B5000F7D0002A00D139E1002908D0914206D10E
:100B6000C0226B4652009B181B783A2B64D000259C
:100B7000002760AB03933A236B4402930CAB0193C1
:100B800026236B440093524607AB2100274806F00A
:100B900047FEA0226B4692009B181B78002B00D1C9
:100BA0006CE72A00A0A9224806F03AFE002F00D1E7
:100BB00064E7E0A8FFF70AFDE0A91E4806F030FE52
:100BC0005CE70421032264E70521042261E7012197
:100BD00000225EE7022101225BE70621052258E799
:100BE0006146092999DC49461954092E00DDC2E005
:100BF000931C9A46B3003200002098468EE70721E6
:100C0000062246E70821072243E70921082240E798
:100C10000A21353A3DE7C0467CFBFFFF202A002031
:100C20002CCA001084040000801F0020ACC90010F2
:100C3000E8C9001010CA00106B460A329B181B78D6
:100C40003A2B94D14378002B5AD082216A46FF3147
:100C5000521812789A428AD18378002B50D06A4673
:100C60000131521812789A4200D080E7C378002BE5
:100C700046D084216A46FF31521812789A4200D039
:100C800075E70379002B3BD06A4601315218127880
:100C90009A4200D06BE74379002B31D086216A4617
:100CA000FF31521812789A4200D060E78379002B06
:100CB00026D06A460131521812789A4200D056E77F
:100CC000C379002B1CD088216A46FF315218127854
:100CD0009A4200D04BE7037A002B11D06A460131CB
:100CE000521812789A4200D041E7437A002B07D07D
:100CF0008A216A46FF31521812789A4200D036E7AC
:100D00008C226B46FF329B181A78002A0FD00B23D7
:100D1000A02519006846AD000B3940194254C02186
:100D20006A46490001335218D25C002AF0D1612191
:100D3000A0226B46894602319200884608319B18F2
:100D400000250027002000228C461B78002B33D082
:100D5000A0266946B60001328919895C7B2B13D025
:100D6000002F31D1AE00B3465D44303B6D00ED182D
:100D7000ADB20B00EAE707AA90466246B3005344BF
:100D80005B004344995475E66B460136FF369B1968
:100D90004E461F181E5443467B70C31C6046B870F5
:100DA000E0276E46BF00F619581CF15401270B00CE
:100DB000CCE701239A46BBE6E0216A468900521837
:100DC0001354D6E6002777E60300E9E7002900D0B0
:100DD000CDE6C5E6F8B53F4C0222200000210930DF
:100DE00006F01AFB3C4B200023603C4B0222636060
:100DF000322300211330237206F00EFB4E23200015
:100E0000412631254327E37201332373033BE37308
:100E1000237404221F3B00211B306773A673A57443
:100E2000637406F0F9FA502344222000A3750A33B4
:100E3000E37562760D3B3A3A00211F3066752376E2
:100E4000A37606F0E9FA2000254B0A222362254BFF
:100E50000021A384293006F0DFFA2000224B04226F
:100E60006385224B0021A385214B4330E38506F0A7
:100E7000D3FA332356226E21E2540133E5542A3A41
:100E80000133E2540133E75443320133E254013376
:100E9000E15401330631E15439333A3963540131B5
:100EA0006254033A01316254013162542E3A2831BE
:100EB000A1540132A354323B1F3AE254103BA355D4
:100EC0000C4A1233E55411680B4B596092881A8111
:100ED000F8BDC046801F00205A4E4F43414C4C2D58
:100EE000494445312D31000049440000453200009D
:100EF0002D320000A0C80010AC200020F0B5DE4666
:100F000057464E464546E0B595B0FFF711FB744B8A
:100F100000249A46734B26009946734B9846734BB0
:100F20009F1ED0231B069B460021504609F0F0FF70
:100F3000051E0ED14B461B78002BF5D0002E03D199
:100F40006B4B9B6A9B059E0D012E21D0013EB6B2D4
:100F5000EAE750460AF06CF90100664806F060FCCA
:100F60000024504609F0E2FA0134634A631ED0546B
:100F7000AC42F6D1130000225A551B783C2B03D10A
:100F80005D4B5B78FF2B20D05C4806F06DFBD1E712
:100F90000021504609F008FE3978002908D00024C5
:100FA00001345046A4B209F047FA395D0029F7D15F
:100FB0000021504609F004FF002150460AF076F95E
:100FC00000234A4600261370AEE74B4B9B78012B5B
:100FD000DAD1032D04DDEA1E494947480BF00CFC29
:100FE000454B9C4600236544033D60462B7006F04C
:100FF0003BFBFFF7D1FC0500041E9BD0252801D93F
:1010000001F0ABF93F4A8300D3589F4640235A462C
:10101000936100223C4B1A704B461B78002B8DD1FC
:1010200082E75B460824FA205C6101F029FE5B46FA
:101030009C610123344AD3704B461B78002B00D0AF
:101040007CE771E710235A4693612F4A0F3B937058
:101050004B461B78002B00D070E765E720235A46EB
:101060005361294A1F3B53704B461B78002B00D01D
:1010700064E759E720235A4693610022224B5A70B5
:101080004B461B78002B00D058E74DE710235A46FB
:10109000536100221C4B9A704B461B78002B00D0EA
:1010A0004CE741E75B460424FA205C6101F0E8FD6F
:1010B0005B4600229C61144BDA704B461B78002B78
:1010C00000D03BE730E740235A4653610E4A3F3B8E
:1010D00013704B461B78002B00D02FE724E7C04647
:1010E00080200020512C0020801F0020422B002057
:1010F0000040054020CB0010202A002040CB0010EB
:10110000232A002008C80010AC200020D84B002162
:101110001B78D8485A1E9341D54A303313725378FE
:101120005A1E9341D24A3033D37193785A1E934159
:10113000CF4A30339371D3785A1E9341CC4A30331F
:101140005371FD2206F068F9C422CA4B5242023B99
:101150001A80C5329A7042465278002A01D100F0B6
:1011600017FCDA7042469278002A01D100F0ADFCFB
:101170001A714246D278002A01D100F020FD5A713E
:1011800042461279002A01D100F048FD9A71424688
:101190005279002A01D100F0E3FDDA7142469279DA
:1011A000002A01D100F040FE1A724246D279002A8C
:1011B00001D100F0D4FE5A724246127A002A01D1BF
:1011C00000F062FF9A724246527A002A01D100F082
:1011D000E9FFDA7218230E210F240D220A930C93D3
:1011E000013B0993013B079301331393023B0693A1
:1011F00001330893023B059301331293023B04939E
:1012000001331093023B039301331193023B02938A
:1012100001330D93023B019301330E93023B009384
:1012200001330B93023B0F93023B9C4601333E2557
:1012300060463D544046457D002D3DD0BD54837DE4
:10124000002B01D100F076FC7B54C37D002B01D133
:1012500000F078FC009ABB54037E002B01D100F013
:1012600041FD019ABB54437E002B01D100F042FDA9
:10127000029ABB54837E002B01D100F004FE039A36
:10128000BB54C37E002B01D100F0A7FE049ABB54CF
:10129000037F002B01D100F0B8FE059ABB54437FB9
:1012A000002B01D100F076FF069A0999BB540A9BE6
:1012B0000C9C0093079A089B4046C57F002D64D084
:1012C0002C20B8547D54202241468A5C002A01D14A
:1012D00000F0FAFD0098D91C3A5421224046845C63
:1012E00089B20A00002C01D100F06FFE7C5422224A
:1012F0004146181D8C5C80B20200002C01D100F028
:10130000FAFE3C5423224046591D845C89B20A00EF
:10131000002C01D100F085FF7C5424224146981D09
:101320008C5C80B20200002C01D100F0A5FF3C547F
:1013300025224046D91D805C89B20A001C00002885
:1013400001D100F0A2FF7854262241460834885C7F
:10135000A4B22200002801D100F0D2FF3855272284
:10136000190040460931805C89B20A00002801D189
:1013700000F0CFFF1A001C000A320B3392B27854EF
:1013800099B213000C34A4B2009429254046405D64
:10139000002863D00335BD5478542A2241468A5C24
:1013A000002A01D100F09AFD0098D91C3A542B2252
:1013B0004046845C89B20A00002C01D100F098FDFF
:1013C00042467C54181D545D80B20200002C01D1AD
:1013D00000F0A1FE3C542D224046591D845C89B288
:1013E0000A00002C01D100F09EFE7C542E224146C2
:1013F000981D8C5C80B20200002C01D100F02AFF05
:101400003C542F224046D91D805C89B20A001C0042
:10141000002801D100F04AFF7854302241460834B8
:10142000885CA4B22200002801D100F060FF38558A
:101430003122190040460931805C89B20A00002837
:1014400001D100F081FF1A001C000A320B3392B266
:10145000785499B213000C34A4B200943A25BD54C8
:1014600042467D54D17A002900D17DE2002005E07A
:10147000AC200020422B00201400180039554146B2
:10148000431C9BB2C918C97A621C92B20029F3D1DD
:101490001100082B42D82021A51CADB28C46B954AE
:1014A0002900072800D15DE26146E01C80B2795531
:1014B0000100072B00D155E26146251DADB239541C
:1014C0002900062B00D14DE26146601D80B279559E
:1014D0000100052B00D145E2614606343954A1B222
:1014E000042B00D13EE22024901D80B27C540100E8
:1014F000032B00D136E2D51DADB23C542900022B9E
:1015000000D12FE21000083080B27C550100002B82
:1015100000D027E2093292B211003C543A237B54A6
:10152000D84B501C197980B2002911D0FE280FD851
:10153000FD239A1A92B201320023381802E00133D7
:101540009A4205D0C154CF49C91849790029F6D12A
:1015500001234A463800137006F086F84B461B7884
:10156000002B00D0EAE4DFE4FD220021C64805F0AC
:1015700053FFC422C44B5242023B1A80C5329A70B8
:1015800042465278002A00D143E2DA70424692780D
:10159000002A00D16BE21A714246D278002A00D1AB
:1015A000DFE25A7142461279002A00D16CE39A7147
:1015B00042465279002A00D1A4E3DA714246927978
:1015C000002A01D100F002FC1A724246D279002AA8
:1015D00001D100F095FC5A724246127A002A01D1DC
:1015E00000F023FD9A724246527A002A01D100F09F
:1015F000A2FDDA7218230E220C210E200C930B93FD
:10160000013B0893013B079301331393023B06937D
:1016100001330993023B059301331293023B049378
:1016200001331093023B039301331193023B029366
:1016300001330D93023B019301330E93023B009360
:1016400001330A930F928C46013B013A01313E254A
:1016500064463D554446657D002D39D0BD54A27D7C
:10166000002A00D15FE23A54E27D002A00D171E203
:10167000009BFA54237E002B00D1FEE2019ABB545A
:10168000637E002B00D19AE3029ABB54A37E002B09
:1016900001D100F000FC039ABB54E37E002B01D182
:1016A00000F0A3FC049ABB54237F002B01D100F06F
:1016B0001AFD059ABB54637F002B01D100F0A9FDF0
:1016C000069A0898BB540C9B079A009309990B9BA8
:1016D0004446E57F002D63D02C24BC543D54202289
:1016E0004046825C002A00D1DCE30098CB1C3A54CF
:1016F00021224046845C9BB21A00002C01D100F0EC
:101700007CFCFC5442462223081DD45C80B20200BB
:10171000002C01D100F081FC3C54232240464B1D9B
:10172000845C9BB21A00002C01D100F06AFDFC54CD
:1017300042462423881DD45C80B20200002C01D1D3
:1017400000F091FD3C5425224046CB1D805C9BB2AD
:101750001A00002801D100F0B1FDF85442462623BA
:101760000C00D05C0834A4B222000B00002801D188
:1017700000F0B5FD3855272240460933805C9BB206
:101780001A00002801D100F0D6FD0A00F8540B0021
:101790000A320B3192B288B211000C339BB2009323
:1017A00029254446645D002C61D00335BD543C546A
:1017B0002A224046825C002A00D17CE30098CB1CA0
:1017C0003A542B224046845C9BB21A00002C00D174
:1017D000F4E3FC544346081D5C5D80B20200002C1B
:1017E00001D100F090FC3C542D2240464B1D845CFE
:1017F0009BB21A00002C01D100F01BFDFC544246A4
:101800002E23881DD45C80B20200002C01D100F090
:1018100018FD3C542F224046CB1D805C9BB21A0021
:10182000002801D100F039FDF854424630230C0065
:10183000D05C0834A4B222000B00002801D100F0D3
:1018400046FD3855312240460933805C9BB21A0070
:10185000002801D100F066FD0A00F8540B000A329E
:101860000B3192B288B211000C339BB200933A252F
:10187000BD5442463D54D07A002800D1B5E0002541
:1018800006E0C046AC200020422B002023001500BB
:1018900041466A1C92B28918F854C87A5C1CA4B2FA
:1018A0000028F3D12100082A3AD82021981C80B2C0
:1018B0008C4639550100072D52D06146DD1CADB272
:1018C00039542900072A4BD06146181D80B279553A
:1018D0000100062A44D061465D1DADB2395429008D
:1018E000052A3DD061460633795599B2042A37D08E
:1018F0002020A31D9BB278541900032A30D0E51D87
:10190000ADB2F8542900022A2AD0230008339BB232
:1019100078551900002A23D10934A4B22100F854C3
:101920003A2342467B54073BD25C601C80B2002ABB
:1019300000D10DE6FE2800D90AE6FD21091B89B277
:1019400001310023381803E001338B4200D1FFE559
:10195000C2541A0044463432A25C002AF4D1F7E59E
:101960000C00DDE70A00D9E52022009903339BB281
:101970007A54FA54A31C9BB2FA54E31C9BB2FA5457
:10198000231D9BB2611DFA5489B222000023AAE5EF
:101990000F230A930C93013B0993013B07930133F7
:1019A0001393023B069301330893023B05930133E3
:1019B0001293023B049301331093023B03930133D0
:1019C0001193023B029301330D93023B01930133C8
:1019D0000E93023B009301330B93023B0F93023BA8
:1019E0009C4605210422013321E420220098033182
:1019F00089B23A547A54991C89B27A54D91C89B262
:101A00007A54191D89B27A54591D89B21C000022DA
:101A10006EE70F23052203210C930B93013B0893E0
:101A2000013B079301331393023B06930133099360
:101A3000023B059301331293023B0493013310934D
:101A4000023B039301331193023B029301330D9345
:101A5000023B019301330E93023B009301330A933F
:101A60000F928C460520013B013A0131EFE510232E
:101A7000062204210C930B93013B0893013B07932F
:101A800001331393023B069301330993023B059301
:101A900001331293023B049301331093023B0393EF
:101AA00001331193023B029301330D93023B0193E7
:101AB00001330E93023B009301330A930F928C463D
:101AC0000620013B013A0131C1E510230A930C9332
:101AD000013B0993013B079301331393023B0693A8
:101AE00001330893023B059301331293023B0493A5
:101AF00001331093023B039301331193023B029392
:101B000001330D93023B019301330E93023B00938B
:101B100001330B93043B9C460F95062107240522B5
:101B20000133FFF784FB019902000A9B00980091A2
:101B30000F99CDE5019B0A000B9C009900930F9B28
:101B4000FFF7BAFB029B009A0199009323000E9CB9
:101B5000FFF7B2FB0299009A0198009119000E9BC1
:101B6000B6E51123072205210C930B93013B089343
:101B7000013B079301331393023B0693013309930F
:101B8000023B059301331293023B049301331093FC
:101B9000023B039301331193023B029301330D93F4
:101BA000023B019301330E93023B009301330A93EE
:101BB0000F928C460720013B013A013147E5112283
:101BC00005200A920C92013A0992013A07920132D9
:101BD0001392023A069201320892023A05920132B9
:101BE0001292023A049201321092023A03920132A6
:101BF0001192023A029201320D92023A019201329E
:101C00000E92023A009201320B92023A0F922B008E
:101C100007210824013A8446FFF709FB12230A939F
:101C20000C93013B0993013B079301331393023B50
:101C3000069301330893023B059301331293023B51
:101C4000049301331093023B039301331193023B3E
:101C5000029301330D93023B019301330E93023B38
:101C6000009301330B93023B0F93023B9C460821E8
:101C7000092407220133FFF7DAFA039B0298009345
:101C8000019A0D9B0A9923E51223082206210C9341
:101C90000B93013B0893013B079301331393023BE2
:101CA000069301330993023B059301331293023BE0
:101CB000049301331093023B039301331193023BCE
:101CC000029301330D93023B019301330E93023BC8
:101CD000009301330A930F928C460820013B013A8E
:101CE0000131B4E4039B029900930D9C019A0B9B74
:101CF000FFF7E2FA049B03990093119C029A0E9B52
:101D0000FFF7DAFA1323092207210C930B93013B07
:101D10000893013B079301331393023B069301336E
:101D20000993023B059301331293023B0493013361
:101D30001093023B039301331193023B029301334F
:101D40000D93023B019301330E93023B0093013349
:101D50000A930F928C460920013B013A013176E447
:101D600013230A930C93013B0993013B079301331F
:101D70001393023B069301330893023B059301330F
:101D80001293023B049301331093023B03930133FC
:101D90001193023B029301330D93023B01930133F4
:101DA0000E93023B009301330B93023B0F93023BD4
:101DB0009C4609210A2408220133FFF738FA049BC4
:101DC00003980093029A119B0E9981E414230A222E
:101DD00008210C930B93013B0893013B07930133BC
:101DE0001393023B069301330993023B059301339E
:101DF0001293023B049301331093023B039301338C
:101E00001193023B029301330D93023B0193013383
:101E10000E93023B009301330A930F928C460A20E3
:101E2000013B013A013112E414230A930C93013B64
:101E30000993013B079301331393023B069301334C
:101E40000893023B059301331293023B0493013341
:101E50001093023B039301331193023B029301332E
:101E60000D93023B019301330E93023B0093013328
:101E70000B93023B0F93023B9C460A210B24092241
:101E80000133FFF7D4F9059B04990093109C039A42
:101E90000D9BFFF711FA059B04980093039A109B82
:101EA0000D9915E49D1C581CACB2009A190080B223
:101EB0000094230074E49D1C581CACB2009A1900D5
:101EC00080B200942300D2E4A51C611CA8B2009A41
:101ED000230089B200900400FFF757FAA51C611C8B
:101EE000A8B2009A230089B200900400FFF7B6FA66
:101EF0005C1DA4B2043399B200941300FFF7AEFA4C
:101F000015230B2209210C930B93013B0893013BF2
:101F1000079301331393023B069301330993023B6A
:101F2000059301331293023B049301331093023B58
:101F3000039301331193023B029301330D93023B50
:101F4000019301330E93023B009301330A930F92E6
:101F50008C460B20013B013A0131FFF778FB15233A
:101F60000A930C93013B0993013B079301331393AD
:101F7000023B069301330893023B0593013312930E
:101F8000023B049301331093023B039301331193FB
:101F9000023B029301330D93023B019301330E93F5
:101FA000023B009301330B93023B0F93023B9C4691
:101FB0000B210C240A220133FFF739F94B1D9BB288
:101FC000043188B20093110051E45C1DA4B20433C3
:101FD00099B200941300FFF7D8F9069B0599009376
:101FE000129C049A119BFFF767F9069B05980093D2
:101FF000049A129B1199FFF76BFB4B1D9BB20431A6
:1020000088B200931100FFF7CBFB079B0699009362
:10201000089C059A109BFFF74FF98B1D9BB2053169
:1020200088B200931100FFF7BBFB16230C220A2194
:102030000C930B93013B0893013B079301331393DC
:10204000023B069301330993023B0593013312933C
:10205000023B049301331093023B0393013311932A
:10206000023B029301330D93023B019301330E9324
:10207000023B009301330A930F928C460C20013BE4
:10208000013A0131FFF7E3FA16230A930C93013B5F
:102090000993013B079301331393023B06930133EA
:1020A0000893023B059301331293023B04930133DF
:1020B0001093023B039301331193023B02930133CC
:1020C0000D93023B019301330E93023B00930133C6
:1020D0000B93023B0F93023B9C460C210D240B22D9
:1020E0000133FFF7A4F8079B06980093059A099B14
:1020F0001099FFF7EDFA9C1DA4B2053399B2009434
:102100000300FFF742F98B1D9BB2053188B20093A3
:102110001100FFF7ACFB9C1DA4B2053399B20094EB
:102120000300FFF79BF9DC1DA4B2063399B20094BB
:102130001300FFF793F917230D220B210C930B9338
:10214000013B0893013B079301331393023B069332
:1021500001330993023B059301331293023B04932D
:1021600001331093023B039301331193023B02931B
:1021700001330D93023B019301330E93023B009315
:1021800001330A930F928C460D20013B013A013135
:10219000FFF75DFA099B07990093139C069A129B1F
:1021A000FFF78AF817230A930C93013B0993013B2D
:1021B000079301331393023B069301330893023BC9
:1021C000059301331293023B049301331093023BB6
:1021D000039301331193023B029301330D93023BAE
:1021E000019301330E93023B009301330B93023BA7
:1021F0000F93023B9C460D210E240C220133FFF766
:1022000016F8CB1D9BB2063188B200931100FFF780
:10221000C7FA089B07980093069A139B1299FFF739
:1022200057FADC1DA4B2063399B200941300FFF7ED
:10223000ACF8CB1D9BB2063188B200931100FFF7BA
:1022400016FB0B00083307319BB288B200931100D4
:10225000FFF70DFB1C0008340733A4B299B20094B9
:102260000300FFF7FBF80B00083307319BB288B27D
:1022700000931100FFF794FA1C0008340733A4B24E
:1022800099B200940300FFF780F809340833A4B230
:1022900099B200941300FFF778F80B000933083166
:1022A0009BB288B200931100FFF7E1FA09340833BA
:1022B000A4B299B200941300FFF7D0F80B000933D1
:1022C00008319BB288B200931100FFF769FA0A3314
:1022D00009319BB288B200932100FFF7C8FA0A3394
:1022E00009319BB288B200932100FFF759FA1C0014
:1022F0000A340933A4B299B200941300FFF7AEF880
:102300001C000A340933A4B299B200941300FFF7F9
:102310003CF81C000B340A33A4B299B200941300A9
:10232000FFF733F80B000B330A319BB288B20093EE
:102330001100FFF79CFA0B000B330A319BB288B2F5
:1023400000931100FFF72CFA1C000B340A33A4B2DF
:1023500099B200941300FFF781F84B4619780029D1
:1023600001D1FEF7E2FDFEF7E9FDC046094A830010
:1023700094464022634410B51C68C0006240C024EB
:1023800014408022520113431C60034B9C4660445E
:10239000416010BD04C00140004001400123D02233
:1023A0008340120693629361094A83009446402257
:1023B00063441968C0004A40C02111408022520184
:1023C00013431960034B9C460523604443607047E8
:1023D00004C0014000400140F8B5EFF3108772B629
:1023E0000D4E3368002BFCD0BFF35F8F0725CB0861
:1023F000C01801230D40AB401D000478254007D1D3
:1024000023430370BFF35F8F356087F31088F8BDF7
:10241000100001F019FAC0462C0100D0F8B5CE46E4
:1024200047468C4680B5EFF3108972B6214D2C6873
:10243000002CFCD0BFF35F8F9A422CD807210125D6
:1024400011408D40D4080419267835421FD0072149
:102450008846063909E045460F001540AF40D408CC
:10246000041926783D00374211D001329342F2D24E
:1024700001204042BFF35F8F00220E4B1A6089F3A8
:10248000108800280FDB0CBC90469946F8BD3543F8
:1024900025701000EEE7BFF35F8F00232B6089F3F8
:1024A0001088012040426346002BECD0089801F0D0
:1024B000CBF9C0462C0100D0024B18688007C00F32
:1024C0007047C04600C006400021044B044ABFF3D9
:1024D0005F8F02C39342FAD17047C046000100D01B
:1024E000800100D0044A1078431CDBB2172B00D9BE
:1024F000102313707047C046E014002000B5054B50
:1025000083B00100009318221F230348FFF786FFC2
:1025100003B000BD64CB00105C25002083680B482D
:1025200010B5844661446244090112019A18591891
:1025300054684B6801209C4201D802D00020C0B2F0
:1025400010BD12680B689A42F9D8F7E7FFFFFF0F3A
:102550000A4B1968EFF3108072B60A68002AFCD0A3
:10256000BFF35F8F1B68BFF35F8F00221A6080F399
:10257000108840BF002000217047C046242B002057
:10258000F8B557464E464546DE46E0B51F000CAB53
:102590001D780DAB1B7881469A4603681600984655
:1025A000002D3BD1987B002832D04246454644005E
:1025B00012682418033C121951780300A9730029EA
:1025C00000D1E9730021050091705170117029E06C
:1025D000D31814199D702278002A00D05A705B46D7
:1025E000237043465D734B463200187D3B0000F07C
:1025F00003FD041E07D05346002B04D14B4629008F
:10260000186800F0E9FE0E9B002B44D028001C70D7
:102610003CBC90469946A246AB46F8BD2B006C00E8
:102620006419033C1D4A94464A46926863449446A2
:102630001B010A9A63449A600B9A1E605F60DA601D
:10264000434600221B681B199A705A701A70434641
:102650005B7B9B46002BC4D043462A0098685946B2
:102660005B6898475B4642465B005B44033B1268ED
:102670000028ADD0D31814195A46A2701A78002A2F
:1026800007D11D705A46434628005A73AB45BFD147
:10269000A9E76270F5E72800BAE7C046FFFFFF0F21
:1026A000F0B5DE46454657464E46724B8200E0B5D1
:1026B000D55800238DB00B909B4627E0069A079BC8
:1026C0001100194303D02B69002B00D093E02B6835
:1026D000DA7B002A07D051008A1819688C464946CF
:1026E0006244033A51704A46DA73EA684B469446AC
:1026F000013B63441A7801321A705B462B616B68A8
:10270000BFF35F8F5A461A6084F3108800F012FC02
:102710006A68EFF3108472B61368002BFCD0BFF325
:102720005F8F2B689C465B7B9946002B5BD0AA6829
:10273000514B90464B441B01984443461A685B68D2
:1027400016001F00361A8F41002F6EDD0B9800F027
:1027500053FC0022002300270026089209936B688F
:10276000BFF35F8F5A461A6084F31088002E76D02C
:10277000534618024B4639001843B0476A68069022
:102780000791EFF3108472B61368002BFCD0BFF3EF
:102790005F8F079B002B91DA2B69002B97D006984F
:1027A0000799089A099B121A8B4108980999069271
:1027B0000793079A914203D807D1069A904204D909
:1027C00001225242D317069207935B4601210493DC
:1027D0004B460391029301970096069A079B2800A7
:1027E000FFF7CEFE89E70022002300270892099315
:1027F00000260020B3E700F09DFB069A079B121805
:102800004B41994202D804D1904202D9012252424E
:10281000D31759460491012103914946019702912A
:1028200000962800FFF7ACFE67E7002F01D1002ECD
:102830008CD10021604600F023FD43461A685B6896
:102840000892099343469E68DF68EB684B44013B5E
:102850001B789A461B021843286100207FE7002856
:1028600000D053E70DB03CBC90469946A246AB461B
:10287000F0BDC046082A0020FFFFFF0F10B5124C24
:102880006368002B04D00A21104800F041FC10BD01
:1028900023000F4A1021206800F0D4FC032000F030
:1028A0003DFB032000F014FC0A49032000F05EFB0E
:1028B000FFF718FE084B9C46032360442375074B23
:1028C00080006060DC60DEE7E4140020242B002040
:1028D0001D250010A126001040000034082A002009
:1028E00000487047E4140020F0B54546DE465746E0
:1028F0004E46E0B585B00092019310AB1B78050001
:102900009B4600239A4698466A68EFF3108972B690
:102910001368002BFCD0BFF35F8F2E68B47B002CB4
:1029200050D067003F193368033FDB195A78B27300
:10293000002A00D1F27342469A705A701A70AA683F
:10294000534B94460099019AE3181B0163441960A4
:102950005A600E9A9A600F9ADA6042463368DB1921
:102960009A705A701A70737B0393002B40D0190031
:10297000736822009C46B068E047039932688C4631
:102980004B006344033B00282BD0D719D318B970F0
:102990001A78002A00D073E01C70039B73739C426A
:1029A00027D0EB681B19013B18786B68BFF35F8F6A
:1029B00042461A6089F310885346002B26D1000244
:1029C000204307E06B68BFF35F8F1C6089F31088BA
:1029D0000120404205B03CBC90469946A246AB4619
:1029E000F0BDD318D7199C703A78002A44D13970B9
:1029F0007473287D009A019B00F0FEFA824600283D
:102A0000CFD02100286800F0E7FCCAE75B46002B26
:102A100030D00E9B0F990020984703000B4329D01C
:102A200006000F1E15DA0098019902000B00921B98
:102A3000BB41994202D808D1904206D901235B429A
:102A4000DC1700930194DA465EE700920193DA46C0
:102A50005AE700F06FFA36184F4100960197B942D5
:102A6000ECD8F0D1B042EED901235B42DC170093E1
:102A70000194E8E70020ADE75A70039B3B70B7E78D
:102A80007A701C70039B73739C4200D089E7B0E797
:102A9000FFFFFF0FF0B557464E464546DE460400A1
:102AA000E0B50D0006267642F71736196F4185B05E
:102AB0008F4200D987E000D182E000F03BFA32007B
:102AC0003B00121A8B41002B00DC87E0674B9946D4
:102AD0005A68EFF3108B72B61368002BFCD0BFF36B
:102AE0005F8F4B461B6898469B7B9A46002B7BD09A
:102AF0005B0053444246033B9C46414612680093A8
:102B0000624453788B73002B00D1CB73002349466A
:102B10009370537013708968554A8C4652445549D6
:102B200012016244166057609160D360009942467A
:102B30008C461268624493705370137043465B7BFB
:102B40000393002B00D16FE01900404643465246E4
:102B50005B6880689847039B9C465A006244033A2E
:102B6000002854D0009940468C46036803999A186F
:102B7000634499701178002900D05970534613703E
:102B80004246039B53739A4551D04B465B68BFF353
:102B90005F8F00221A608BF31088BC46B046009409
:102BA000019500266546344F344A7B6A9D424CD8D5
:102BB000B96A414501D29D4247D0009C019D1BE06E
:102BC000864200D879E70026002700F0B3F93200EA
:102BD0003B00121A8B41002B00DD77E7002B0BD155
:102BE000002A00D072E707E04B465B68BFF35F8FB7
:102BF00052461A608BF310882000290000F0A6F9D5
:102C000005B03CBC90469946A246AB46F0BD434653
:102C10001968009B8A18CB185146917019780029C1
:102C200000D05170039A1A70434652465A734B466D
:102C30003200187D3B0000F0DFF90028A5D04B469C
:102C40005146186800F0C8FB9FE71168EFF3108049
:102C500072B60B68002BFCD0BFF35F8F1368BFF315
:102C60005F8F1E6080F3108820BF9EE7E414002071
:102C7000FFFFFF0F5125001000400540242B0020CE
:102C800070B5060000F056F9FA2204000D0092001B
:102C900000233000002104F053FB001969418D42EC
:102CA00005D901204042C117FFF7F4FE70BD8D42E7
:102CB000FAD18442F5D8F7E7F8B557464E46DE46D6
:102CC0004546664CE0B581460F006268EFF3108818
:102CD00072B61368002BFCD0BFF35F8F2668B57BFC
:102CE000002D00D19FE06B005B19033B9A463368CF
:102CF00053441A005B78B373002B00D1F3730023A5
:102D0000937053701370A168554A8C464946AA18AF
:102D10001201624411605349D36057609160326878
:102D20005244937053701370737B9B46002B6DD08D
:102D30002A001900B068736898475B465A005A44E5
:102D4000033A002857D0594633689A18534499706B
:102D50001178002900D059705B46157073735D457A
:102D600055D00026E36862685B19013B1B78BFF30E
:102D70005F8F0021116088F31088002E59D11B024B
:102D80001D4320BF6268EFF3108872B61368002BF2
:102D9000FCD0BFF35F8FFF232068E9B2427B2B405A
:102DA0008A4250D05A00924602689A44944652464B
:102DB0006244033A9278002A45D123699D4200D1AA
:102DC00022616368BFF35F8F00221A6088F3108866
:102DD000254A536A9F4207D8926A01264A4503D280
:102DE000FF1A7B1E9F41FEB230003CBC90469946C4
:102DF000A246AB46F8BD534631688A18CB18957089
:102E00001978002900D051705A461A707573207DC8
:102E10004A463B0000F0F0F8061EA2D029002068C8
:102E200000F0DAFA9EE76368BFF35F8F1D6088F3F6
:102E300010880D4A0026536A9F42D5D8926A0136FF
:102E40004A45CDD3D0E7E2682D0A94466344013B5E
:102E50001B78AB42B5D100F0BFFAB2E7E414002012
:102E6000FFFFFF0F5125001000400540F0B5C6469A
:102E700000B5EFF305833F22134018001038EFF33D
:102E8000108772B61F4D2A68002AFCD0BFF35F8FEF
:102E9000012211008140884644461B494C631B4C6B
:102EA0002678A4463400C440224007D1BFF35F8F88
:102EB0002A6087F3108804BC9046F0BD4C6A144920
:102EC000820051588C420FD3124BD25843469E4336
:102ED00063461E70BFF35F8F00232B6087F310885B
:102EE000002AE8D09047E6E70B4A9B0094466344EB
:102EF0001A681A60BFF35F8F00232B6087F3108876
:102F0000D9E7C046280100D000400540582C0020D9
:102F1000302B00204C240020D03F054010B501008C
:102F2000024A0348FFF758FA10BDC04680CB001094
:102F3000552C0020044A516A00E01900906A536A37
:102F40009942FAD17047C04600400540064A536A8C
:102F50009942FCD807D1044B02E05A6A914202D14F
:102F60009A6A8242F9D370470040054070B5040068
:102F70000D00EFF3108672B61A4A1368002BFCD0CE
:102F8000BFF35F8F002D1BD0200000F0FFFD16491E
:102F900088420AD0200000F001FE0121200000F04C
:102FA000DBFD0123A340114A1360114BA400E5503F
:102FB000BFF35F8F00220B4B1A6086F3108870BD41
:102FC0000B4BA200D5500122A2400A4920000B78E9
:102FD00093430B70044900F00BFE0021200000F029
:102FE000BBFDE5E7280100D06D2E001038600540DC
:102FF0004C240020582C0020F0B5D6464F464646BB
:103000002E4CC0B5656A00E00D00A66A616AA9424F
:10301000FAD1AB4248D9EFF3108972B6284C216837
:103020000029FCD0BFF35F8F264901268C46097822
:1030300086400F00884661463743FFB20F70041D7B
:103040001E49A400204D4E636250840063510D6AF6
:10305000002435421BD04D6A00E025008C6AA24650
:103060004C6AAC42F9D1AB4224D801D1524521D8A7
:10307000474521D0114B154A1E625E631F2318403D
:103080001E3B834013606346424601241A70BFF31F
:103090005F8F00220A4B1A6089F3108820001CBC45
:1030A00090469946A246F0BDAB4201D1B242B2D899
:1030B0000124F3E70024EAE70124E8E700400540A3
:1030C000280100D0582C0020302B002080E200E0A6
:1030D00010B5EFF3108472B60A490B68002BFCD0D0
:1030E000BFF35F8F01238340074A084813620278C9
:1030F0009A430270BFF35F8F00230B6084F3108844
:1031000010BDC046280100D000400540582C0020CA
:10311000024B9C46614489000160704740000034C6
:1031200010B50400FFF7DEF901002000FFF7F0FF03
:10313000FF232371BFF35F8F10BDC04610B504009D
:10314000FFF7D0F901002000FFF7E2FFFF23A38083
:10315000BFF35F8F10BDC04610B504000120FFF71C
:10316000CDF9044B9C46604480002060BFF35F8F24
:1031700010BDC04640000034F8B54746CE4680B585
:103180004C0003686418033C1A19567807000D00B8
:10319000002E04D128000CBC90469946F8BD710061
:1031A0008919033988464344597889460021597062
:1031B0005170002D11D07B6832002900806898473B
:1031C0003B68002832D01A1943449D7011780029B9
:1031D00000D059701670A04600E035004B46002B19
:1031E000D8D049463800FFF7C7FF041ED2D00200EE
:1031F0007B682900B868984763001B19033B3A684D
:10320000002809D1D318424494701978002900D0BD
:1032100051701D702500BDE74146D31851189D70AF
:103220000A78002A00D05A700C70B3E742461C1985
:103230009A18A6701378002B00D0637015703500B3
:10324000CCE7C04610B583600023CCB24373013392
:10325000047342608373C4730068012C06D9421C56
:103260000133DBB2137003329C42F9D8FF231940BB
:103270004B005918002340180338437010BDC04656
:10328000F0B54E4657464546DE46E0B5467B0368F8
:103290007400A419033C1A19177883B005008946F5
:1032A000002F1ED1002911D0C07B00282AD0410058
:1032B0000918591803394E70EE73002F06D07900A3
:1032C000C91903398846002143449970002330000E
:1032D00053706F7303B03CBC90469946A246AB4610
:1032E000F0BD7900C91903398846591848788246D3
:1032F000002809D149460029E5D0E87B0028D6D12D
:10330000EE73DCE7EE73E1E742005244033A934682
:103310005B445A78019200225A704A706B6802002E
:103320003900A86898472B68002830D1414650469C
:103330005A4659189A1888701078002800D048709A
:103340001770D8465746019A002A2DD01100280040
:10335000FFF712FF8246002825D0020039006B6873
:10336000A868984753465900514403392B680028F0
:103370001CD04246591898188F70027894461A1932
:103380006446002C00D04C7051460170B2E759469B
:10339000424659189A188F701078002800D048704B
:1033A00051461170CFE72B681A19A3E75A189844B1
:1033B00093465046424690705A461278944660466C
:1033C0001A19002802D04046644644705846884680
:1033D000077057468EE7C046F0B54546DE4657466D
:1033E0004E46E0B50C0083B005000023002927D02D
:1033F0006600477B01683619033E8819A74233D01F
:103400008278002A1CD053009B18033BCB181A78F3
:10341000A2421FD142781A70002302788370437051
:103420009146002A33D1EA7B002A66D053009B18CC
:10343000C91803394C70EC730023437001236F7378
:10344000180003B03CBC90469946A246AB46F0BD7E
:10345000002AE1D053009B18033BCB185A78A242B4
:10346000F6D142785A70D7E702780192002A46D105
:10347000EA7B002A3FD053009B18C91803394F70CC
:10348000EF7300234370019B6B730123D8E7520055
:103490004A44033A90468A185778002F42D1EB7B72
:1034A000002B00D029E14F466E7BEC730023937014
:1034B0004370002EC2D03A006B683100A86898476C
:1034C00073009B19033B2A68002808D0D318424494
:1034D0009670197800290CD11F703700AEE741466D
:1034E000D31851189F700A78002A00D05A700E70B5
:1034F000A4E75170F0E7EF73C3E7EC739CE71400A7
:10350000A44652006244033A90468A185478A14671
:10351000002C58D1EB7B002B00D0F7E0EF73002399
:103520009370AEE77800C01903388246514448785A
:103530004B7053706B6883463A004946A8689847B9
:103540002B68002800D1A2E04246981852469918EC
:103550004A468A70019002000078002801D0019A42
:10356000487017704F465A46002A28D059462800FE
:10357000FFF702FE8146002820D002006B68390068
:10358000A86898474B465B004B44033B9C46002889
:103590006DD042462B689818624699188F7001903A
:1035A0000078002800D083E04A4601980270E97B49
:1035B00098196E7B002951D1019A76E72B68424613
:1035C0009A180192F3E76000484403388246514458
:1035D00048784B7053706146220083466B68A86838
:1035E000644698472968002878D0524643468A188E
:1035F000CB1894701878002800D050704A46C24604
:103600001A705B46002B50D059462800FFF7B4FDD6
:103610008046002848D0019C020021006B68A86801
:10362000984743465A004244D31E2968002844D094
:103630005246CB188A189C701078002800D0587019
:1036400043461370EB7B8819002B00D166E75E00C0
:10365000F318C91803394F70EF7360E74A009446B6
:1036600061445B18033B5C70019AEC731EE72968A8
:103670004846CA184346CB18987010788046881977
:103680004646002E00D05E701770E04607E74146C0
:10369000524659189A188F701078002800D0487038
:1036A0004946D04611705EE729685346CA18C9E7F3
:1036B0004A46487001990A7079E7CA18534640464D
:1036C000CB1898701078844664468819002C00D076
:1036D0005C70019B1370434601931BE75346CA1865
:1036E00043464846CB1898701078002800D0587090
:1036F000019B13704B46019383E703267343C9185C
:1037000003394C706E7BEC734F46CFE60326734350
:10371000C91803394F7001E72D4B2E4A70B51A6056
:103720002D4A2E4B2E491A6010008B689843FBD10E
:103730002C4C2D4DAC4209D20322231D0335ED1A2A
:103740009543ED1808CC9847AC42FBD100F09AF8AD
:10375000264A224B1A60224A9368DB018033FBD150
:103760004022234B2348244D9A675A671A67DA662A
:10377000A84205D30EE0FFF7E1FC2000AC4209D2DD
:10378000040003680834002BF5D1FFF7C9FC2000C2
:10379000AC42F5D3194D1A4CC022A168280003F0A1
:1037A00041FEA560FEF790FE00F05CFBFFF766F8B7
:1037B000144C154DAC4209D20322231D0335ED1ADA
:1037C0009543ED1808CC9847A542FBD170BDC04683
:1037D00000E00040BFCDFBFEFE7F3C0000F000405B
:1037E00000C00040081E0020181E0020FFFFFF013F
:1037F00000F00140001E0020081E002000000020F4
:1038000000ED00E0181E0020281E002000BEFDE78D
:10381000094A1368002B06D008491818884208D8AE
:10382000106018007047064B04491818136088424E
:10383000F6D901235B42F4E7F825002000000420BC
:10384000202F002000BEFDE70FB400B5084883B06C
:1038500003F00AFF049B002B07D005A91800019173
:1038600002F0ECFE034803F0FFFE00BEFDE7C04699
:10387000B0CB00100CCA001010B50148FFF7E4FFF0
:10388000A4CB001030B50C2083B000F04FFBFEF746
:1038900013FE00280ED0964B964A1A605A609A6022
:1038A000DA601A615A619A61DA611A62924A5A625E
:1038B00003B030BD914CA06700F08CFB0122904B0F
:1038C0001A60636C012BFCD103228E4B1A608B4A69
:1038D000936B012BFCD1022405338B4A01218B48C9
:1038E000009400F0D1FA0523894A00940121894807
:1038F00000F0CAFA884B5A68FF2A02D88022520088
:103900005A6080227A4C7F4B21691201824D1A60E5
:10391000002900D0E5E0E0217F4B02201A68114029
:10392000802252012A431160196848400321014056
:10393000116004219A681142FCD0802280219201FA
:103940002A4309011160802252005A60734B23619F
:10395000734B5968FF2900D8C1E00322684B7048B7
:103960001A60012103009A681142FCD0E0251A6810
:10397000154080225201024315601B684B40032111
:10398000194011600221664A93681942FCD08023D5
:1039900080219B010343090119608021614B49008B
:1039A00051606361604B5A68FF2A00D859608022D9
:1039B0005E4BE16912015C4D1A60002905D0606917
:1039C00002F0B2FE01300138FDD1E02256490B6809
:1039D0001A4080235B012B431A60802380229B01C5
:1039E0002B4312011A608022424B52004A60E3616D
:1039F0004F4B5968FF2900D85A6080224D4B216AED
:103A000012014B4D1A60002905D0606902F08CFE4E
:103A100001300138FDD1E02245490B681A4080236E
:103A20005B012B431A60802380229B012B431201F0
:103A30001A6080235B004B602E4B3F4A23623F4B52
:103A40005968914201D801325A6080223C4B616A28
:103A500012013A4D1A60002905D0606902F064FE37
:103A600001300138FDD1E02234490B681A4080232F
:103A70005B012B431A60802380229B012B431201A0
:103A80001A608023DB024B601B4B63622D4B5A682C
:103A9000FF2A02D8802252005A6080222A4BA16954
:103AA0001201284D1A60002905D0606902F03CFE21
:103AB00001300138FDD1E02222490B681A408023F1
:103AC0005B012B431A60802380229B012B43120150
:103AD0001A6080235B004B60124BA361E8E65A60DA
:103AE0003BE7606902F020FE01300138FDD112E7AA
:103AF00060250020006CDC021BB700000080004045
:103B00003CB0004030B00040002F685900800240B7
:103B100000389C1C00C0024030800040001BB700F1
:103B20003C800040405973075480004054B000402E
:103B30006080004060B00040FFFF03006C800040E8
:103B40006CB000404880004048B00040014B80000D
:103B5000C05870476025002001238340002902D10E
:103B6000034A13607047034A1360034A1360F9E77E
:103B700080E100E080E200E000E100E0012383401A
:103B8000014A13607047C04600E200E0024B10306B
:103B90009B688000C058704700ED00E070B50D00D4
:103BA000EFF3108672B60F4A1368002BFCD0BFF3F8
:103BB0005F8F0D4B10309B6884001B590B4A93425A
:103BC00003D09D4201D0FFF757FE074B9B681D5164
:103BD000BFF35F8FBFF35F8F0022024B1A6086F343
:103BE000108870BD240100D000ED00E0CD01001070
:103BF000F0B54546DE4657464E46E0B50D0083B06B
:103C0000EFF3108A72B65D4A1368002BFCD0BFF345
:103C10005F8F1022914681444A46594B96009B681B
:103C20009C59584B98469C4205D0AC4251D0564FB7
:103C3000E31B2F2B12D9524B9B689C51BFF35F8F14
:103C4000BFF35F8F00224D4B1A608AF3108803B0D8
:103C50003CBC90469946A246AB46F0BD012383404A
:103C60009B465A46494B1B681A4000925A46484B9D
:103C70001A60BFF35F8FFCF7F6FA0190002803D0BB
:103C8000814501D0FFF7F8FD012322009A43414B03
:103C900006209C4613006146DB1B5B415943090D1E
:103CA00093688C4610569D420AD151E043001B1880
:103CB00006209B00FB1899681856A94211D01A00DB
:103CC0000028F3DA009B002B05D15A46304B1A60CE
:103CD000B1E71C00AFE75A462F4B1A602B4B1A6016
:103CE000A9E7002825DB4200111889007D188846C5
:103CF000A9689960E979D971062169569971A979FC
:103D00007F2913D8AD88F91A6D052D154544491939
:103D1000E0250905490D2D022943998012181F4BF2
:103D20009200BF181A781870BA71CBE7BD2109024A
:103D3000F3E70199002913D1002A0FD0FF209071D9
:103D400017489080154A1078987163461370B9E748
:103D500013000028C7DA019A002A01D14446F1E78E
:103D6000104A1149D21A083A5002400D0143998075
:103D70000E4952080A43DA80A4E7C046240100D065
:103D800000ED00E0CD0100100C15002000E100E086
:103D900080E100E0AAAA000080E200E0562C0020AA
:103DA00000BDFFFF4615002000F0FFFF00F8FFFFF9
:103DB000F8B5012504000543FCF755FAEFF310862A
:103DC00072B6214A1368002BFCD0BFF35F8F1F4BE4
:103DD0001F4A2100C91A49414A43120D1D4980005A
:103DE0008F6852B23F58AF421CD0062159569142BB
:103DF00026D012215956914224D01E215956914263
:103E000014D02A2159560320914210D0124B197810
:103E10001A70A171BFF35F8F00220B4B1A6086F3FB
:103E20001088F8BD8B680D491950EFE7022041005A
:103E3000091889005B18FF21997109499980E5E704
:103E40000020F4E70120F2E7240100D00C15002047
:103E5000AAAA000000ED00E0562C0020CD010010C1
:103E600000BDFFFF054B064A1360064A136053600E
:103E70009360D36013615361936170478080808049
:103E800000E400E004E400E0F8B504000C201E00AB
:103E900017000D0002F048FC4201121A9101891A24
:103EA000C90009188901380002F03EFC069B36045F
:103EB0001B031E432368002B21DB184BE2185342DF
:103EC0005A4180235B019C4652421A40144B624483
:103ED0001A60144B1A60144B170099688F43FBD17A
:103EE000C023221D9B01134321222560A0601A607C
:103EF0002268002AFCDA0822E6601A60F8BD3F2337
:103F000022681340AB42D8D1A3681B051B0D834226
:103F1000D3D1E368002ED0D1F0E7C0460040FDBF0A
:103F200000E0004000F0004000C0004080239B0003
:103F30001843014BD86270470080054010B58024BB
:103F40001B4BE4051C6000281AD00123194C1843B0
:103F5000194BDC61194C44401C6259629862802103
:103F6000134BC9051960164816490860E021C904B9
:103F70001960002A07D18022134B12061A6010BD67
:103F80000D4BD861EBE753019B1A9B009A180F4B1E
:103F900012019A4208D80E4B1A60074B5A608022D1
:103FA000094BD2051A60EAE7094A13601A00F4E7E0
:103FB00000B00540D3C007B0008005402D3FF84F4A
:103FC000FCFF01000820014000A00540FFFFFF00AA
:103FD000002A0020AA23064A1B0113602F2305494B
:103FE000D360054B19605368002BFCDA7047C0465C
:103FF0000040024000B0FA00006002407047C04636
:1040000010B5002803D04A680B681100984710BD0E
:1040100010B5002801D003F0D7FA10BDF0B557460F
:104020004546DE464E46E0B585B0984610AB1D7855
:10403000139B93469A460223149A0F0013400600DE
:104040000F9C12990193002B2DD1013313409C46F4
:104050005346002B66D18C420DD21F2C00D912E1A1
:104060000E9B30201B1902E00133202C03D00134B9
:104070001870A142F8D86346002B14D0A24512D97B
:104080000E9B30201B191F2C21D8AC461500524620
:1040900002E00133202C17D0013418709442F8D17B
:1040A00092462A006546D3062ED5530519D4002C16
:1040B00011D1119B102B00D1D9E0022B1FD10E99E9
:1040C00060330B7001241AE092462A006546D3063D
:1040D0003ED5530505D4A14200D19FE0544500D1FF
:1040E0009CE0119B102B65D0022B06D11F2C65D8AC
:1040F00062210E9B1B19197001341F2C5ED83021D0
:104100000E9B1B19197001341F2C57D8002D1BD181
:10411000530700D570E0130750D520230E990B5597
:10412000013415E06346002B6BD0002D00D070E009
:104130000C2313426DD18C42A0D21F2C90D9534630
:104140002024202BC3D8AEE72D230E990B55013424
:10415000930736D05B4603931A000E9B0294994650
:104160004B46013C551C185D39004346B0472A00B8
:10417000002CF5D1039A029B944663441D00019BD9
:10418000002B0FD05B46EB1A53450BD22A005D463D
:10419000541C434639002020B0472200631B53457E
:1041A000F6D32500280005B03CBC90469946A246AF
:1041B000AB46F0BD930641D51F2C52D95D469307FF
:1041C00012D1544538D25B4653441B1B0F941C003C
:1041D0000F9B5A469946551C434639002020B0474C
:1041E0002A00A542F7D14C46002CC8D00E9B03955F
:1041F00002942A009946B3E72B230E990B550134FC
:10420000A6E78C4200D34EE71F2C00D828E72024D5
:1042100049E701235B429946CA448CE7631E002BA1
:1042200015D1119B102B19D0022B00D147E7302359
:104230000E9901240B7069E75D46D5E71F2C00D964
:1042400086E778210E9B1B191970013455E71199E7
:10425000023C1029AED01C000B0045E793060DD59B
:10426000002458210E9B1B191970013445E7930651
:1042700004D558230E9901240B7040E778230E993A
:1042800001240B703BE72024F5E6C046F0B5454617
:10429000DE4657464E46E0B59BB09846259B249C8B
:1042A0001D00089009910A920C930022002320001F
:1042B00029000B9402F0EEFC002800D0A7E10B9A35
:1042C0000C9B92469B468023289ADB001A400E9254
:1042D00001D1062326938023289A1B011A405646B3
:1042E0005B460D92334300D161E15B465800CC4BF5
:1042F000400D9C46604402F0FBFCCA4ACA4B02F0E7
:1043000086FCCA4ACA4B02F05BFC5B46C94A1B03E7
:104310001B0B1A4304000D00C74B1100504600222E
:1043200002F045FCC54AC64B02F071FC02000B00CE
:104330002000290002F044FC02F0F2FC814602F069
:10434000D7FCC04AC04B04000D0002F060FC002204
:10435000BE4B02F035FC02F0E3FCBD4A0600BD4B4B
:104360002000290002F053FC040030000D000F96DD
:1043700002F0BEFCB84AB94B02F049FC02000B0047
:104380002000290002F013FC02000B0006000F00C1
:1043900002F03DFC320004000D003B00300039000B
:1043A00002F00EFC002210901191AD4B200029006C
:1043B00002F00FFC0022AB4B02F002FC02000B00EB
:1043C0002000290002F005FC0022A74B02F0F8FBB8
:1043D00002000B002000290002F0FBFB0D008021F1
:1043E000040032003B000020C90502F0E0FB02009F
:1043F0000B002000290002F0E3FB02000B001098E4
:10440000119902F0E6FB00228A4B02F0D9FB974A91
:104410000F9B9446634400221B0502F0F8FB050045
:104420000C0002000B005046594602F033FC0028F5
:104430000BD001235B429C46280021000022894BBF
:10444000E14402F0C6FB05000C004B46C626633370
:104450009E42B6410D9B76420436002B00D0BCE054
:10446000279B00279E4200D29F1B0223289A1A40B6
:104470000D9203D0734273415B421F404B46002BA9
:1044800007D0504659462A00230002F0A2FB82467C
:104490008B46002200230B980C9902F0FBFB0028AE
:1044A00003D08021090659448B4652465B4650464C
:1044B000594602F00AFC002800D044E101226C4B6E
:1044C00052425046594602F0E5FB002800D0D7E0A2
:1044D000289A684B039713400493269B52460293F5
:1044E0005B4609990092019308980A9A434600F0A6
:1044F000FFFC0200002E52D02020289B089C034085
:1045000059424B415B421840531C45309A46099929
:104510004346A0474B46DA179D18DB0F9946731E9A
:1045200055409B46002412AE02E03C00202F0DD0E7
:1045300028000A2102F0F8F8671C30313419217084
:1045400028000A2102F0F0F8051EEED1052306939B
:104550005B460593002304930A3303934B4601976C
:104560000096099F089E0293524643463900300048
:10457000FFF754FD0D9B0200002B10D00A99431A3F
:10458000279898420BD989460500434639002020D8
:10459000541CB0474B462200E31A9D42F5D8100048
:1045A0001BB03CBC90469946A246AB46F0BD0D9B65
:1045B00055465C46002B27D000239946269B4B4549
:1045C00000DDB1E0002326938023289ADB001A4304
:1045D000002328920026994642E723002B43EDD082
:1045E000254A264B5046594602F062FB002800D06F
:1045F0009FE0269B002B00D132E70E9B5A1E934171
:10460000269AD31A26932BE70426994628E7802278
:10461000120694460C9BA24663449B4653E6C04652
:1046200001FCFFFFFB799F501344D33FB3C8608B5D
:10463000288AC63F0000F03F0000F83F61436F63E7
:10464000A787D23F71A379094F930A400000E03F4A
:104650001655B5BBB16B0240EF39FAFE422EE63F6C
:1046600000002C400000244000001840FF03000020
:10467000FFFFEFFFFFF7FFFF2D431CEBE2361A3F72
:104680000A9A289B14009B0715D1042F13D9B24610
:104690004646151FED19BB46099F0B95330039009F
:1046A0002020089D541CA8470B9B22009C42F5D15A
:1046B000B0465F4656464D4B49469A464346B94634
:1046C00022000425A346B0461F000B915346013D2E
:1046D000541C585D09993B00089EB0472200002DEC
:1046E000F4D13B005C460B9A464698460D9B4F46DC
:1046F0009146221D002B00D1FCE60A9BD31A9F4253
:1047000000D8F7E6B3464646BA46099F330039005B
:104710002020089D541CA8470A9B2200E31A9A45B2
:10472000F4D8B0465E46E5E64A469B1A013B26931E
:104730004AE700222E4B5046594602F0ABFA0028B9
:1047400000D03BE755E70A9B289A9A46920717D173
:10475000032F15D9B2461A004646DC1EE419BB46A3
:10476000099F0B94330039002020089C551CA0475A
:104770000B9B2A009D42F5D1B0465F465646AA469D
:104780001C4B49469B464346B94652460324B04615
:104790001F000B915B46013C551C185D09993B00BD
:1047A000089EB0472A00002CF4D13B000B9A4F46DC
:1047B00091465246464698460D9B0332002B00D147
:1047C00098E60A9BD31A9F4200D893E6B346464622
:1047D000BA46099F330039002020089D541CA84781
:1047E0000A9B2200E31A9A45F4D89AE7A4CD001058
:1047F00080842E41A0CD0010F0B5DE4657464E46CF
:104800004546E0B597B005000E0093461F00209A7C
:10481000219B1000190002F058FA002800D0AEE2E7
:10482000209821990122C54B524202F033FA002808
:1048300000D034E1209821990122C14B524202F06C
:104840003FFA002800D0C1E0209821990022BD4BFA
:1048500002F036FA002800D008E1209821990022C1
:10486000B94B02F017FA002800D0FFE020982199F8
:104870000022002302F00EFA002800D074E2002388
:104880000D938023249ADB001A40904600D0BAE1B1
:104890000023AE4C069307940EAB06249A4620984C
:1048A000219902F03DFA099002F022FA02000B0071
:1048B0002098219902F07BF9069A079B02F0A7F94C
:1048C0000A900B9102F050FA81460C9002F00CFA1B
:1048D00002000B000A980B9902F069F900229C4B28
:1048E0000A900B9102F0ECF9002800D1E5E14B466B
:1048F000013318000C9302F0F7F9069A079B02F0B7
:10490000D7F9002800D0FBE1002C00D09CE1099CE5
:10491000200002F0EDF902000B002098219902F02E
:1049200046F900228A4B0690079102F0B3F900285D
:1049300000D1D5E14346202B00D112E15C1C099B3C
:104940000A211800994601F0C7FE4246534630310D
:10495000995448460A2101F0BFFEA046814600282E
:104960001ED05346A846BA464D461F00B14600E049
:104970003400202C00D162E228000A2101F0ACFEB4
:10498000661C30313C19217028000A2101F0A4FE78
:10499000051EEDD13B0045465746B0469A464E4669
:1049A0000323249A1340012B00D1B1E14246202475
:1049B000202A00D1DCE00D9A002A00D135E24246DF
:1049C0005146541C40462D220A54D1E0249B5B07DB
:1049D00000D5ADE05F4B9A46032398465B460693AD
:1049E000249B9B0718D1239B434500D84EE25B4490
:1049F0001C004346E41AB9465A4637002E002500EB
:104A0000541C4B4639002020B0472200AC42F7D15D
:104A100035003E004F460694B14644465646BA46D7
:104A20002F00069A013C551C305D53464946B84755
:104A30002A00002CF6D1069B3D0043441A00249B1B
:104A40009B0724D55B462399D31A99421FD92E0080
:104A5000D0464F460D00434639002020541CB04735
:104A60005B462200E31A9D42F5D810E0249B5A468B
:104A70000493239B31000393229B28000293209BE5
:104A8000219C009301943B00FFF700FC0200100002
:104A900017B03CBC90469946A246AB46F0BD249B5D
:104AA000D8469B0718D1239B042B15D95B461C1FA6
:104AB000239BB8469C46644437005A462E00250086
:104AC000541C434639002020B0472200AC42F7D1A5
:104AD00035003E004746A0461F4BB94642463700C8
:104AE00004249A462E005346013C551C185D39009B
:104AF0004B46B0472A00002CF5D14246249B350096
:104B000004323E009B07C2D55B462399D31A9942D3
:104B1000BDD93700C8462E000D004346390020207D
:104B2000541CB0475B462200E31A9D42F5D8AEE71D
:104B30000A4B9A460423984650E7C046FFFFEFFF12
:104B4000FFFFEF7F65CDCD4165CDCDC180842E4186
:104B50000000E03FB4CD0010A4CD0010ACCD00109B
:104B6000A2460323249A1340012B00D1CEE0202437
:104B7000D846002B17D1239B9C4214D25B441B1BAD
:104B8000B8465A463700A1462E001D00541C434625
:104B900039002020B0472200AC42F7D135003E005A
:104BA0004746A0464C4643464246A146B8463700D3
:104BB0002E0006935346013C551C185D39004346B0
:104BC000B0472A00002CF5D106994B468C46634429
:104BD0001A00249B35003E009B0700D457E75B4634
:104BE0002399D31A994200D851E737002E000D00BF
:104BF000434639002020541CB0475B462200E31A8C
:104C00009D42F5D843E7229B092B00D85BE10EAB10
:104C10009A4630235246137001229046229B2F322F
:104C20005C1E4146203B504605E0013C42540131A8
:104C30009C4200D1EEE0092CF7D10022A84B884617
:104C40008246069207932AE64346202B89D0631EAC
:104C5000069301230C9C434420000A21994601F04D
:104C600063FD534642463031995420000A2101F039
:104C70005BFD041E00D122E1A84625004C46B94642
:104C80005746B24612E0069B2800013B0A210693D4
:104C900001F04AFD661C30313C19217028000A21C0
:104CA00001F042FD051E00D1CFE03400202CEAD1F6
:104CB00056464546BA464F4653E700220A980B9996
:104CC000884B01F0E7FF002800D01DE60C9B002B6D
:104CD00002D0DB0700D417E60C9B01330C9313E6DC
:104CE0000022069807997F4B01F0EAFF002800D0C8
:104CF00020E60123A44623409C446346099319E619
:104D0000099B0133099300230C93FDE5202398466A
:104D1000239B002B00D1BFE00D9B002B03D1249AD5
:104D20000C33134202D0239B013B2393239B434527
:104D300000D8B1E042463023202A00D1B1E04246FB
:104D400050462399541C83548C4200D1A1E0220088
:104D5000202CF7D1202399465B46B846824637007F
:104D600006935A462E0025E7209A219B0020002119
:104D700001F01DFF0123209021910D9381E5249BDB
:104D8000D8469B0718D1239B032B15D95B46DC1E05
:104D9000239BB8469C46644437005A462E002500A3
:104DA000541C434639002020B0472200AC42F7D1C2
:104DB00035003E004746A0464B4BB94642463700B9
:104DC00003249A462E005346013C551C185D3900B9
:104DD0004B46B0472A00002CF5D14246249B3500B3
:104DE00003323E009B0700D451E65B462399D31A59
:104DF000994200D84BE63700C8462E000D004346C6
:104E000039002020541CB0475B462200E31A9D4223
:104E1000F5D83CE6354BE2009B181A685B680692B1
:104E2000079320238246984639E5249A52073BD5BA
:104E300042465146541C40462B220A5498E63B00F9
:104E4000454657464E469A468BE64546B046564638
:104E5000BA464F464346202B00D182E6069B404689
:104E60001A004244110054463022002B29D0431C22
:104E70002254202B00D173E618008B42F7D1A246B2
:104E80005A1C904651462E22CA5453E55B4606935F
:104E9000C2E5239B8246984642460123202A00D041
:104EA00089E52024D8467EE6249A4446120700D499
:104EB0005EE620225146404601340A5458E6C84670
:104EC000C8E74346DCE7DA00084B9B185C681B68C0
:104ED00006930794002398460EAB229C9A46DEE484
:104EE00065CDCD410000E03FA0CD0010B8CD001051
:104EF000F0B557464E464546DE46E0B597B00792B8
:104F0000012206000F002098219998465242CF4B6B
:104F100001F0D6FE00284DD0249B5B0700D541E16F
:104F2000CB4B9A4603239B46079A249B14009B076E
:104F300011D1239B9B450ED2190013008C4663446C
:104F40001D005B46ED1A541C434639002020B04733
:104F50002200AC42F7D1B946220037005D465646E2
:104F6000A246013D541C705D43464946B8472200A5
:104F7000002DF6D15246249B3E005A444F469B07D3
:104F800010D507992398531A98420BD989460500E2
:104F9000434639002020541CB0474B462200E31AF8
:104FA0009D42F5D8100017B03CBC90469946A246E9
:104FB000AB46F0BD002220982199A64B01F080FE5F
:104FC000002800D0F3E0209821990022A24B01F0A4
:104FD00061FE002800D0EAE02098219900220023F9
:104FE00001F058FE002800D092E100230D938025A7
:104FF000249BED001D4000D017E10023974C08933F
:1050000009940EAB06249B462098219901F088FE56
:1050100081460C9001F06CFE02000B002098219953
:1050200001F0C5FD089A099B01F0F1FD0A900B9172
:1050300001F09AFE824601F057FE02000B000A982A
:105040000B9901F0B4FD0022854B0A900B9101F001
:1050500037FE002800D148E101239C46E244504637
:1050600001F042FE089A099B01F022FE002800D0C0
:105070009CE1002C00D006E10C9C200001F038FEE1
:1050800002000B002098219901F091FD0022744B41
:105090000890099101F0FEFD002800D176E1202D55
:1050A00000D1BAE00C9B0A211800994601F014FBCC
:1050B0005B463031595548460A2101F00DFB6C1C06
:1050C0008146250000281AD04D46BA46B1465F46B3
:1050D00000E03400202C00D103E128000A2101F077
:1050E000FBFA661C30313C19217028000A2101F0BE
:1050F000F3FA051EEDD13500BB464E465746032355
:10510000249A1340012B00D10EE12024202D0BD036
:105110000D9A002A00D034E1249A520700D46FE19E
:105120002B2259466C1C4A55079A1500002B12D1A8
:10513000239B9C420FD2190013008C4663441B1B17
:10514000A1461C00551C434639002020B0472A00C8
:10515000A542F7D14C46A246A9462A005B46013C2F
:10516000551C185D39004346B0472A00002CF5D184
:105170004B4653441A00249B9B0700D412E707991F
:105180002398531A834200D30CE78946050043460F
:1051900039002020541CB0474B462200E31A9D42A0
:1051A000F5D8FFE62F4B9A4604239B46BCE6209A8F
:1051B000219B1000190001F088FD00281AD12098C9
:1051C00021990122284B524201F064FD002811D19F
:1051D000249B079A0493239B39000393229B30005E
:1051E0000293209B219C009301944346FFF74EF8C5
:1051F0000200D7E6249B079A0493239B390003936C
:10520000229B30000293209B219C009301944346F3
:10521000FFF7F2FA0200C5E683460323249A1340FF
:10522000012B00D17FE020247EE7229B092B00D8B0
:10523000F2E00EAB9B4630235A461370229B0125A9
:105240005C1E3022203B594615E0C046FFFFEF7F31
:10525000B4CD001065CDCD4165CDCDC180842E414A
:105260000000E03FACCD0010FFFFEFFF013C4A55CE
:1052700001359C427BD0092CF8D100226C4B8B4627
:1052800008920993C0E6202DC7D06B1C50460A2116
:10529000994601F049FA5B463031595550460A218A
:1052A00001F042FA013C8246002800D1B2E04B46B0
:1052B0005546B146BA465F4611E09B4628000A2192
:1052C0005E1CBB4401F030FA5B4630311970280097
:1052D0000A2101F029FA013C051E76D03300202B6B
:1052E000EBD1BB464E46574697E700220A980B99EA
:1052F000504B01F0CFFC002800D0BAE65346002BFB
:1053000002D0DB0700D4B4E601239C46E244B0E6B9
:10531000209A219B0020002101F049FC01232090CC
:1053200021910D9363E62025239B002B46D00D9BF6
:10533000002B03D1249A0C33134202D0239B013B50
:105340002393239BAB4239D93023202D3AD05946A1
:10535000239A6C1C4B5594422ED02500202CF8D15A
:105360002023079D8B469A46A9462A00F6E6324B33
:10537000E2009B181A685B688B4608920993202507
:1053800042E62D2259466C1C4A55CDE6002208986B
:105390000999284B01F094FC002800D07FE60123F6
:1053A000A44623409C4463460C9378E64B46013365
:1053B0000C9300239A465CE68B46239D0123202D07
:1053C00000D0A5E62024079DC5E63500BB464E4625
:1053D0005746202D00D120E7611930222B00002CE8
:1053E00009D058466B1C4255202B00D114E71D00F4
:1053F0008B42F7D183462E2259465D1CCA544EE695
:10540000249A2C00120700D48EE62022594601343B
:105410004A5589E64D46DCE7DA00074B00259B1824
:105420005C681B68089309940EAB229C9B46EBE5D5
:1054300065CDCD410000E03FB8CD0010F0B5DE46AF
:1054400057464E464546E0B5A9B01E00329B9046F1
:105450000A93BF4ABF4B83468A461A60002968D028
:10546000D1460025DA46307800280BD001362528B1
:105470001BD02A0043464946D04730786C1C250093
:105480000028F3D1D3462A00CA46454501D34346F6
:105490005A1E434651460020D847280029B03CBC3C
:1054A00090469946A246AB46F0BD102330789B4605
:1054B0000E3B9C460300203B721CDBB20027A64C2F
:1054C0001100102B0DD89B00E3589F4601231600B6
:1054D0001F433078721C0300203BDBB21100102BFD
:1054E000F1D90300303B092B00D8AEE100239B46E5
:1054F0002A2800D1CFE100242E2800D1BDE10300ED
:10550000683BDBB2122B00D9D3E3944A9B00D358FB
:105510009F46042316001F43DBE7634616001F4324
:10552000D7E75B4616001F43D3E7082316001F4347
:10553000CFE78B4B9B4693E780235B0070781F433C
:105540004E1C0300253BDBB2532B92D8854A9B00AF
:10555000D3589F4670786C2801D100F0C0FC80239E
:105560005B001F434E1CECE780239B0070781F43B9
:105570004E1CE6E77078682801D100F019FD802301
:105580004E1C1F43DDE7462801D100F058FC0722DE
:105590000A9B049707339343013294469C44624626
:1055A0000A925A46029403925C681B682A00009390
:1055B0000194494643465046FFF71EF9050052E75D
:1055C0002A006C1C434649462520D04725004AE75F
:1055D0000A9B1A1D1B680C920A931878002C00D0A5
:1055E000ABE3002801D100F0A2FF02211A004942DA
:1055F00001239C46434608900B9307E00A986346B4
:1056000080469B1A43445B18002B03D00132137869
:10561000002BF3D10B9B089898460A9BD31A08934A
:105620008023DB003B400B9303D0089BA34200D9AF
:10563000089402231F4001D100F0DBFC002801D1B7
:1056400000F0BCFC0B9B002B01D000F062FE0A9B1B
:105650002A005C1B23005446B2464E46B9464746D4
:1056600098463B003100551CA0474346585D2A0030
:105670000028F6D1B8464F46B1465646A246002FFE
:1056800001D000F09BFC0C9B0A93ECE60A9B1A1DD0
:105690001B689346002B00D142E3212217430A974F
:1056A0000F2020A90B940022089184460C0002E0F0
:1056B00020290CD00A0061461940CFB2380037309B
:1056C000092900D80738511CA0541B09F0D10B9CA4
:1056D0000A9B019106930823059308330393002343
:1056E0000293089B2A00009304944346494650467F
:1056F000FEF794FC5B4605000A93B4E60A9B6C1C1B
:1057000004330B940893BB0700D478E30A9B2A0068
:10571000187849464346D0475B465D44012B01D883
:1057200000F07EFE2B0057464D46B1464646984651
:105730000B9A541C330029002020B847220044450E
:10574000F7D1B046BA464E46A946250073E3C04697
:105750003D540010FC290020C0CB001004CC0010E8
:10576000FD3F001050CC0010782800D1ECE2582802
:1057700001D100F067FC6F2801D100F051FD6228D3
:1057800001D100F04FFE10233A009A430B92692892
:1057900001D000F039FF7B0501D500F02BFD8023FF
:1057A0009B001F40F73BFF3B0C93002F01D000F004
:1057B000C3FC80230B9A5B001A40130094460A9A9C
:1057C00004320D92002B01D000F0CAFD0B9B5B064A
:1057D00001D400F0BCFD0A9B1B78DA1798185040E2
:1057E000DA0F0A92002B08D10B9A1033110099435B
:1057F0000B91520501D500F0A2FE0B9B61279B0681
:1058000000D541275A4620ABFFB20E950F94B34600
:1058100008930A3F644610920C9D1E000CE0303342
:10582000DBB2621C3355002801D100F017FC202A9E
:1058300001D100F013FC1400290000F075FFCBB279
:105840000929ECD9DB19DBB2EBE70023010001E009
:10585000160001329800C01840004018117803006B
:1058600008003038303B0928F2D908009B46B11CAB
:10587000002416002E2800D041E680237078DB003B
:105880001F430300303B092B15D92A2800D1DAE247
:105890000E00013133E60A990B1D09688B46002979
:1058A00004DA02210F43594649428B467078B11CF5
:1058B0000A9316001FE6030000E03100A000001963
:1058C0004000C0184B7830381A00303A4E1C0400A3
:1058D000092AF2D91800023111E6202302009A4366
:1058E000472A02D180231B011F43022398434528E6
:1058F00001D11E331F4307220A9B07339343013212
:1059000094469C44624619685868089109900A9226
:1059100003000A000B910C900898099901F0D5F941
:10592000002800D09BE20122E34B52420B980C99D5
:1059300001F0C6F90122E14B5242002800D0D5E225
:105940000B980C9901F0A6F9002800D0A2E30022E0
:1059500000230B980C9901F09DF9002801D000F06C
:1059600055FD0B9A0C9B08920D938023DB003B4066
:10597000179300D1062480230D9A1B013B400E9300
:10598000130008990F910B4301D100F0B6FCCC4BEA
:1059900050009C46400D604401F0AAF9C94ACA4B28
:1059A00001F035F9C94ACA4B01F00AF90D9A109075
:1059B00011911303C74A0F991B0B1A431B921A919B
:1059C00000221A981B99C44B01F0F1F8C34AC44B4A
:1059D00001F01DF902000B001098119901F0F0F888
:1059E00001F09EF90F9001F083F9BE4ABE4B109072
:1059F000119101F00CF90022BC4B01F0E1F801F02B
:105A00008FF9BB4ABB4B16901098119901F0FFF823
:105A100010901191169801F06BF9B74AB74B01F04D
:105A2000F6F802000B001098119901F0C0F802007E
:105A30000B001090119101F0EAF814901591109854
:105A4000119902000B0001F0BBF800221E901F917B
:105A500014981599AA4B01F0BCF80022A94B01F04B
:105A6000AFF802000B001498159901F0B2F800226B
:105A7000A54B01F0A5F802000B001498159901F050
:105A8000A8F8109A119B1490159180210020C90547
:105A900001F08DF802000B001498159901F090F8B0
:105AA00002000B001E981F9901F093F80022894B09
:105AB00001F086F8169B1A00944B9C46624413052D
:105AC0001D9300231C931C9A1D9B01F0A0F81490B9
:105AD000020016910B0008980D9901F0DBF80028E0
:105AE0000AD00F9B1498013B0F9316990022854B07
:105AF00001F06FF814901691C6230F9A6332934207
:105B00009B415B42043310930E9B002B1DD0169BD0
:105B1000149A134301D100F0C1FC7D4A7D4B0898D3
:105B20000D9901F0C5F8002809D000227A4B089899
:105B30000D9901F0AFF8002801D000F0AFFC002C67
:105B400003D0179B5A1E9341E41A00230E93109B17
:105B50009B4502D95A46D31A0E9302233B40179312
:105B600006D0109B5A4253410E9A5B421A400E9245
:105B70000F9B002B07D008980D99149A169B01F0E3
:105B800028F808900D91002200230B980C9901F041
:105B900081F8002805D08020000684460D996144D4
:105BA0000D910D99089A0B00089801F08EF80028C5
:105BB00001D000F0E2FC0122404B524208980D99BE
:105BC00001F068F8002801D000F075FC534B089AEA
:105BD0003B4004930E9B029403930D9B4946009215
:105BE000019350462A004346FFF782F90200109BBA
:105BF000002B00D170E1202007403B0059424B416F
:105C000000275B42511C18400B91434649464530E2
:105C1000D0470F9A109BD117013B54180D93D20F08
:105C200020AB0E954C403D000C9208930F961F0040
:105C300002E03500202E0DD020000A2100F074FD76
:105C40006E1C30317D19297020000A2100F06CFD96
:105C5000041EEED1052306930D9B3200059300230D
:105C600004930A3303930C9B01920293089B0B9AB3
:105C700000934946434650460E9D0F9EFEF7CEF9CF
:105C8000179B0200002B00D126E1431B9B4500D847
:105C900022E15C465746531C9A464946434620201B
:105CA000B8475246531B9C42F5D8BA461500FFF739
:105CB000DAFB0E0045E4C046FFFFEF7FFFFFEFFF7A
:105CC00001FCFFFFFB799F501344D33FB3C8608BA7
:105CD000288AC63F0000F03F0000F83F61436F6331
:105CE000A787D23F71A379094F930A400000E03F94
:105CF0001655B5BBB16B0240EF39FAFE422EE63FB6
:105D000000002C400000244000001840FF03000069
:105D10002D431CEBE2361A3F80842E41FFF7FFFF34
:105D2000102239009143113211430A917A0500D4AF
:105D3000B6E420AB00210893CAE4002801D100F0AA
:105D4000F6FB611E1A0053E480231022DB003B4067
:105D50000C920C2297430B973A00002B02D00123A0
:105D60009A430B9280270B9BBF001F40692800D1EC
:105D70001BE5642800D118E5002F00D07CE28023C9
:105D80000B9A5B001A40130094460A9A04320D9253
:105D9000002B00D050E30B9B5B0600D445E30A9B2D
:105DA0001878002807D10B9A1023110099430B9102
:105DB000520500D5BFE30B9B61279B0600D5412709
:105DC00020ABFFB20A950E940F9608930A3F6546E2
:105DD0000C9C1E000AE03033DBB26A1C73550028AD
:105DE00000D111E2202A00D10EE21500210000F0BE
:105DF0009BFCCBB20929EED9DB19DBB2EDE75B46A0
:105E0000012B00D8A7E36B1E9B4433005E469B46E4
:105E100001E02500013443462A004946202027009E
:105E2000D047B442F5D15E4602350A9B3A00187855
:105E300049464346D047089B0A93FFF714FB2023AB
:105E40001F43FFF7A4FB0A9AB0781468F11CE343E0
:105E5000DB171C40131D0A930236FFF750FB2C0082
:105E6000BB0710D15B46032B0DD9EC1E23002A0083
:105E70005B440893434649462020541CD047089B66
:105E800022009C42F6D103230893DC4B22000B93A3
:105E90002B003D001F00089B0B98511C013B0C91EF
:105EA0000893C05C49464346D047089B0C9A002B98
:105EB000F2D13B002F00E21C1D00BB070CD5531B89
:105EC0009B4509D95F46541C434649462020D0478C
:105ED0002200631B9F42F6D81500FFF7C4FAC023C7
:105EE0009B00B0781F430336FFF72BFB0B980C99F0
:105EF00000F0D0FE002800D0CCE07B0700D46BE29D
:105F0000BF4B089304230C930B95BB071CD10C9B30
:105F10009B4500D82DE35A465419E41A33002A0051
:105F20004E46A94655469A460D97571C43463100A2
:105F30002020A8473A00BC42F7D15346AA464D4616
:105F4000B1461E000B970D9F330056469A460B9A9A
:105F50000C9C0D95089B013C551C185D4946434619
:105F6000B0472A00002CF5D153460B99B2468C4617
:105F70001E000C9B0D9D63441A00BB07ACD5531B40
:105F80009B45A9D933005C464E4657469946531C5B
:105F90009A46310043462020B8475246531B9C4244
:105FA000F5D84B46BA46B14615001E00FFF75BFA1E
:105FB000C023B0781F430336FFF7C3FA089B9B4505
:105FC00001D8FFF760FB5A465419E41A33002A003F
:105FD0004E46574699460135434631002020B84782
:105FE0002A00A542F7D14B46BA46B1461E00FFF73C
:105FF0004AFB089A531C934500D8A8E25B465B19FC
:106000009B1A08971F0033002A004E46A1465446AB
:106010009A460135434631002020A0472A00BD4260
:10602000F7D15346A2464C46B1461E005B460133AB
:10603000089F08930A9B1878002801D0FFF702FBFD
:10604000FFF721FB0C233A009A4314331A430B92B7
:106050007B0500D4C7E010230C9380E6109B5E46BE
:106060009B460E9D0F9C0B9B049406935B460593E9
:106070000C9B03930A9B0293089B019200932A00B6
:10608000434649465046FDF7C9FF0D9B05000A935C
:10609000FFF7E9F90B95BB071BD15B46042B00D832
:1060A000B0E233002C1F2A004E46A94655469A46B8
:1060B0005C440897571C434631002020A8473A000B
:1060C000A742F7D15346AA464D46B1461E000B974C
:1060D000089F4C4B0424089333004E46B94657465C
:1060E0009A460B9A0C95089B013C551C185D310093
:1060F0004346B8472A00002CF5D15346BA464F46CE
:106100000B9AB1460C9D1E000432BB0700D4E3E697
:10611000531B9B4500D8DFE633005C464E4657468E
:106120009946531C9A46310043462020B8475246B0
:10613000531B9C42F5D834E707220A9B073393434D
:10614000013294469C4462465F680A921A68FB17C3
:1061500018931993189819990300534012930B0040
:106160007B4013939446129A139B121A8B411292FE
:1061700013936246FB0F14933A4307D10B9A1023F3
:10618000110099430B91520500D5E7E10B9A612369
:10619000920600D54123DBB220AA0A3B0E950F944C
:1061A00010960027129C139D08920D930C9E0CE0F4
:1061B0003032D2B2089C7B1CE255020004000D0074
:1061C0000A433FD0202B3DD01F0032000023200087
:1061D000290000F0EBFAD2B2092AE9D90D9B9C46BE
:1061E0006244D2B2E6E780239B001F40F13BFF3BB5
:1061F0000C93C1E50A230C93B1E5C046A0CD001075
:10620000ACCD0010A4CD00100A9D0E9C0F9E0B9BE0
:10621000049406935B4605930C9B039300232AE7A3
:1062200008230C938023DB003B40642800D090E5DA
:106230003A000B97002B00D091E58027BF00174054
:10624000FFF7B3FA12941395109E0F9C0E9D0B9AB4
:10625000049406925A4605920C9A01930392149A5A
:106260000292089B2A000093494643465046FDF798
:10627000D5FE0500FFF7F7F807220A9B0733934383
:10628000013294469C44624603CB03000A920B43BE
:1062900007D10B9A103317009F430B97520500D577
:1062A00063E10B9A6123920600D54123DBB220AA59
:1062B0000A3B0E950F94002708920D930C9C1096A4
:1062C00015000CE03032D1B2E95518007A1C3100CB
:1062D000334300D185E0202A00D182E0170022005C
:1062E000002300F063FAD2B203000E00092AE9D9B4
:1062F0000D998C466244D1B2E6E70E9B002B00D08C
:10630000C7E00D9B149116930423109300230F9361
:106310001BE40A9B64195B1B0A9333002A004E4658
:10632000B94657469A4608E043463100551CB847DF
:106330000A9B585D002862D02A00A242F4D153463D
:106340001500BA464F46B1461E00FFF798F90B9B61
:106350001B0600D4F7E00A9B00229B5EFFF73DFA84
:106360000A9B1B68DA1798185040DA0F0E92002B20
:1063700006D10B9A1033110099430B9152051FD48B
:106380000B9A6123920600D54123DBB220AA0A3B77
:1063900008920A9309E03033DBB208997A1CCB5596
:1063A000002810D0202A0ED017000C9900F0BCF95C
:1063B000CBB20929EFD90A9A94466344DBB2ECE7E1
:1063C000002220AB08930B9B049406935B46059335
:1063D0000C9B03930E9B4EE68D4B089303230C936B
:1063E00092E50E9D0F9C109E0B9B049406935B46BA
:1063F00005930C9B019203930023029331E75346CC
:10640000BA464F46B1461E00FFF739F98022120600
:1064100094460B9B08930C9B63440D93FFF7A5FADE
:10642000250008E502230C93FCE60B9B1B0600D419
:1064300098E00A9B1888B4E40A9B1868002806D1E3
:106440000B9A1023110099430B91520573D40B9AA8
:106450006123920600D54123DBB220AA0A3B0892B1
:106460000A930BE03033DBB208997A1CCB55002835
:1064700000D1CCE6202A00D1C9E617000C9900F023
:1064800053F9CBB20929EDD90A9A94466344DBB299
:10649000EAE70D9B1491169300230F930F9B9C42E8
:1064A00057DDE41A013C8023DB001F4300231093D7
:1064B0000F93FFF74AFB0B95BB070FD10E9B042BE5
:1064C00059D99C462A002C1F6444531C0B934946FF
:1064D00043462020D0470B9A9442F6D104244D4BDA
:1064E0000B9A08930C97089B013C571C185D494672
:1064F0004346D0473A00002CF5D10B9A179B0C9FCE
:106500000432002B01D1FFF772FB0E99531B8B4213
:1065100001D3FFF76CFB434649462020541CD0476B
:106520000E992200631B8B42F5D3FFF760FB00231B
:106530000893FFF775F820AB0022089367E620ABBD
:10654000002208938FE50A9B1B68FFF746F9089322
:1065500072E50024A7E72F00250066E420AA0023A7
:10656000089274E60A9B18681BE420AB002208938B
:106570003AE70B95E8E40B95B0E72C00BB0710D188
:106580000E9B032B0DD99C462A00EC1E64440894F4
:10659000434649462020541CD047089B2200A34272
:1065A000F6D1032308931C4B22000B932B003D00D4
:1065B0001F00089B0B98511C013B0C910893C05C79
:1065C00049464346D047089B0C9A002BF2D13B002A
:1065D0002F001D00179BE21C002B01D1FFF707FBCA
:1065E0000E99531B8B4201D3FFF701FB43464946EB
:1065F0002020541CD0470E992200631B8B42F5D3F8
:10660000FFF7F5FA0B9564E5063B17000C9309E6D6
:10661000B4CD0010A4CD0010A0CD001000B585B001
:106620000391012102900093034813004A4202A9FA
:10663000FEF704FF05B000BD0140001010B5094A87
:1066400084B01468002C09D001220091030052424A
:1066500003A90548A047012004B010BD01F004F8CB
:106660000020F9E7FC290020114000100148042116
:10667000014B1847601500209D660010142310B5CB
:106680000100188804331B88984710BD162310B5E5
:106690000100188802331B88984710BDF0B5C64624
:1066A00000B5002916D014230400012598461827A8
:1066B000890046184346216818883B88984701C4DA
:1066C000431E984140420540A642F3D1280004BC35
:1066D0009046F0BD0125F9E7124A936F9B0815D249
:1066E0009066D166002905D0FFE7FFE7FFE7516F0D
:1066F000106F704704B580210906C2175140002869
:1067000000D0C84306F040F8002104BDF0B5146E77
:10671000556E576F166FFFF7E3FF146655665767A0
:106720001667F0BD000000D0114A936F9B0813D28A
:1067300010665166002905D0FFE7FFE7FFE7516FBC
:10674000106F704704B5002801D00020C04306F048
:106750001BF8002104BDC046F0B5146E556E576F8E
:10676000166FFFF7E5FF1466556657671667F0BDAD
:10677000000000D094464E4A926F9208624601D2C1
:1067800030E0C046F0B54A4EB56F6D08FCD3346EAC
:10679000756E776F366F00F025F89446444A14669C
:1067A0005566576716676246F0BDC0469446404A34
:1067B000926F9208624601D258E0C046F0B53C4E56
:1067C000B56F6D08FCD3346E756E776F366F00F061
:1067D0004DF89446364A1466556657671667624602
:1067E000F0BDC046002B24DB11D000293EDA00B5F5
:1067F000C943404200D1013100F038F8C94340425A
:1068000000D10131DB43524200D1013300BD002AE7
:10681000EBD1002801D1002905D00020C90FC907FC
:1068200001D1C043410800B505F09EFF00220023BE
:1068300000BD00B500290ADBDB43524200D1013321
:1068400000F014F8C943404200D1013100BDC943F2
:10685000404200D10131DB43524200D1013300F00C
:1068600005F8DB43524200D1013300BD002923D19A
:10687000002B18D1002A0CD0BC460D4F38667A6622
:1068800000210023FFE7FFE7FFE77A6F386F6746D5
:106890007047002801D00748010000B505F064FFEB
:1068A0000022002300BD02000B00002000217047E1
:1068B000000000D0FFFFFFFF002B00D0BFE0130C53
:1068C00028D1002AE7D080B4114F39667A66FFE7F5
:1068D000FFE730B4040C7B6F396F1B0423433B6626
:1068E0007A66FFE7FFE7FFE7C04684B27B6F3D6F44
:1068F0001B0423433B667A66FFE7FFE7C04600239D
:106900002C042D0C7A6F386F00196941B0BC7047A8
:10691000000000D0F0B594460025140E01D11202FB
:106920000835140F01D112010435940F01D19200E2
:106930000235D40F01D152000135D40B0134254F5B
:106940007C66254C3C660E0C93B2FFE7FFE7FFE741
:106950003C6F6643360C7703BE467343DF0B5B0424
:10696000C01AB941130C7343DB18C91ACE08664329
:10697000360CB64493B273431F0F1B01C01AB941C2
:10698000130C73431F0B1B05C01AB941860D8F02F0
:106990003E436643360C092D24DB520A7243801AAB
:1069A0007703460A6643360C16235B1BDE40DF4046
:1069B000BF1964466643821B7046043506330100E6
:1069C000D940A840C01900D30131A24206D2002309
:1069D000F0BD0000000000D0FFFFFFFF121B0130E0
:1069E000F3D3F1E709277F1BFE406446A2B272434E
:1069F000801A00D20139220C7243130C1204821A3D
:106A000099410B007046043513370100F940A84046
:106A1000801900D30131002B02D1A2420AD2F0BD6D
:106A2000013000D30131121BFAD2013BF8D1A2424E
:106A300000D2F0BD013000D30131121BF7E7F0B5F1
:106A40001C0C00D080E00CB400251C0A04D11B02F1
:106A5000160E3343120208351C0B04D11B01160F0E
:106A60003343120104359C0B04D19B00960F334332
:106A700092000235DC0B02D192185B4101351C00FB
:106A8000971864410134464F7C66464C3C660E0CB8
:106A9000FFE7FFE7FFE7C0463C6F6643360C77032E
:106AA000BE4697B27743C01B00D20139C01B00D24B
:106AB00001399FB27743C91BC91B170C77437E046A
:106AC000FF0B801BB941CE086643360C0C2D33DB1F
:106AD000B644120B1F053A431B0B97B27743C01BFA
:106AE00000D201399FB27743C91B170C77433E048C
:106AF0003F0C801BB941860D8F023E436643292718
:106B00007F1BFE400C3D7746AF40BF1930BCA2B2A0
:106B1000ABB272437343801A9941220C7243130C37
:106B20001204801A994102000B000137001BA94191
:106B3000F9D2781E0021F0BD0C277F1BFE4077465E
:106B40007F0BAF40FF19E0E700245D1C07D0144F16
:106B50007D663966FFE7FFE7FFE7FFE73C6F95B229
:106B60009EB265436643401BB141150C1E0C654344
:106B7000664336042F0C3E432D04401BB14199421D
:106B800004D202000B0020000021F0BD01D1904290
:106B9000F7D3801A994101349942F2D3F6E7000005
:106BA000000000D0FFFFFFFF48404140484018B4BC
:106BB0001B4B5B68FC46019308BD04DF136E00109D
:106BC00018B4174B1B68FC46019308BD00DF1D6E0F
:106BD00000109446134A926F920809D2624618B484
:106BE0000F4BDB68FC46019308BD0CDFD57000102D
:106BF0000C4AF0B5146E556E576F166F6246FFF76C
:106C0000EEFF084A1466556657671667F0BD18B45C
:106C1000034B9B68FC46019308BD08DF796F0010A9
:106C20005C2C0020000000D0FFB550404240504096
:106C300059404B40594000E0FFB5154F4C00640DE2
:106C400003D0BC4204D10C0314D80020090D09055F
:106C50005C00640D03D0BC4204D11C030AD800229E
:106C60001B0D1B0501264B4009D44B4003D58B421D
:106C700000D18242FFBD9942FCD19042FFBD0B433F
:106C8000DB1803431343F5D0C9434918FFBD000087
:106C9000FF07000000B5FFF7CFFF804100BDC046F1
:106CA00000B5FFF7C9FF01D9002000BD012000BDDC
:106CB00000B5FFF7B9FF01D9002000BD012000BDDC
:106CC00000B5FFF7B1FF804100BD012040054A003B
:106CD000121804D85A00121801D800207047012059
:106CE00070470020704700000021002805D1704740
:106CF000C1174840401AFAD0C90713B5064B1B68A4
:106D000098470CBC441CA2401005120B0349091BF8
:106D100009051943114310BD202B00201F0400005A
:106D200010B54C00620D8023D218DB00D21A5B052F
:106D30007E2A10DD9E3A13DACC170903490819435D
:106D40005242D140640001341532202A05DAD04085
:106D50000843604310BD002010BD0846604310BDCD
:106D6000C80FC018013810BD18B4044B5B6AFC464C
:106D7000019308BD24DF8572001000005C2C002008
:106D8000132370B51C78012C11D01ADD0F48FFF7C2
:106D90007DFC0F4D01008022280000F043FB022CF7
:106DA00010D00C48FFF76AFC0B4B186070BD084D03
:106DB0000A4A29002B00803104C38B42FCD1AA640B
:106DC000EFE7034D054AAA64EBE7C04653440000D1
:106DD0005C2C00204C330000202B0020E16D0010C3
:106DE00007B5604601880A0A0230DF2AFAD1C9B223
:106DF000820804D3028840880004104300E0006841
:106E0000014A5050039007BD5C2C00200FB403BC16
:106E10000CBCF0B50124E407634000E0F0B50C0DB4
:106E2000CF0F661E3605891B640503D3C943404254
:106E300000D30131640D03D0661CF60A07D0E41BB1
:106E400000207F00791C89078912803C24031D0DD6
:106E5000DF0F6E1E36059B1B6D0503D3DB435242CD
:106E600000D301336D0D03D06E1CF60A07D0ED1B65
:106E700000227F007B1C9B079B12803D2D032F1B54
:106E8000661B58D4A446202E46DA20371400BC4096
:106E90001D00BD40F24033412A4380185941CB0FB9
:106EA00005D0C943C043002264425041514162466B
:106EB0004D0D28D10D0D07D100281FD024194041B8
:106EC0004941013A0D0DF9D0640006D3013000D3D9
:106ED0000131002C01D140084000013A0BD4941C30
:106EE000E40A04D112051144DB071944F0BDD907A7
:106EF000204B194300E0D9070020F0BD0029DDD167
:106F0000002CDBD1F0BD0132C6074008CD07284375
:106F10004908002EE1D0D9E73C2E29DA203E40373F
:106F20001400BC4000D00124F24014431A00BB40BE
:106F30001C43D317ACE7AC46202F08DA20360400F8
:106F4000B4400D00B540F84039412843A5E73C2F37
:106F50000CDA203F40360400B44000D00124F84051
:106F600004430800B1400C43C117EAE710001900C0
:106F7000002494E70000F07FF0B50C0D661E360586
:106F8000891BE60A6405640D02D0651CED0A04D075
:106F9000002001210905803C2403A4461C0D671E26
:106FA0003F05DB1BE70A6405640D02D0651CED0A92
:106FB00004D0002201231B05803C24037740644455
:106FC00097B484B296B27443070C7E43150C6F439A
:106FD00080B26843361802D3012000043F18300401
:106FE000350C00197D41844688B29AB250430C0C8E
:106FF00062431F0C7C438EB27E43921902D301265A
:107000003604A4191604170C3618674101BC81B266
:107010009AB25143040C62431B0C5C4380B2584348
:10702000121802D30120000424181004130C401875
:1070300063412D185E410020474106BC88B293B2DF
:1070400058430C0C6343120C544389B251435B18F0
:1070500002D301210904641819041A0C09186241A9
:107060006D1856410020474118BCF902720D1143BA
:10707000F0026A0D1043ED020A0D03D16D19404173
:107080004941013B124E9B1B7600B3420ED26D006C
:1070900007D30130002671416646354301D14008CF
:1070A00040001B05C918E4072144F0BD0BDA013389
:1070B00006D1013004D101314F0D01D04908F2E76A
:1070C000E1070020F0BD013631050020EBE70000AC
:1070D000FF030000F0B51C0D671E3F05DB1BE70A30
:1070E0006405640D02D0661CF60A04D00022012358
:1070F0001B05803C2403D0252D060026F6432E6672
:107100001E096E66CE0FF619B44649004F0D02D027
:107110007E1CF60A03D000200021403F3F033E1BA7
:10712000B600B444013F7F05C91B49082E6F0136E4
:1071300076089C02950D25437543ED137543AD13F9
:1071400001356D10F603761B0CB4CC02450D2C43B3
:10715000A2B2B3B25A43270C7B43350C6F43A4B29F
:107160006C431B1902D3012424043F191C041D0C79
:10717000A4187D4124196D41009A91B2ACB26143CB
:10718000170C7C432B0C5F4392B25A43A41802D3D2
:1071900001221204BF182204230C52187B41019CC7
:1071A0006C431B19520ED9010A434401A01A81B243
:1071B000B2B2514303145A43360C734387B2774338
:1071C000D617D21900277E4136049B191704160CD6
:1071D0007F185E417316ED18F30100268033754168
:1071E000A90F06D16400690AE8055B0A184309D2B1
:1071F0002FE00422944480337541A90AA8059B0A14
:10720000184326D3404149412404009A019B0D00B4
:107210005543641B4343E41A95B286B27543170C79
:107220007E43030C5F4392B25A43B61802D3012245
:107230001204BF183204330C52197B4152429C4154
:10724000002C02D40022013051414008CA071043EB
:10725000490802B06246D7079210084BD218084B73
:107260009A4203D212058918C919F0BD0020002ADC
:1072700001DC3900F0BD01331905F5E7FD0300001D
:10728000FE070000002200B5203200F004F80800DC
:1072900000BD000000220B150AD410B5944600F082
:1072A00031F81414013400DA0021CB17144C2047B4
:1072B0000020002170476244343A0CD40C2A07DACB
:1072C00004009140904052422032D440214310BDEE
:1072D000D843D94310BD203207D40C4694405242C3
:1072E00020321141D040204310BD0800C917203280
:1072F00003D452422032104110BD1800190010BDB5
:10730000B77200100A0DCC0F531E1B05C91A520587
:1073100003D3C943404200D30131520D03D0531C63
:10732000DB0A07D0121B00206400611C8907891248
:10733000803A1203014BD21A70470000FF0300008D
:1073400051434343C9188C46110C83B24B4310B4CC
:10735000040C614392B280B2504362431C041B0C84
:10736000001910BC59411304120CC018514161445A
:1073700070470000132310B51C781348FFF786F9F7
:10738000012C0BD004DD01008022104800F04AF8E7
:107390000F48FFF773F90F4B186010BD0B4C01003D
:1073A0005422200000F03EF80B4B6365A365E365B3
:1073B00023666366A366E36623676367A367E36781
:1073C0002362E361E4E7C046534600005C2D0020E1
:1073D0004C330000202B0020DD73001007B5604601
:1073E00001880A0A0230DF2AFAD1C9B2820804D31E
:1073F000028840880004104300E00068014A5050B1
:10740000039007BD5C2D002001480421014B184763
:10741000701500209D660010014B1B681847000086
:1074200070150020014B5B681847000070150020A4
:10743000F0B5C64600B5437C06000C001500002BD5
:1074400006D1036811002000984704BC9046F0BDA7
:10745000002AFADD0A78037C00200A2A2CD00121B8
:10746000012D1BD0184B984602E03900BD4215D0C3
:107470004B1EE25C635C4F1C0A2BF6D10D2AF4D044
:107480003368884203DA091A2018984733680221C2
:107490004046984738003900BD42E9D1854203DDB6
:1074A000291A3368201898476419013C23780D3B4A
:1074B0005A4253413374C8E7002BD0D1024802210D
:1074C000336898470120CAE768CE0010F0B54F46F0
:1074D000D6464646314BC0B51C680700002C1BD071
:1074E0002F4B98462F4B9A4602E0E468002C13D0AD
:1074F0002368002BF9D042461268002A01D0A2422C
:10750000F3D1627C3D1D3E68002A0CD13100280079
:107510009847E468002CEBD100233B601CBC9046EC
:107520009946A246F0BD002EDFDD3979227C00208D
:107530000A292BD00121012E03D119E049464E45DD
:1075400016D04B1EEA5C4B1C99466B5C0A2BF5D19E
:107550000D2AF3D02368814203DD091A28189847C1
:107560002368022150469847484649464E45E8D18F
:10757000864203DD311A236828189847AD19013D6A
:107580002B780D3B5A4253412374AEE7002AD1D1E8
:107590000448083998470120CCE7C046F025002070
:1075A000F425002068CE00100B6870B505000C00B3
:1075B000802B04D05A1C2260E418257170BD08008D
:1075C000FFF784FF2368F5E7F0B5CE46474680B560
:1075D00083B06B46DD1CD02328701B061C681F4B34
:1075E000804601A91800994605F0D6F8071E2DD14E
:1075F000019B64B29C4224D0484605F0F5F8184B34
:1076000001271C68002C25D0164E07E00122290016
:107610002000FFF70DFFE468002C0AD02368002B40
:10762000F9D03368002BF1D0A342EFD0E468002CEE
:10763000F4D1002F0ED1404603B00CBC90469946C1
:10764000F0BD074B1C68002CDED1F4E7044B1C682E
:10765000002CD9D1484605F07FF8ECE7001E002049
:10766000F0250020F4250020F0B5DE4657464E46B2
:107670004546E0B583B0070004F0E8FED02301AD35
:107680001B06060029002F481C6805F085F8824675
:10769000002849D1019B64B29C423FD0294805F0A3
:1076A000A3F8294B9B461C6801239A46002C40D026
:1076B000264B98460A2399460EE0320039002000F6
:1076C000FFF7B6FE4B460122290020002B70FFF782
:1076D000AFFEE468002C0BD02368002BF9D04346A2
:1076E0001B68002BE9D0A342E7D0E468002CF3D15B
:1076F0005346002B1DD15B461C68002C06D06368E6
:10770000002B1AD09847E468002CF8D1300003B061
:107710003CBC90469946A246AB46F0BD0A4B1C685D
:107720009B46002CC4D1F1E7074B1C689B46002CFC
:10773000BED1044805F010F8DDE7E468002CDED186
:10774000E4E7C046001E0020F0250020F4250020BC
:107750000D4B1A68002A12D0824203D109E09842E8
:1077600007D01A00D368002BF9D1002900D0D060CF
:1077700070470029FCD1C368D360C160F8E70029D5
:10778000F6D01860F4E7C046F0250020F0B5C646F4
:10779000D02300B51F4EA2B01B060700884630005C
:1077A00001A91C6804F0F8FF051E07D1019B64B213
:1077B0009C4203D0300005F017F8013584220021E7
:1077C00001A8FFF729FE43463A0001A91248FEF737
:1077D00025FF019B0700002B18D1104B1C68002CC3
:1077E00006D06368002B0DD09847E468002CF8D1D0
:1077F000002D02D0300004F0AFFF380022B004BCEE
:107800009046F0BDE468002CEBD1F1E701A8FFF74A
:107810005DFEE2E7001E0020A9750010F0250020A3
:107820000FB400B583B004A901C90191FFF7AEFF01
:1078300003B008BC04B0184710B500F035F910BD0E
:107840007047C0460022014B1A707047572C002029
:10785000012070474B790020FF2B00D070478B79B7
:10786000002BFBD1CB79012BF8D1082AF6D98A78E5
:10787000014B09301A70F1E7572C002070B5002930
:1078800015D115495379107909781B02034300205B
:10789000994200D070BD5378012B0AD0022BF9D148
:1078A000002064220021FCF749FB0120F2E70120BF
:1078B000F0E7D478917824020C430500E20502D564
:1078C000620A93401D000548FEF7D8FE7F210300A1
:1078D000214028009847C046572C00205542000000
:1078E00001230370004870476CCE00104A780B7873
:1078F00012021A438B7810B51B041A43CB781B066F
:1079000013439622D200934200D010BD0348FEF7E5
:10791000B5FE0021030008009847C046554200000C
:1079200070B5184C82B005000E00200001A904F0CB
:1079300033FF002808D1D0231B061B68019A9A4206
:107940001CD0200004F050FF002001F049FE002868
:1079500007D103256D42200004F0FEFE280002B08E
:1079600070BD002001F054FE0028F2D02900320042
:10797000002001F05BFE051EEBD0ECE703256D4215
:10798000ECE7C046282B002010B51F20FCF7F6F8C6
:10799000FA200021800010BD10B5064C0021200007
:1079A00004F0FAFE002804D000F074FE200004F079
:1079B000D3FE10BD282B0020F0B546464F46D646D4
:1079C000C0B5364F82B080460E00380001A904F0E1
:1079D000E3FE00280ED1D0231B061B68019A9A42B1
:1079E00005D102B01CBC90469946A246F0BD3800B5
:1079F00004F0FAFE002001F0F3FD002832D000244C
:107A0000002E34DD264B99469A4612E0002843D1D9
:107A100000F040FE002001F089FE002001F0E0FDB2
:107A2000002824D0002001F0BDFE002823D0A6426B
:107A30001DDD0020351B01F0B5FE8542E6DC434626
:107A40002A001919002001F029FE050000F022FE8D
:107A5000002001F06BFEFBF76DFA4B4664191860CD
:107A60005960E4E7002000210D4B18605960380090
:107A700004F072FEB5E7FBF75DFA53460D001A6895
:107A80005B6800218446074812184B419D42EED89E
:107A9000CDD19445CBD9EAE70500D0E7282B0020CB
:107AA000281F002020A1070010B51D4B84B01B78B3
:107AB00002F08AF81B491F20FCF770F801211F20F3
:107AC000FCF74AF81848FBF72BFBFAF709FF04000C
:107AD000FBF730FAFA220023920012184B41994228
:107AE00018D901225242D31701210291002101919C
:107AF0000E4920000091FAF7F7FE0400631E9C4136
:107B0000E4B2002803D001210948FFF721FE20003C
:107B100004B010BD9942E7D19042E2D8E4E7C046F4
:107B200084D3001099790010282B00208979001047
:107B3000801500200048704724CF0010004870478F
:107B4000D0CE001070B5040016480378002B20D06A
:107B5000002C06D1C1241448144BA4004380048097
:107B600070BD052C1CD8124B0F48A400E558811C91
:107B7000002304E001330A800231132B0DD0EA5CAC
:107B8000DCB2002AF6D1C023013464009B001C4300
:107B9000E5E7112102F0A0FADAE7CA24A400DEE743
:107BA0000020DDE7402C0020C8250020090400004B
:107BB00038CF0010F0B55746DE464E46454698236E
:107BC0008024E0B56B4A6402D75883B0274228D09E
:107BD00001222321684B00205A54DA70674901F0D2
:107BE000B3FA8022664B92021A65664B9A46FB06F0
:107BF0001CD480235B011F424AD18023DB011F423A
:107C000000D08DE080231B021F4200D096E0BC42D2
:107C100000D0AAE003B03CBC90469946A246AB46D1
:107C2000F0BD102300249A46FB06E2D5514B9B6D14
:107C30009846002B27D0524B00249B46012399469F
:107C400043460126B8461F0004E001347600E4B242
:107C5000202C17D03E42F8D05B469E654B46650807
:107C6000A3436D00ED18444B6D019C46654428000C
:107C700000F08CFB00286CD10134B743E4B27600ED
:107C8000002FE5D1474680235B0154461F42B4D004
:107C90001C430023374A00211360384A3A48936056
:107CA000D3603A4A9360D360394A9360D360394ACB
:107CB0009360D360384A9360D360384A9360D3604E
:107CC000374A9360D360374A9360D360364A9360F3
:107CD000D360364A9360D360354A9360D360354AA7
:107CE0009360D360344A9360D360344A9360D36026
:107CF000334A9360D360F0229200FFF78DFB314B43
:107D0000314A00211A600020012201F0F1F980229D
:107D10001B4B12031A658023DB011F4200D171E760
:107D20000122042100201C4301F050F91022144BC1
:107D30001A6580231B021F4200D168E7012205213A
:107D400000201C4301F042F980220D4B12011A65FC
:107D50005DE74B46AA8AA97800200093002301F032
:107D60001BFA280000F03AFA86E72100174879400C
:107D7000FBF76AFD00001150FC25002000001050A8
:107D800000301150100001003C2600200800105067
:107D900010001050180010502000105028001050F3
:107DA0003000105038001050400010504800105063
:107DB00050001050580010506000105068001050D3
:107DC00070001050042A00208001105050CF001085
:107DD00010B501210520FBF7BFFE10BD10B5002234
:107DE0000021024800F02CFA10BDC0461C260020DD
:107DF0008022024B5202DA647047C04600201150C4
:107E0000F0B5C64600B5070000F0C2F90C23354DA9
:107E10003549AB670520FBF7C1FE40239846334C3C
:107E2000402200212000FFF7F7FA43460126A383F2
:107E3000212100232E4A6670A260136063545F31D3
:107E400061844146A187023963542A4A2A49636002
:107E5000E260A1620B60E262284A63629360D360D1
:107E6000274A20009360D360264A00219360D360A4
:107E7000254A40309360D360244A9360D360244AFB
:107E80009360D360234A9360D360234A9360D360A6
:107E9000224A9360D360224A9360D360214A936060
:107EA000D360214A9360D360204A9360D360204A14
:107EB0009360D3601F4A9360D360F0229200FFF773
:107EC000ABFA1D4B1D4A38001A6080239B052E64B7
:107ED000EB6490231A4AEA50FFF78AFF04BC9046ED
:107EE000F0BDC04600001150B57B0010FC250020FD
:107EF00084001050000110508000105000001050FD
:107F000008001050100010501800105020001050A1
:107F10002800105030001050380010504000105011
:107F20004800105050001050580010506000105081
:107F30006800105070001050042A0020800110507A
:107F400010D001000B785B0602D14B78052B00D0D6
:107F500070478A78014B1A60FAE7C046000011505A
:107F6000F0B5CE46474680B58B7848799C460723C6
:107F70000340C8780A798007800F1B021343C2B2FE
:107F800091467F21624666461140D4094F00294D33
:107F90003A195201AA1896700126B4466646664000
:107FA000567000269383D6709077CA00012C27D094
:107FB00021488046880142442818826016600029C2
:107FC00027D01E4AC9009446614441603F223F3396
:107FD00093434A46022A00D15B0019493F190A68B7
:107FE0007F01D3180B60174BED19EA605A408023CC
:107FF0001B0613434A4696061E436B681E600EE03E
:10800000114880468801424428188262166000297F
:108010000AD1002364012D196B600C4BEB60012029
:108020000CBC90469946F0BD064AC900944661448E
:108030004162CBE7FC250020840010500400105062
:10804000042A002000001050800010500001105041
:1080500000231C4A10B59360D3601B4A0021936033
:10806000D3601A4A1A489360D3601A4A9360D36067
:10807000194A9360D360194A9360D360184A936099
:10808000D360184A9360D360174A9360D360174A4D
:108090009360D360164A9360D360164A9360D360AE
:1080A000154A9360D360154A9360D360144A936075
:1080B000D360F0229200FFF7AFF9124B124A1A6018
:1080C00010BDC046000010500800105010001050A5
:1080D0003C2600201800105020001050280010509E
:1080E0003000105038001050400010504800105020
:1080F0005000105058001050600010506800105090
:1081000070001050042A0020800110507F2020B5FC
:10811000150008404000C9094018044940014018B2
:108120001A00290000F08CF8012020BDFC25002059
:108130007F2310B50B40C909002B03D10222074849
:10814000521A8266802258004018054B4001C01820
:108150001201002100F048F810BDC0460020115067
:10816000FC2500207F2310B50B400BD0C909580017
:108170004018054B4001181800230022C370034922
:1081800000F032F810BDC046FC250020FFF7FFFFCD
:1081900080220D4B520410B51A600C4B0C491A602A
:1081A00010008B689843FBD10A4C9C2200212000D0
:1081B000FFF732F98022002152010748FFF72CF91E
:1081C0000923636710BDC04600E0004000F0004096
:1081D00000C0004000001150000010500023037444
:1081E000438283828361704710B58368002901D080
:1081F0001C682140002A11D08024E400114322424F
:108200000CD01A6822420BD10A4A0A401A60FFE7D2
:10821000FFE7FFE7FFE7FFE7FFE78368196010BDAF
:108220007F2281780448CB091140044A9B009A5868
:10823000FBF70AFBFFFBFFFF64CF00109415002043
:10824000F0B5C646002300B583820133037443684A
:1082500004001E68838B81611F1C934200D9171C88
:108260008025BFB2D21BE37892B2ED0062823D431B
:10827000002B02D09025AD013D4301204340E37027
:108280006378002B50D0002A1DD1A023DB011D43B1
:10829000384B1B6C384B33408026B6051E43636851
:1082A000A2681E6013685B0559D4344B2B401360E1
:1082B000FFE7FFE7FFE7FFE7FFE7FFE7A3681D60D2
:1082C00004BC9046F0BD80235B011D43294B1B6C11
:1082D0009B0702D4A378DB09DCD0A38B191C934243
:1082E00000D9111C80278BB2FF00D21A98461F4379
:1082F000E37892B26282002B03D090274146BF01FF
:108300000F4301214B40E3706378002B19D0002A02
:1083100002D18023DB011F43194B3F043340A026C9
:10832000F6053D431E43BAE73A00E068FFF77AF8E6
:10833000A369628A9C46802367441B02A7611D4390
:10834000A1E7E06842464030A169FFF76BF8A369F6
:10835000628A4344A36180231B021F43D7E77F2225
:10836000A1780848CB091140074A9B009A58FBF7AF
:108370006BFAC04600001150FFFFFFAFFFFBFFFF8D
:10838000FFFFFFDF64CF001094150020F0B5C64654
:1083900000B5067C0400002E00D1D8E083681A687E
:1083A0001D684378AD05AD0D002B50D1838AEB18C5
:1083B0009BB28382A18B62688D4206D200236382C6
:1083C0001368300004BC9046F0BD1268520001D51D
:1083D0008D4269D0638A002BF3D062681F1C166837
:1083E0008B425FD88025BFB2DB1BE2789BB2ED00E9
:1083F00063823D43002A37D101214A40E27062780E
:10840000002A3AD0002B47D0802252011543584A07
:10841000126C920757D4A278D20954D1554B3340ED
:108420008026B6051E436368A2681E6013685B055C
:1084300000D593E0504B2B401360FFE7FFE7FFE7C9
:10844000FFE7FFE7FFE7A36800261D60B9E72A0002
:10845000C1688069FEF7E6FFA38AA269EB189BB2A8
:108460005219A382A261A5E7012190254A40E2703A
:108470006278AD013D43002AC4D13A00A169E068A9
:10848000FEF7D0FFA3699C4680231B021D43638A2D
:108490006744A761002BB7D1A023DB011D43344BF8
:1084A0001B6CBBE70F1C9DE7A26815686278AD01E5
:1084B000AD0D002A3DD1EB18A3828D4200D389E790
:1084C000002363827DE7A28B111C9A4221D880276A
:1084D0008AB2FF009B1A90461743E2789BB26382F0
:1084E000002A03D090274146BF010F4301214A4093
:1084F000E2706278002A0ED0002B02D18023DB01CB
:108500001F431E4B3F043340A026F6053D431E4348
:1085100089E7191CDBE7E06842464030A169FEF7B5
:1085200081FFA3694344A36180231B021F43638A25
:10853000E2E7E1682A004031A069FEF773FFA38AF1
:10854000A18BEB18A382A3695B19A361B5E77F2315
:1085500081780B4A19400B48FBF776F97F22A17806
:108560000948CB091140064A9B009A58FBF76CF961
:1085700000001150FFFFFFAFFFFBFFFFFFFFFFDF1A
:108580009415002084CF001064CF0010024B58785F
:10859000431E9841C0B27047F0230020024B187868
:1085A0004007C00F7047C046F0230020014B1878E9
:1085B0007047C046532C0020F8B54746CE462B4D99
:1085C00080B52B780700002B04D001200CBC90460E
:1085D0009946F8BD532200212548FEF71DFF254C82
:1085E0002000FAF79DFD244B1C60244C20001C3019
:1085F000FAF7B2FD200001F023FD214B1C60214B56
:10860000002B2AD0204E00243000FFF769F91F4BC1
:108610001F4A98461860914633780BE04246630043
:108620001B191268DB009B58984701343378E4B279
:10863000A34209D39C42F1D315D14B46984701344C
:108640003378E4B2A342F5D23800FFF7D9FB380003
:10865000FFF7BEFB01232B70B7E701F0B1F80A4B1F
:108660001B78002BF0D000231B68FFDE532C00206A
:10867000F0230020A8230020442400209C15002083
:1086800048240020E1780010522C0020B82000205F
:10869000C1970010F0B5DE4657464E464546E0B558
:1086A0008BB001F097FA002800D18FE1CF4BD04E6C
:1086B0009B4607AC3568EA69EFF3108172B6136820
:1086C000002BFCD0BFF35F8F29622800210001F04E
:1086D0003DFBEA692B6ABFF35F8F0021116083F3D2
:1086E0001088002800D171E16378082BE2D85A463F
:1086F0009B00D3589F466368002BDBD0A068984747
:10870000D8E77F222179BB4B0A405500C8095B1985
:108710001B18180001273030C578BD43C570C578D7
:108720000337BD43C570002A00D199E1B24ADB7C12
:10873000002A00D190E1B14A1278934200D389E136
:108740005A00D318AE4ADB001268D318002B00D1B0
:108750003CE11D6962792078A368A847AAE7012255
:10876000A44F01213B78042013433B703323FA5C70
:108770008A43FA54FA5C8243FA540133FA5C8A431E
:10878000FA54FA5C8243FA5423780020019300F0F3
:1087900095FE602322791340602B00D151E1402BDC
:1087A00000D141E1D206D20E012A00D16AE1002AAD
:1087B00000D15BE1022A00D043E17F22217A0A4006
:1087C0000F2A00D93DE1C80984465200B8188A4DE5
:1087D0006044C07C002D00D18FE1884D2D78A842E7
:1087E00000D388E145002818854DC0002D682D185C
:1087F000002B00D187E1002D00D122E1E86800F0D4
:108800005DFEEB6808AA00210198984716E1794BB4
:108810001B78DB0700D44DE77A4B002B00D149E7EA
:1088200000E000BF46E7734B1A78D20700D441E757
:10883000754A002A00D13DE718780007C00F00E014
:1088400000BF37E76D4D6C4A2B78002A00D1B7E0A6
:1088500000276B491A0088469F4214D24146096896
:108860007B008C46DB19DB0063445B69002B0DD079
:108870002078984701372A78FFB2974200D919E744
:1088800013009F42EAD39F4200D09CE00137FFB221
:10889000974200D90EE71300F3E72378574D564A65
:1088A000984600272B78002A00D1B3E0574A924619
:1088B000534A91462A00454690460FE04A461268C0
:1088C0007B009446DB19DB0063445B682800984713
:1088D000434601371B78FFB2BB420BD39F42EDD317
:1088E0006BD1534628009847434601371B78FFB2A7
:1088F000BB42F3D23F4D532200212800FEF78CFDEE
:108900001022FF21E81CFEF787FD28002022FF210E
:108910001330FEF781FD00F0C7FD3D4B002B00D169
:10892000C8E600E000BFC5E62378344D324A9846D9
:1089300000272B78002A50D0344A9246304A91467C
:108940002A00454690460FE04A4612687B0094464E
:10895000DB19DB0063445B68280098474346013716
:108960001B78FFB2BB420BD39F42EDD325D15346B8
:1089700028009847434601371B78FFB2BB42F3D229
:108980001C4D532200212800FEF746FD1022FF2136
:10899000E81CFEF741FD28002022FF211330FEF7DE
:1089A0003BFD00F081FD2379AB7083E6019800F078
:1089B00045FF2B78002B00D192E200235B68FFDE9D
:1089C000002B00D176E600235B69FFDE0BB03CBCD8
:1089D00090469946A246AB46F0BD404600F02EFFB9
:1089E0002B78002BCCD000235B68FFDEB8CF0010C3
:1089F00048240020F0230020E1780010522C0020B1
:108A0000B820002000000000000000003D98001089
:108A100000000000404600F011FF2B78002B00D131
:108A200068E700235B68FFDEC948002809D000F032
:108A300045FD08AA0021019800E000BF002800D0F1
:108A400038E620780021FFF773FB20788021FFF7BC
:108A50006FFB2FE69B1ADBB2002BB7D1BD4D79E639
:108A600062792078A36800F03DFD23E6202B00D139
:108A700028E1002BE5D16379092BE2D8B64A9B00A7
:108A8000D3589F46237A0F2BDBD8B44AFB18DB78E8
:108A9000002A2BD0B24A1278934225D2B14A5D0007
:108AA000EB181568DB00ED18002DCAD0E86800F05F
:108AB00005FDEB6808AA002101989847002800D01E
:108AC000F8E5602523791D40BBD163790A3B012B72
:108AD000B7D800F0F3FC63790A2B00D150E108A964
:108AE000019800F06FFCE5E59B1ADBB2002BA8D1E2
:108AF0009D489E4DDBE7401BC0B2002800D1F8E046
:108B00000025002B9DD163799946012B04D0002BC1
:108B100000D1FAE0032B94D1E388002B1BD14B4604
:108B2000BA18012B00D1FAE01300302290466344BA
:108B300098444346DB789B070DD40198FFF7F8FA79
:108B400043460222DB7813434246D370D378012296
:108B500013434246D370002D00D1ABE5E86800F026
:108B6000ADFCEB6808AA002101989847002000F0AE
:108B7000A5FC3423FB5CDB0700D59BE5AFE7A379BD
:108B800003931A007B789A4207D07B78002B00D0A1
:108B90007EE1039B002B00D0FBE0039B08A901981A
:108BA0007B7000F00FFC85E57B7806AA023213701B
:108BB00008A90123019800F01DFC7BE5E088030A69
:108BC000C0B20F2B00D93CE769499A008A589746F2
:108BD00008A800F079FCA1790198FFF7FFF80222BC
:108BE0003B7813433B7065E5E388012B00D028E711
:108BF00008223B7808A9934301983B7000F0E2FB00
:108C000058E50220397806AB9A1C8B068908DB0FE1
:108C100001400B43138008A90223019800F0EAFBEE
:108C200048E5E388012B00D00BE708223B7808A930
:108C3000134301983B7000F0C5FB3BE54D4B002B07
:108C400000D1FEE600E000BFC37881781B0202007D
:108C50000B43019808A900F0CDFBEFE6464B002B33
:108C600000D1EEE600E000BF021E00D1E9E6137875
:108C700008A9019800F0BEFBE0E62189FEF762FF3B
:108C8000021EF4D1DDE6022B00D176E13B4B002B36
:108C900000D1D6E600E000BF002800D1D1E6C378BD
:108CA00082781B02134308A90200019800F0A2FB7E
:108CB000C4E6FEF73FFF1223020008A9019800F066
:108CC00099FBBBE6237A0F2B00D9BAE6234AFB189F
:108CD000DB78002A13D0224A127893420DD2214A1F
:108CE0005D00EB181568DB00ED18002D00D1A8E63B
:108CF00084E5002B06D11D4D05E79B1ADBB2002B46
:108D000000D09EE61848194D79E5BA18130063445F
:108D10003033DB7806AA9B07DB0F02327AE72F336A
:108D20009846624490444346DB789B0700D412E7A0
:108D30000198FFF717FA43460222DB789343424635
:108D4000D370D3784A4693434246D37003E7C04674
:108D500000000000319A0010DCCF0010E178001014
:108D6000522C0020B82000204D99001044D0001053
:108D700004D000100000000000000000000000000F
:108D800006AB9A1C08A901230198157000F032FB6C
:108D900090E4581EC0B2FEF7D1FE002800D150E684
:108DA0004378022B00D04CE60125C3795A112A40A2
:108DB000120191463A789B11904610224146914308
:108DC0000A0049460A4320212B408A435B01134392
:108DD0003B7009239946C37882781B021343C3185A
:108DE00081440493994500D3C0E04D4601226B783D
:108DF00002920B2B04D1EB7802932B78ED186B7851
:108E0000042B00D01DE60022049B90465B1B9BB206
:108E10009A46674A674B1B78002A25D02A004546A8
:108E200090469D421AD2644A6B0012685B199146C3
:108E3000DB0099444B469B68059252464146019897
:108E40009847082803D95346834200D3A7E0594BDB
:108E500001351B78EDB2AB42E3D2F2E59D4214D16D
:108E6000564A574B9146E8E752462900019800F0D0
:108E7000FBFCD0468246082802D94346834242D2B0
:108E80004C4B1B78002B00D1DBE500239B68FFDEF9
:108E90000198FFF7DDF8BB78464D454A9A46002118
:108EA0002B78002A00D181E5434A90462A000D0024
:108EB00091460FE0424612686B0094465B19DB0056
:108EC00063445B68019898474B4601351B78EDB2C7
:108ED000AB4205D39D42EDD300D06EE5394BF1E7AF
:108EE000532200213800FEF797FA1022FF21F81CC8
:108EF000FEF792FA380020221330FF21FEF78CFA99
:108F00005346BB7045E62D4B9946294B9846029B2C
:108F1000012B35D0029B002B17D0A9787A18D27874
:108F20000B00FF2A00D08CE5002206E08B18DBB294
:108F3000F818C078FF2800D083E54046FB18D870A9
:108F40000132029BD2B29A42F0D338004346290044
:108F50001330524600F07EFE164B55441B784345B5
:108F600000D26EE5049BAB4200D93FE7164B002BC5
:108F700000D112E600E000BF0FE6FEF7DFFD8BE652
:108F800048468068A97884460D487B18DA7884457D
:108F90000AD0FF2A00D054E54246DA70D5E74346AE
:108FA0008246A8461D00B2E702230293B6E7C046F8
:108FB000E1780010522C0020B820002044D000108E
:108FC000699800103D9800100000000070B586B050
:108FD0006B4605000C00981C0A220021FEF71CFAC3
:108FE0006B461D705C70032C4FD01BD9042C07D02E
:108FF000052C40D13C4B1A78D20766D406B070BD20
:10900000394B1A78D207F9D504211A780A431A7015
:10901000364B1C68E269EFF3108172B61368002BBF
:1090200019D1FBE7022C26D101212F4B1A788A4354
:109030001A701A780331A2431A7000225A701A78F3
:109040008A431A70294B1C68E269EFF3108172B6EB
:109050001368002BFCD0BFF35F8F216269462000AC
:1090600000F03AFFE269236ABFF35F8F00211160CD
:1090700083F31088C2E71D4B1C68E269EFF310818F
:1090800072B61368002BE6D1FBE7174B1A7852072C
:10909000B4D504210E201A7868448A431A7000213E
:1090A0000A22FEF7B9F9052303AE73700F4B357032
:1090B0001C68E269EFF3108172B61368002BFCD0D4
:1090C000BFF35F8F21623100C9E704211A788A4318
:1090D0001A70064B1C68E269EFF3108172B61368D0
:1090E000002BB8D1FBE7C046F02300204824002025
:1090F00070B584B06B4606000D000A220021981D51
:10910000FEF78AF9012301AC63700E4B25711D68CF
:109110002670EA69EFF3108372B611680029FCD05B
:10912000BFF35F8F2B622100280000F0D5FEEA69B3
:109130002B6ABFF35F8F0021116083F3108804B0A6
:1091400070BDC04648240020002330B585B001AD75
:109150006B8028700633082202A86B70FEF762F954
:109160000C4B1C68E269EFF3108372B6116800299A
:10917000FCD0BFF35F8F23622900200000F0ACFE1B
:10918000E269236ABFF35F8F0021116083F31088C7
:1091900005B030BD48240020F0B5C64600B584B007
:1091A0001D006B4680460F00160000210622981D08
:1091B000FEF732F9434601AC2370072363700F4B6F
:1091C00065711D682771A660EA69EFF3108372B6B6
:1091D00011680029FCD0BFF35F8F2B6221002800AB
:1091E00000F07AFEEA692B6ABFF35F8F00211160FD
:1091F00083F3108804B004BC9046F0BD48240020DE
:10920000F0B5DE464F4646468346C0B50C00002A00
:1092100043D04978052916D1E678B607B60FB34290
:1092200011D17F23A1780B400F2B0CD8531E9846E9
:109230001B4B002599467F274B462000997800F06C
:10924000CDFC002805D100201CBC90469946A346C1
:10925000F0BD21005846FEF783FE0028F3D0A37826
:10926000DA09012A13D0089A13702378E4184545C7
:1092700013D06378052BE6D1E3789B079B0FB342AD
:10928000E1D1A37801353B400F2BD5D9DBE7099A13
:1092900013702378E4184545EBD10120D4E7C0468C
:1092A000F02300207F2370B58A7805000C0013405E
:1092B0000F2B01D9002070BD054B2000997800F0DC
:1092C0008DFC0028F6D021002800FEF749FEF2E7C9
:1092D000F02300207F2370B50B40134C5B00C909BD
:1092E000E41864183034E578ED07ED0F04D1E37825
:1092F0005B0703D5280070BD0025FBE701210B4E5D
:109300004942306803F058FAE378DB0707D4E37882
:109310005B0704D404220125E3781343E37030682B
:1093200003F01AFAE6E7C046F023002044240020A8
:1093300070B50D0001210F4C4942206803F03CFA42
:109340007F2129404B000C49ED09C91849193031DA
:10935000CB780025DB0707D4CB785B0704D5042244
:10936000CB7801359343CB70206803F0F5F92800E2
:1093700070BDC04644240020F023002070B57F2437
:109380000C4065000E4C06006419C80924183034DE
:10939000E5780020ED0700D570BD0125E078284371
:1093A000E0703000FEF7B2FE0028F5D10122E3782C
:1093B0009343E370E37803329343E370ECE7C046F2
:1093C000F023002070B50A4C0600082220000D0092
:1093D000FEF728F800230021A360E36069563000FF
:1093E000C943C90FC9010022FFF7C8FF70BDC046BD
:1093F00094230020F0B5C6469046294C082200B5BB
:10940000060020000D001F00FEF70CF84346A36085
:109410000023E381EB79AA791B0213431A1CBB4298
:1094200000D93A1C97B2A281002B12D0002F1DD078
:109430004346002B2ED03B1C402F1DD89FB22378D3
:109440007F2B1ED80021174A3B003000FFF796FF04
:1094500009E0002169560023C943C90FC901002250
:109460003000FFF78BFF04BC9046F0BD23787F2BC4
:1094700012D800210022E7E740239FB223787F2BF8
:10948000E0D9084C3A0041462000FDF7CBFF80218F
:109490002200D9E70020E6E780210022D4E7C04679
:1094A00094230020B023002010B51422002102488C
:1094B000FDF7B2FF10BDC04694230020014B186198
:1094C0007047C0469423002010B5054C01000822C7
:1094D0002000FDF7A7FF0023A360E36010BDC04696
:1094E00094230020F8B53B4C1D0023780600DA09D0
:1094F000C9098A4212D00020002D0ED1364B002B14
:1095000003D021003000FEF71DFD2369002B5AD047
:1095100022000221300098470120F8BDA7687F2B68
:1095200008D80020002FF8D038002A002B49FDF77A
:1095300079FFA768E289E388521992B27F19E28124
:10954000A760934201D03F2D13D82369002B05D08B
:10955000220001213000984700281DD000216156CB
:109560000023C943C90FC90100223000FFF706FFDD
:10957000D3E7A089811A0D1C89B2402916D8237817
:10958000ADB27F2B14D8002182421ED0134A2B008B
:109590003000FFF7F3FEC0E700213000FEF7C8FD02
:1095A00030008021FEF7C4FD0120B6E74025E6E744
:1095B00082420CD0094C2A0039002000FDF732FF0E
:1095C00080212200E3E70120A7E70022DFE78021D6
:1095D0000022DCE794230020457F0010B023002008
:1095E00010B50400FEF7D2FF002801D1002010BD05
:1095F000FEF7D4FF0028F9D1B62080004443034889
:109600000019037901201840F1E7C046BC20002072
:109610000300B6208000584310B5034B1030C0182B
:1096200000F06AFB10BDC046BC200020F0B5B62596
:10963000AD0045432C00C646174E1034A41900B5A2
:1096400092B2200000F0D0FB0700200000F06EFB7B
:109650003F2803D8380004BC9046F0BD7319D97870
:1096600000209846FFF736FE0028F3D0200000F0D7
:109670005DFB3F2805D843460020D978FFF758FE08
:10968000E8E796239B00EA1843469219D978002010
:109690004023FFF773FEDDE7BC200020F0B5B625C0
:1096A000AD0045432C00C6461F4E2C34A41900B50E
:1096B00092B2200000F050FC0700200000F01CFBDC
:1096C0003F2803D8380004BC9046F0BDFEF75EFF8B
:1096D0000028F7D0FEF762FF0028F3D1200000F049
:1096E0000BFB0028EED07319997800209846FFF7FD
:1096F000F1FD0028E6D0A6239B009C466544AE19E8
:1097000031004022200000F06FFB4346997800288A
:1097100005D0030032000020FFF730FED2E7002022
:10972000FFF706FECEE7C046BC200020F8B50500D6
:10973000FEF72CFF002801D10020F8BDFEF72EFF18
:109740000028F9D1B624A40065432E00144F2C360E
:10975000F619300000F0D0FA0028EDD07C19A1787D
:109760000020FFF7B7FD0028E6D0A6239B009C460B
:109770006544ED1929003000402200F035FBA17846
:10978000061E08D003002A000020FFF7F7FD00287E
:10979000D2D03000D1E70020FFF7CAFDCCE7C046A9
:1097A000BC2000200300B6208000584310B5034BB6
:1097B0002C30C01800F0BAFA10BDC046BC20002002
:1097C000B622F0B51B4C83B0920000212000FDF7BB
:1097D00023FEFF236371184B80260025E3800127B9
:1097E00008232100200076002373278132004831AE
:1097F0000095073B103000F043FA2100200049316A
:109800003200FF31009701232C3000F039FA922307
:109810009B00E6183000F9F783FC94239B00A662B6
:10982000E61865623000F9F77BFC2664656403B0D6
:10983000F0BDC046BC20002000C2FFFF10B5094C9F
:10984000052200212000FDF7E7FD20002C34103018
:1098500000F0F6FB200000F0F3FB0121200000F0F7
:1098600015FC10BDBC200020F0B54B7983B006007C
:10987000022B03D00025280003B0F0BD8B79022B0A
:10988000F8D12F4FBB78002BF4D18B7809253B7092
:109890000C780C196378242B0BD1082A02D81FE00E
:1098A000AA421DD32378E418ED186378ADB2242BB7
:1098B000F6D0052B2CD0042B12D163790A2B0FD1B3
:1098C000204B2778019301330093E11902230222F0
:1098D0003000FFF795FC0028CCD00E35ED19ADB265
:1098E000194C200000F022FA3F28C4D92600103E6F
:1098F000F1780020FFF7EEFC0028BCD0200000F03B
:1099000015FA3F2812D8F1780020FFF711FDB2E7D1
:1099100021003000FFF7C6FC0028ABD0A3787B7095
:109920002378ED18E418ADB26378C4E792239B0066
:10993000E218F17840230020FFF720FD9BE7C046A6
:10994000BC200020BE200020CC200020F8B56023E1
:109950001400127813400022202B01D01000F8BD13
:109960002E4D637927792E781B023B439E42F5D119
:109970006378212B43D009D9222B24D0232B14D157
:10998000002945D0022912D00122E7E7202B0CD173
:10999000002936D00229F7D1214B002BF4D0A91D84
:1099A0000020FDF7A3FF0122D8E70022D6E71D4BD8
:1099B000002BE9D0E178A37809021943002000E0E8
:1099C00000BF0122CAE7002922D00229DCD10126EA
:1099D000A178E478280024020C4331002C71A143C3
:1099E0002C3000F053FB104B002BCDD0310062081F
:1099F00032402140002000E000BF0122AEE70029F4
:109A0000C2D10A4A07232100FFF7F4FC0122A5E78F
:109A10002100FFF7D7FC0122A0E7C046BC200020B0
:109A2000ED7800100000000000000000C2200020BF
:109A3000F8B54746CE4680B55D4C1E00E3788046BB
:109A40000D008B4263D1962327009B001037E1184D
:109A5000B2B2380000F080FA564B002B1CD063796C
:109A6000FF2B19D0002E17D00022914605E00123CC
:109A70009C46E1444E450FD06379962292004A44B9
:109A8000A25C9A42F3D1380000F048F90028EED1E8
:109A9000617900E000BFEAE7474B484C002B04D057
:109AA000200000F03BF900285BD0200000F03EF9D8
:109AB0003F2859D8103CA378AB4205D001242000A0
:109AC0000CBC90469946F8BD3D4B002B02D00020BF
:109AD00000E000BFFEF75AFD00281DD1394C2000E0
:109AE00000F00AF90028E9D1002EE7D0B306E5D14D
:109AF0002C3CA1784046FFF7EDFB2500041EDDD08D
:109B0000A978002300224046FFF738FCD7E7A37866
:109B10008B42D9D00024D2E7FEF740FD294C002823
:109B2000DDD1200000F0E8F80028D8D025002C3D39
:109B3000A9780020FFF7CEFB0028D0D09B239B0004
:109B4000E71839004022200000F04EF9A9780028DB
:109B500029D003003A000020FFF710FC0028ADD107
:109B6000BDE700E000BFA0E72700103FF978002024
:109B7000FFF7B0FB002801D1BB789DE7200000F083
:109B8000D5F83F2805D8F9780020FFF7D1FBBB783E
:109B900092E792239B00E218F97840230020FFF718
:109BA000EDFBBB7888E70020FFF7C2FB97E7C046D4
:109BB000BC2000200000000000000000CC2000209D
:109BC00000000000E820002010B50020FEF7F4FCA3
:109BD00010BDC04610B5FEF7E9FC10BD072310B557
:109BE0004479027923401B021A43C3789B079B0FD9
:109BF000022B1BD00DD80020012B09D102394B427A
:109C00005941124B00209C46614491424041C0B2F0
:109C100010BD02394B425941F023002049429B00BC
:109C20001940403191424041C0B2F1E7022905D0CC
:109C30000020402393424041C0B2E9E7044B9C46D8
:109C4000624450425041C0B2E2E7C046FF03000008
:109C500000FEFFFFF0B500247F27002A0FD04D78CB
:109C6000052D06D13D008E7835406D00F609451969
:109C7000AB550D786419A4B24919A242EFD8F0BDD2
:109C8000F8B54746CE4680B5984608AB1F78802386
:109C90000400894615001B0200269A4227D8406915
:109CA000002803D00121494202F086FDA069002866
:109CB00003D00121494202F07FFD4B462360434619
:109CC000A5806D00ADB2E3806B1EA38100236069A7
:109CD0006D42E381277265812382002801D002F062
:109CE0003BFDA0690126002801D002F035FD3000BF
:109CF0000CBC90469946F8BDC189028A89B292B2DD
:109D00008B1A9BB2914202D242899B1A9BB28288E3
:109D1000101C9A4200D9181C80B27047C389008A6F
:109D2000181A43425841C0B27047C04610B5C489A2
:109D3000018AA4B289B2631A82889BB28C4202D291
:109D400040891B1A9BB2D01A80B210BD70B50400B6
:109D500080690D00002803D00121494202F02CFD4A
:109D6000E089218A80B289B2421A92B2884202D234
:109D70006389D21A92B2A388934208D2C21A92B2CD
:109D800098422DD26089121A92B222821A00002AB9
:109D900002D11EE0C91A89B28B42FBD92368E2883E
:109DA0009C46514328006144FDF73CFB228A012573
:109DB00092B2531C9BB29A420ED9002362899B181F
:109DC0009BB2A0692382002801D002F0C5FC2800C4
:109DD00070BD0025238A9BB2A2899A42F1D2EDE799
:109DE000A0899042D1D2CDE7F8B54746CE460400CF
:109DF000806980B50E001700002803D00121494278
:109E000002F0DAFCE289218A92B289B2551AADB227
:109E10008A4202D26389ED1AADB2A388AB420AD25C
:109E2000D11A89B29A424CD26289891A89B21D002C
:109E30002182218A89B2002D47D03A1CAF423BD8FB
:109E400095B28B4203D8C91A89B28B42FBD95B1AEF
:109E50009FB2E3885943984623689C466144BD42BB
:109E600024D94046784383B21A0030009946FDF762
:109E7000D9FA43463000EA1B5A43484492B221685B
:109E8000FDF7D0FA228A92B253199BB29A421ED998
:109E900062899B189BB2A0692382002801D002F03E
:109EA0005BFC28000CBC90469946F8BD4246300049
:109EB0006A43FDF7B7FAE5E72A1C95B28B42C2D98F
:109EC000C5E7A2898A42B2D2AEE7238A9BB2A289B1
:109ED0009A42E0D2DCE7C046F8B5040040690E00C3
:109EE000002803D00121494202F066FCE589238A5B
:109EF000ADB29BB2EA1A92B2AB4202D96389D21ACE
:109F000092B2A388934222D028009D4203D3C01A64
:109F100080B28342FBD92368E2889C4650433100DB
:109F20006044FDF77FFA6B1C9BB29D420BD962899E
:109F30009B189BB26069E3810127002801D002F0E1
:109F40000BFC3800F8BDA2899A42F3D2EFE7277ADA
:109F5000002FD9D1F5E7C046F0B54F46D646464664
:109F60000500C0B514000F00002A05D120001CBC5C
:109F700090469946A246F0BD4069002803D00121D1
:109F8000494202F019FCEA88EE899046298A2A7A29
:109F9000B6B289B2AB88002A0ED1721A92B28E4242
:109FA00002D26989521A92B29A1A111C92B2A24232
:109FB00000D9211C8CB207E09C4205D34246E41A2A
:109FC00054430E003F191C0030009E4203D3C01AB8
:109FD00080B29842FBD21B1A9BB299464346584323
:109FE0002B689C4660444C4515D842463900624374
:109FF000FDF718FAA3199BB29E4202D8AA899A4289
:10A0000002D26A899B189BB26869EB810028ADD0A7
:10A0100002F0A2FBAAE74B46414659438BB21A0015
:10A0200039009A46FDF7FEF94B46E21A43463900DD
:10A030005A43514492B22868FDF7F4F9DAE7C04672
:10A0400010B504004069002803D00121494202F004
:10A05000B3FBA069002803D00121494202F0ACFB08
:10A060000023E3812382A38860695B009BB25A1EB0
:10A070005B42A2816381002801D002F06DFBA069E0
:10A08000002801D002F068FB012010BD70B504006B
:10A0900040690D00002803D00121494202F08CFBE9
:10A0A000A069002803D00121494202F085FB6069C4
:10A0B0002572002801D002F04FFBA069002801D0D2
:10A0C00002F04AFB012070BD10B5024800F0EAF82A
:10A0D00010BDC046182A0020013930B5002900D132
:10A0E000B4E06F4B1A781211D5B22C003034092A23
:10A0F00000DDAEE00470012900D1A6E00F221C783B
:10A10000224014003034092A00D9A4E04470022906
:10A1100000D19AE05A781211D5B22C003034092AB5
:10A1200000DD9BE08470032900D18EE00F225C7873
:10A13000224014003034092A00D991E0C470042967
:10A1400000D182E09A781211D5B22C003034092A5D
:10A1500000DD88E00471052977D00F229C78224029
:10A1600014003034092A00D97FE0447106296CD0EC
:10A17000DA781211D4B225003035092A00DD77E0F3
:10A180008571072961D00F22DC7822401400303419
:10A19000092A00D96FE0C471082956D01A79121122
:10A1A000D5B22C003034092A00DD073404720929A5
:10A1B0004BD00F221C79224014003034092A01D9D7
:10A1C0003732140044720A293FD05A791211D4B29E
:10A1D00025003035092A01DD3734250085720B2929
:10A1E00033D00F225C79224014003034092A49D838
:10A1F000C4720C2929D09A791211D5B22C003034AE
:10A20000092A42DC04730D291FD00F229C792240B9
:10A2100014003034092A3AD844730E2915D0DA795B
:10A220001211D5B22C003034092A33DC84730F2983
:10A230000BD0DA790F2313401A003732092B2BD9B0
:10A24000C273102901D0103000E0401800230370C1
:10A2500030BD07344EE73732140057E7073461E763
:10A26000373214006AE7073474E7373214007CE7AA
:10A270003734250084E737321400C471082900D030
:10A280008CE7E2E737321400B2E70734BAE7373237
:10A290001400C1E70734C9E730331A00D0E7C046DD
:10A2A000182A002010B588B004000D22002168464D
:10A2B000FDF7B2F80D22002104A8FDF7ADF84B23FD
:10A2C0006A4604A9137068460D2202F03DFA152172
:10A2D000082269442000FDF7A5F808B010BDC0466B
:10A2E000F0B546468046354BD64643445A1E934108
:10A2F0008022520294464F465B421340304A6344E8
:10A30000C0B513602F4A0D002F49136018008A68EA
:10A310009043FBD10620F9F719FC80268146E90D10
:10A320006802AB0DAA020224760006E0914507D32D
:10A3300012184B413C00B74202D0A71C002BF5D0AD
:10A3400080272602361B7F0003E05746361B012F6D
:10A3500031D07B1E310048469A46FCF7E5F985422C
:10A36000F3D23900534661431B024246146112681E
:10A3700040465340FF221202134080225201024302
:10A380001360036807205840CF2303401360424600
:10A39000802303209B0124321A4310604246171D7C
:10A3A0001F43022348463B60FCF7BEF91CBC9046A5
:10A3B0009946A246F0BD21000023D6E70040FCBF2D
:10A3C00000E0004000F0004000C000400020704766
:10A3D0007047C046F0B5CE46474680B583B06B4661
:10A3E000591D13230B700D3B6B44994601244A46BB
:10A3F000002313702300C268D02793403F06BB613F
:10A400000C4B050001221800984602F0DDF96B465E
:10A41000DE1D320001234946404602F0DDF9EB68BB
:10A420009C407C613078EB69C01A03B00CBC90464C
:10A430009946F0BD00C00340F0B5CE46474680B512
:10A4400085B06B46D9710368364A5B680400934255
:10A4500062D10921222369440B70183B6B44984652
:10A4600001274246002313703B00C268D026934068
:10A470000F253606B36101226D442B4802F0A4F982
:10A4800001232A004146284802F0A6F93B00E26871
:10A49000934073612A789046FF2A3AD00B2180209E
:10A4A0006A466944087003A88146D2790270B36194
:10A4B00001221D4802F088F901232A0049461A4862
:10A4C00002F08AF93B00E2689340012273610126A1
:10A4D0000E2742446F443A700D21D022A2206944D5
:10A4E00012060870904693610F48012202F06CF941
:10A4F00001232A0039000C4802F06EF90123E268BA
:10A50000934042465361300005B00CBC90469946DA
:10A51000F0BD00220026DBE769460122073198479B
:10A520000600F0E7E9A5001000C00340F0B5C646FC
:10A5300000B503682A4A1B6982B00400934249D1DE
:10A540006B46D91C13230B7001AB984601250023E1
:10A55000424613702B00C268D02793403F06BB6170
:10A560000122204802F030F96B46DE1D3200012343
:10A5700041461C4802F030F9E3689D407D61307827
:10A58000E369C01A002827D0E36906220133E3619A
:10A590006B460125591D00236A440B7013702B0074
:10A5A0009046E268D02793403F06BB6101220D48E8
:10A5B00002F00AF96B46DE1D3200012341460948CC
:10A5C00002F00AF9E3689D407D61307802B004BC76
:10A5D0009046F0BD9847D5E701204042F6E7C046D7
:10A5E000D5A3001000C00340F0B55746DE464E46E6
:10A5F0004546E0B587B004AB0C00591C22230B7014
:10A6000004AB9F1C012500233B702B008146C068D2
:10A61000D0268340360602929046B3610122374825
:10A6200002F0D2F804AA9446072363449A463900FC
:10A6300001235246314802F0CFF84B46DB685146C1
:10A640009D40C446756109782A008C446046039099
:10A65000FF2805D9FF20401A8446614402900391E7
:10A660000299002927D08C46A4446246019204AA8C
:10A67000D71C802293467F3A904605AE2278D0259B
:10A680003270424659469A402D0639701B48AA61DD
:10A690003900012202F098F8012352463100174890
:10A6A00002F09AF84B464246DB6801999A40013421
:10A6B0006A618C42E2D104AB591DA223D0240B70F5
:10A6C00004AB9D1D039B24062B700C48A261012244
:10A6D00002F07AF8524601232900084802F07CF87B
:10A6E0004B46DA68012393400298636107B03CBC93
:10A6F00090469946A246AB46F0BDC04600C0034016
:10A70000F0B5D6464F464646C0B50368454A1B6974
:10A7100084B00400934200D07FE06B46D91D132320
:10A720000B7002AB984601250023424613702B00A4
:10A73000C268D02793400F263F06BB6101226E44BA
:10A74000394802F041F8012332004146364802F010
:10A7500043F8E3689D407D613078E369C01A0028C2
:10A760005DD00D210D2369440B7001336B44994674
:10A770000023984601264B4642461A703300E26891
:10A78000D02593400F272D066F44AB610122264848
:10A7900002F01AF8494601233A00234802F01CF857
:10A7A0003300E2680B2193406B613A78694492462A
:10A7B000424640460A7003AA91461070AB610122DE
:10A7C000194802F001F8494601233A00164802F000
:10A7D00003F83300E268092193406B613A786944D9
:10A7E00090468D220A70833A6A4450469146107012
:10A7F000AB6101220C4801F0E7FF01233A00494612
:10A80000094801F0E9FFE36840469E406E6104B0EC
:10A810001CBC90469946A246F0BD98479FE7012090
:10A820004042F4E7D5A3001000C00340F0B5454610
:10A83000DE464E465746E0B50126050089B0C068A1
:10A840008846F7F7ABFD3300EA68D02493402869C7
:10A85000240663626361431C0FD0F7F79FFD33004A
:10A860002A690A2093406362A361F8F709FA2B6909
:10A870000A209E406661F8F703FAC849C848FFF706
:10A880002FFD01211020F7F771FD01211220F7F7AC
:10A890006DFD01211320F7F769FD0820F7F77EFD14
:10A8A000D024802324065B00636263616B46D91C5D
:10A8B000422301260B70002301AF3B703300EA688E
:10A8C000B74893400122A36101F07EFF1F220123BC
:10A8D0006A443900B24801F07FFF3300EA6800277C
:10A8E00093406A466361D27F122A07D0380009B0CC
:10A8F0003CBC90469946A246AB46F0BD11216F3252
:10A9000069440A7091466F3A6A44924680225046E2
:10A910000270A3617F3AA24801F056FF1F22514600
:10A9200001236A449E4801F057FF3300EA689340D0
:10A930009A4663614346D917AB61C9045B0B19435F
:10A940004346984AD8040023FBF730FF172186239B
:10A95000694480460B7006AB9B4643465A461B0C27
:10A96000137053460122A3618D4801F02DFF1F2271
:10A9700001236A4459468A4801F02EFF3300EA68F1
:10A98000152193408722694463610A70713A6A44D1
:10A99000924642465046120A0270A3610122804844
:10A9A00001F012FF1F22514601236A447C4801F046
:10A9B00013FF3300EA68132193408822404669441C
:10A9C00063610A7005AA10709246A361012274485F
:10A9D00001F0FAFE1F22514601236A44704801F03B
:10A9E000FBFE3300EA680F2193408E2269446361C5
:10A9F0000A7004AA17709046A3610122684801F00A
:10AA0000E3FE1F22414601236A44654801F0E4FE4B
:10AA10003300EA680D2193408F22694463619046B8
:10AA20000A70813A6A4417709246A36101225C4819
:10AA300001F0CAFE1F22514601236A44584801F022
:10AA4000CBFE3300EA680B2193400C22694463611A
:10AA50000A7003AA17709246A3610122504801F0C0
:10AA6000B3FE1F2201236A4451464D4801F0B4FE53
:10AA70003200EB6809219A408C206B466944626180
:10AA800008700320DB7F0A3703436F443B70444860
:10AA9000A261012201F098FE1F22390001236A44BD
:10AAA0003F4801F099FE3300EA6802AF93406A46DE
:10AAB000D11DA62263610A70A23A3A703848A36198
:10AAC000033A01F081FE1F22390001236A44344811
:10AAD00001F082FE3300EA681B219340CD226944D5
:10AAE000636107AF0A70493A3A702D48A361833A0F
:10AAF00001F06AFE1F22390001236A44284801F050
:10AB00006BFE3300EA68192193401A278B226944AF
:10AB100063616F440A70603A3A702148A3612A3A2F
:10AB200001F052FE1F22390001236A441C4801F043
:10AB300053FE3300EA681D219340892269441E2791
:10AB400063610A7042466F443A701548A3618E3AB9
:10AB500001F03AFE1F22390001236A44104801F037
:10AB60003BFE3300EA680E4893406A46511D4A4650
:10AB700063610A706A46971D4A463A70A361803A3B
:10AB800001F022FE1F22012339006A44044801F02B
:10AB900023FEEB6801279E406661A7E6D4300000E3
:10ABA00000C003400048E801F0B5CE46474680B5F6
:10ABB00087B06B4601258946D91C002301AF3B7045
:10ABC00098462B00C268D026934036060D700400CC
:10ABD000B3610122794801F0F7FD172201236A448D
:10ABE0003900764801F0F8FD2A00E36800209A4019
:10ABF0006B467261DB7DDB439B0700D19FE06B46B8
:10AC0000591D12230B706B469F1D43466B483B70CA
:10AC1000B261012201F0D8FD172201236A443900F4
:10AC2000664801F0D9FD2B00E26893406A467361E3
:10AC3000D17D08220A4200D086E009210A25D026CB
:10AC4000812269446D4436060A702A705B48B361FC
:10AC5000803A01F0B9FD17222900012501236A4439
:10AC6000564801F0B9FD2B00E26893404A467361F3
:10AC7000002A00D07FE0112122621D2269441227A0
:10AC80000A704A466F443A704C48B361012201F0A1
:10AC90009BFD1722390001236A44484801F09CFDBE
:10ACA0002A00E3680F219A406B469D207261DB7D8C
:10ACB0006944087004AFAB433B704048B261012265
:10ACC00001F082FD1722390001236A443B4801F05C
:10ACD00083FDE36815219D408D2375616944162726
:10ACE000D0260B70002336066F443B700122B561FD
:10ACF0003248984601F068FD1722012539000123EA
:10AD00006A442E4801F068FD2B00E268132193404D
:10AD1000A222694473610A70424605AF3A7027481F
:10AD2000B361013201F050FD172201236A4439005A
:10AD3000224801F051FDE36801209D40756107B094
:10AD40000CBC90469946F0BD69469220073102AF8F
:10AD500008703A701948B361073A01F035FD1722BF
:10AD600001236A443900154801F036FD2B00E268E2
:10AD70009340736161E70D211D2269440E270A701B
:10AD800000226F443A7025620132B3610B4801F032
:10AD90001BFD1722390001236A44084801F01CFDFD
:10ADA0002A00E3680B219A409D206B46694472613A
:10ADB00008700120DB7D03AF03437DE700C0034043
:10ADC000F0B50124D6464F4646462300C0B5C268BA
:10ADD00084B00500934000293DD00F226A4490467C
:10ADE000826A002A17D06A46D026D11DC02202AF3F
:10ADF0000A703606803A3A704448B3613F3A01F02F
:10AE0000E3FC012342463900404801F0E5FC230001
:10AE1000EA6893407361092181220A26D02469449B
:10AE20000A706E440232240632703848A361823AB6
:10AE300001F0CAFC012342463100344801F0CCFC49
:10AE40000123EA6893406361012004B01CBC904672
:10AE50009946A246F0BD092181220A27D0266944DD
:10AE60000A706F44360602323A702848B361823A5B
:10AE700001F0AAFC0F236B44984639000123424697
:10AE8000224801F0A9FCEB6812229C400B27924655
:10AE9000113A74616F4403AE914603E00020F7F766
:10AEA000EFFEEB6852463A70002232704A46D024D8
:10AEB0009A402406A26139000122144801F084FC62
:10AEC000012342463100114801F086FC4B46EA68F6
:10AED000934042466361117808220A42DED00D2178
:10AEE0000E26922069446E44087032700748A361B0
:10AEF000012201F069FC012342463100034801F0C0
:10AF00006BFC4A46EB689A4062619DE700C00340D3
:10AF1000F0B5DE4657464E464546E0B58BB06B462B
:10AF20008A46D91D12230B7002AB9846002399461E
:10AF3000012643464A461A703300C268D027934020
:10AF400027243F060500BB6101226C44B74801F08D
:10AF50003BFC012322004146B44801F03DFC330094
:10AF6000EA6893407B61227890465246002A00DCD2
:10AF700037E10D211D2269440A700F3A6A444846A0
:10AF8000934610702E620122BB61A84801F01CFCA0
:10AF9000012322005946A54801F01EFC3200EB684F
:10AFA0000B219A409D2069447A61087003A881466C
:10AFB00001202378034348460370BA619B4801226D
:10AFC00001F002FC494601232200984801F004FCEC
:10AFD0003300EA6809219340A22269447B610A7028
:10AFE000983A6A44504691461070BB6101228F48DE
:10AFF00001F0EAFB4946012322008C4801F0ECFBFA
:10B00000EB6815219E4092237E61D0274246694419
:10B010000B7099467C3B6B443F069A461A70BE61A2
:10B0200001260122814801F0CFFB01232200514675
:10B030007E4801F0D1FB3300EA68132193404A4671
:10B0400069447B6140460A7005AA91461070BB6155
:10B050000122764801F0B8FB0123220049467348DB
:10B0600001F0BAFB3200EB6841469A4060237A61F6
:10B070000B40402B00D073E000202B6AE861002BCE
:10B0800066D119211320694408700730684480464E
:10B090000370BA616548012201F096FB4146012325
:10B0A0002200624801F098FB3300EA681F219340B8
:10B0B0007B612278694490461022D0270A700022D2
:10B0C0003F0608AE32705948BB61013201F07CFB8B
:10B0D0003100012601232200544801F07DFB33009A
:10B0E000EA681D2193408D2069447B6108706F38A8
:10B0F0006844814622780270BB6101224B4801F00E
:10B1000063FB494601232200484801F065FB3300F8
:10B11000EA681B21934007A88122814669447B612C
:10B120000A700270BB61803A404801F04DFB012378
:10B13000220049463D4801F04FFBEB689E407E618E
:10B1400040460BB03CBC90469946A246AB46F0BD8B
:10B150001721222369440B7006AB9846187098E7B4
:10B1600022236B4498462121002340466944037002
:10B170000E702E48BA61012201F026FB41460123E0
:10B1800022002A4801F028FB3300EA68002193409E
:10B190007B6122788846862AD2D08D222531694467
:10B1A0000A70673A6A44404691461070BB610122BA
:10B1B0001E4801F009FB4946012322001B4801F00B
:10B1C0000BFB3300EA6823219340812269447B61B1
:10B1D0000A7009AA9146862248460270BB61853AE8
:10B1E000A2E74A4611212A621D2269440A700B3ADD
:10B1F0006A44484692461070BB6101220B4801F038
:10B20000E3FA012322005146084801F0E5FA320032
:10B21000EB680F219A409D207A6123786944087079
:10B22000B34304A803708146BA61DFE600C003405F
:10B23000F0B5C64600B582B06B46591D1A230B7097
:10B24000143B6B44984601244246002313702300AC
:10B25000C268D02793403F060500BB610122114818
:10B2600001F0B2FA6B46DE1D3200414601230D4863
:10B2700001F0B2FAEB689C407C61A869FBF738FDED
:10B280008022094BD205FBF705FD431E984143423E
:10B290000720347818409D30201A02B004BC904634
:10B2A000F0BDC04600C00340DD4ABF41F0B5CE4608
:10B2B000474680B585B06B468946591CC02301249A
:10B2C00000270B70BE3B6B441F7098462300C2687A
:10B2D000D02593402D060600AB6101224E4801F0B7
:10B2E00073FA0F2201236A4441464B4801F074FA75
:10B2F0002300F26893404A466B61002A67DD6A4684
:10B30000D11D1D220A7002AA177034629046AB61EB
:10B310000122414801F058FA0F2201236A444146B4
:10B320003D4801F059FA2200F36869469A409D2091
:10B3300005316A61087068466B46871D0120DB7B1A
:10B3400003433B703448AA61012201F03DFA0F2209
:10B35000390001236A44304801F03EFA2300F268C4
:10B3600001AF93406A46D11CA2226B610A704A4623
:10B370003A70AB610122284801F026FA0F22390009
:10B380006A440123244801F027FAF3680D219C4008
:10B390000E276C618123D02569440B706F44043300
:10B3A0002D063B700122AC611B4801F00DFA0F2203
:10B3B00001236A443900184801F00EFA0123F268AB
:10B3C00093406B6105B00CBC90469946F0BD0B21D3
:10B3D0001D2269440A7003AA177037629046AB6158
:10B3E00001220D4801F0F0F90F2201236A44414681
:10B3F000094801F0F1F92200F36809219A406B46EF
:10B400000A279D206A61DB7B69446F44A34308706F
:10B410003B70AA61AEE7C04600C00340F0B5CE461F
:10B4200047460500012080B5EB6885B09840002AAA
:10B4300025D10B000E2900DDA5E06A46D11C89222A
:10B440000A70DA43D2171340D026702201AC13439E
:10B45000360623700122B0614E4801F0B5F90F2283
:10B4600001236A4421004B4801F0B6F90123EA6840
:10B470009340736105B00CBC90469946F0BD11290C
:10B4800029DD142900DD80E06B46CC1ED91DCD23BB
:10B4900002AE0B70463B3370D0230F271B0698611A
:10B4A00001223C48984601F08FF9310001266F4493
:10B4B00001233A00374801F08FF93300EA689340DE
:10B4C000424653616A46511D8B220A70853A6A448E
:10B4D0009146312227E00C00022958DB0B21CD23B5
:10B4E00069440B7003AE493B3370D0230F271B0612
:10B4F000986101222748984601F066F9310001263B
:10B500006F4401233A00234801F066F93300EA68EA
:10B5100009219340424653618B2269440A70813A63
:10B520006A4491462B22484602704246194893616C
:10B53000012201F049F901233A004946154801F07A
:10B540004BF93300EA680D2193404246536189224A
:10B550000E2669440A700A3AFF3A023C14436E44CC
:10B560003470D0242406A36181320A4801F02CF9FA
:10B5700001233A003100074801F02EF90123EA685F
:10B580009340636176E70E2357E714217CE702249A
:10B59000A4E7C04600C00340F0B54546DE46574626
:10B5A0004E46E0B5050087B0052900DC0AE10C290C
:10B5B00000DDFCE0062900D104E109014BB2984608
:10B5C0000921B12369440B70A73B6B4499460126BE
:10B5D0004A46C32313703300EA68D02793401724E8
:10B5E0003F06BB6101226C44944801F0EDF84946E6
:10B5F00001232200914801F0EFF83300EA689340FC
:10B600006A46D11DB7227B610A7002AA91460A22BE
:10B6100048460270BB61093A884801F0D5F8012319
:10B6200022004946854801F0D7F83300EA68934084
:10B630007B610D211E2269440E26D0270A7000224C
:10B640003F066E4432709146BB6101327B4801F087
:10B65000BBF83100012601232200784801F0BCF834
:10B660003200EB680B219A409E2369447A610B708B
:10B6700003AB9A460F23207803404046184303004B
:10B6800050460370BA616D48012201F09DF8012314
:10B6900022005146694801F09FF83300EA680F2103
:10B6A00093401D2269447B6148460A7004AA904673
:10B6B0001070BB610122614801F086F8012322006D
:10B6C00041465E4801F088F83200EB689A407A61A2
:10B6D00023781B11092B6EDC59499B005B58994656
:10B6E00013211E236944D0270B7000233F0605AEAB
:10B6F00033705248BA6101229B4601F065F831006F
:10B700000126012322004D4801F066F83300EA6863
:10B71000112193407B6122786944924626220A7067
:10B72000143A6A44584690461070BB61012243485F
:10B7300001F04AF8414601232200404801F04CF84C
:10B740003300EA68310093407B61984653461B11F1
:10B7500099404846FAF7C0FF0100FA208000277898
:10B76000FAF7BAFF10282ADC08239F431521A623E5
:10B7700069440B70903B6B44D0261F70994643463A
:10B780003606B36101222D4801F01EF82200012384
:10B7900049462A4801F020F80123EA689340736182
:10B7A00007B03CBC90469946A246AB46F0BD40234C
:10B7B0005B42984604E701235B42994690E70823E1
:10B7C0001F43D3E76B46591DB1230B70AB3B6B4452
:10B7D000984601264246C52313703300EA68D027F5
:10B7E000934017243F06BB6101226C44134800F0CC
:10B7F000EBFF414601232200104800F0EDFF33002B
:10B80000EA6893406A46D11CB7227B610A7001AA9C
:10B8100090460C2240460270BB610B3A074800F08C
:10B82000D3FF012322004146044800F0D5FF330036
:10B83000EA68934060227B619046FAE600C00340CC
:10B840005CD00010F0B5DE46454657464E46E0B5A2
:10B85000050085B00800FBF74BFA974B0022060065
:10B860000F00FBF71DFA00239846002855D1934B93
:10B87000002230003900FBF713FA10239846002805
:10B880004BD18F4B002230003900FBF709FA2023FF
:10B890009846002841D18B4B002230003900FBF73D
:10B8A000FFF930239846002837D1874B002230001B
:10B8B0003900FBF7F5F94023984600282DD1834B3A
:10B8C000002230003900FBF7EBF95023984600289E
:10B8D00023D17F4B002230003900FBF7E1F96023D0
:10B8E0009846002819D17B4B002230003900FBF725
:10B8F000D7F97023984600280FD1774B00223000EB
:10B900003900FBF7CDF9431E98410F2270234042C6
:10B9100090435B4280469C46E0446B46591D1D2384
:10B920000B709A46173B6B449B46002399460126B1
:10B930005B464A461A703300EA68D02793400F24CA
:10B940003F066C44BB610122644800F03DFF59464C
:10B9500001232200614800F03FFF3200EB689A406B
:10B960006B46D91C9D237A610B7001AB9B460F235C
:10B970002078034040461843030058460370BA61DC
:10B980005648012200F020FF594601232200534867
:10B9900000F022FF3300EA68484693406A46D11D12
:10B9A00052467B610A7002AA90461070BB61012268
:10B9B0004A4800F009FF012322004146474800F0B1
:10B9C0000BFF3200EB689A407A6123781B11092B38
:10B9D0006ADC43499B005B5899460B211E2369444E
:10B9E000D0270B7000233F0603AE33703B48BA618B
:10B9F00001229B4600F0E8FE3100012601232200CF
:10BA0000364800F0E9FE3300EA68092193407B6183
:10BA100022786944924626220A701C3A6A445846A3
:10BA200090461070BB6101222C4800F0CDFE4146CB
:10BA300001232200294800F0CFFE3300EA683100DC
:10BA400093407B61984653461B1199404846FAF74C
:10BA500043FE0100FA2080002778FAF73DFE102807
:10BA600026DC08239F430D21A62369440B70983BD5
:10BA70006B44D0261F70994643463606B3610122B7
:10BA8000164800F0A1FE220001234946134800F0A9
:10BA9000A3FE0123EA689340736105B03CBC904665
:10BAA0009946A246AB46F0BD01235B42994694E716
:10BAB00008231F43D7E7C0460078BE400050C4406B
:10BAC0000078CE400050D4408084DE40805CE4406A
:10BAD0008084EE408084FE4080840E4100C003409C
:10BAE0005CD00010F0B5CE46474680B5050083B067
:10BAF0000C00082900DD08246B46591D1D230B701E
:10BB0000173B6B44994600234A461370EA68013399
:10BB1000D027984693403F06BB610122194800F0A8
:10BB200053FE6B46DE1D320001234946154800F0E6
:10BB300053FE4346EA68694693409D207B6103318A
:10BB40003278087001AF052C00DA05240E20043C81
:10BB50008243640014433C70D0242406A361012274
:10BB6000084800F031FE320001233900054800F09A
:10BB700033FE0123EA689340636103B00CBC904636
:10BB80009946F0BD00C00340F0B5CE46474680B5AB
:10BB900083B06B468946591DA0230B709A3B6B44BA
:10BBA00098464B46424601241B1213702300C2687C
:10BBB000D0259340174E2D060700AB6101223000BF
:10BBC00000F002FE6A46414601230732300000F0D1
:10BBD00003FE2300FA68484693406A46D11CA1221E
:10BBE0006B610A7001AA10709046AB6101223000AF
:10BBF00000F0EAFD6A46012307324146300000F0BA
:10BC0000EBFDFB689C406C6103B00CBC9046994610
:10BC1000F0BDC04600C00340F0B5CE46474680B5F3
:10BC200083B06B46591D1E230B70183B6B4499461D
:10BC300001244A46002313702300C268D025934094
:10BC4000194E2D060700AB610122300000F0BCFD4B
:10BC500007236B449846494642460123300000F0D2
:10BC6000BBFD2200FB6869469A409E200331434693
:10BC70006A61087001A8814604201B780343484686
:10BC80000370AA613000012200F09EFD01234246AC
:10BC90004946300000F0A0FDFB689C406C6103B099
:10BCA0000CBC90469946F0BD00C0034009490A4BC0
:10BCB000083119600949002299600821D9600331CF
:10BCC000196101395A6059619A61DA611A625A62DE
:10BCD0009A62704784D000108020002000C003408A
:10BCE00010B5062000F06AFB0120F7F78FFDC04673
:10BCF000F0B557464546DE464E46E0B50D000B35DD
:10BD000083B00700162D28D8102900D9C1E000F013
:10BD1000A7FA102518230220CE4EF3181A005C68EB
:10BD2000083A944200D160E1032362689A43130009
:10BD3000E268A168CA6091600122E318596838007E
:10BD40000A435A6000F08EFA2000083003B03CBC71
:10BD500090469946A246AB46F0BD07239D4300D5C9
:10BD600097E0A94200D994E000F07AFAF823FF3373
:10BD70009D4200D85EE1680A00D18EE0042800D917
:10BD800039E138239846A80980443930C100B14EC2
:10BD900071180839CC68A14218D0032362689A430D
:10BDA0001300521B0F2A00DD1DE1002AC0DA032315
:10BDB0009C4608E06246636893435A1B0F2A00DDE5
:10BDC00011E1002AB4DAE468A142F3D13200346907
:10BDD0000832944267D00323616899438A460B0076
:10BDE000491B0F2900DD12E1726132610029A3DADB
:10BDF000994A924500D948E1DB08FF3A9910FF3A89
:10BE00008A40DB0071689B190A4399687260E3609D
:10BE1000A1609C60CC60012183109940914248D878
:10BE20000A4205D103239843490004300A42FBD05B
:10BE300003239846C3009946B144CC4682466346E4
:10BE4000DC68A44507D1F9E0002A00DB0EE1E468D4
:10BE5000A44500D1F2E04246636893435A1B0F2A7F
:10BE6000F2DD01208046611905436560A068E56840
:10BE70000836C560A8604046F160B1601043486074
:10BE8000CE608E603800E25000F0ECF920000830FF
:10BE90005CE70C2300203B6058E780213F238900AA
:10BEA0004020984673E701217268831099409142BF
:10BEB000B6D90323B46862689A439046AA4203D372
:10BEC000531B0F2B00DD80E0644B654A9A46934676
:10BED0001B681268EB18013200D138E1614A9446C0
:10BEE00063441B0B1B0300930099380000F0BCF95E
:10BEF00003008146013300D1F6E04346E218824256
:10BF000000D9EFE051464968009B8C465146634496
:10BF10004B60824200D14BE159460968013100D1A2
:10BF20005DE149468A1AD3185246536007234A46B0
:10BF30001A40019200D120E108214B4689469B1A04
:10BF400099440099484B49449B1A5B1A1B051B0DE9
:10BF50000091380019009B4600F086F9431C00D17F
:10BF60005AE1534652465B6849465B4453604A4631
:10BF7000B260801A0122584410434860B44211D084
:10BF800041460F2900D827E107200C39814360681A
:10BF9000024005200A4362606218506090600F29D9
:10BFA00000D941E15246D26A934201D95246D36246
:10BFB0000322B468616891430A005146096B8B42C1
:10BFC00000D895E051460B6392E00122290013430B
:10BFD0001143651961603800B5606B6000F042F98B
:10BFE00020000830B2E64046F0E6DC680230A342AA
:10BFF00000D1EBE698E614286ED9542800D9A9E0C0
:10C000006E239846280B80446F30C100BFE60123A1
:10C0100060191D43656070613061C26082601A0002
:10C0200053460A4342603800E15000F01BF92000FB
:10C0300008308BE62B00E80808336DE608239B46A2
:10C04000073BDC449B46DA4443465246134200D049
:10C05000F5E667E0F8190020FF0100004C1F002002
:10C06000F01900200F100000081000000122E31852
:10C07000596838000A435A60E368A268D3609A603E
:10C0800000F0F0F82000083060E65A0A042A3AD995
:10C09000142A00D983E05B23984690445C32D20096
:10C0A00008235B429C46B218944463469968032374
:10C0B00099468C4559D04B464A689A43524502D915
:10C0C00089688C45F7D1CB6872689C466346A1604D
:10C0D000E3609C60CC609EE65B23984680445C30C5
:10C0E000C10054E6B4427ED00323B46862689A4328
:10C0F000531B954202D80F2B00DD66E7380000F095
:10C10000B1F8002022E69A09382398469044393243
:10C11000D200C5E74B461A68083B013891469A425F
:10C1200000D098E043460342F4D173688B437360B8
:10C130004900994200D9BCE6002904D1B9E604229D
:10C1400094464900E2440B42F9D0504672E610335F
:10C150000093C9E6AA235B00984233D8DD3B98469A
:10C16000E80B80447830C10011E6434601229B1061
:10C170009A4073681A437260A8E7009B38004B44EA
:10C1800000931B055B421B0D19009B4600F06CF8E9
:10C19000431C00D0E5E6002300989B46E1E6542AC4
:10C1A00029D81A0B6E23984690446F32D20077E755
:10C1B000110500D0B0E60120009AB1684244024364
:10C1C0004A60EFE6254B984220D87C239846A80C7D
:10C1D00080447D30C100DAE54B465A608EE75B460D
:10C1E0004A461A60A2E651464968009B8C46514671
:10C1F00063444B6090E6AA2149008A421CD8DA0BBE
:10C200007723984690447832D20049E7FE217E2376
:10C2100089007F209846BAE5009B01989C46002340
:10C22000083860449B469CE621003800083100F045
:10C230008FF953465B68B5E608498A4206D89A0CDE
:10C240007C23984690447D32D20029E7FE227E234B
:10C250009200984624E773686AE7C04654050000D8
:10C260007047C0467047C046002370B5064C0500B5
:10C2700008002360F7F7CCFA431C00D070BD236898
:10C28000002BFBD02B60F9E71C2F002010B580217C
:10C290000400FFF72DFDB7239B00E050002807D0D6
:10C2A00002000023803208C09042FCD1002010BD63
:10C2B00001204042FBE7C046B7239B00C25810B59F
:10C2C0000023002A01D0180010BDFFF7DFFF030094
:10C2D000F9E7C046F8B505000C0016001F2909D87B
:10C2E000B727BF00C359002B09D0A4001C19206830
:10C2F0002660F8BD1623036001204042F9E7FFF7EE
:10C30000C5FF002801D1EB59EFE701204042F0E7DB
:10C3100070B505000C001F2922D8B7239B00C35815
:10C32000002B0ED08A009B181A68002A09D0012A17
:10C3300010D0511C10D0002120001960904700201F
:10C3400070BD280000F07EF822000100280000F0F7
:10C3500065F8F5E70020F3E7162303600120EFE717
:10C360001623036001204042EAE7C04670B505008D
:10C370000C001F291DD8B726B6008359002B10D0FA
:10C38000A2009B181A68002A09D0511C0FD0012A5C
:10C3900012D00021200019609047002070BD0120BC
:10C3A000FCE7FFF773FF002803D1AB59E8E7022051
:10C3B000F4E701204042F1E70320EFE710B5034B1B
:10C3C00001001868FFF7A4FF10BDC046C01500208B
:10C3D00010B5044B0A001B6801001800FFF77AFF34
:10C3E00010BDC046C0150020B722064B92001B6846
:10C3F00010B59A580020002A00D010BD1800FFF791
:10C4000045FFFAE7C015002010B5034B010018687E
:10C41000FFF7ACFF10BDC046C0150020002370B56B
:10C42000074C050008001100236000F083F9431C4D
:10C4300000D070BD2368002BFBD02B60F9E7C0460D
:10C440001C2F002010B500F06DF910BD10B50400D0
:10C4500083070AD00378002B23D0032202E003785D
:10C46000002B1CD001301042F9D102680E4B0F494D
:10C47000D31893430B420FD1043002680A4BD318F0
:10C4800093430B4208D104300268074BD3189343FF
:10C490000B42F1D000E001300378002BFBD1001BF0
:10C4A00010BD0020FCE7C046FFFEFEFE80808080BD
:10C4B000F8B50C000600FFF7D3FE204FBB685D689F
:10C4C00003239D431E4B2C1B9C466444240B1D4B95
:10C4D000013C24039C4207DD00213000FFF7C4FE2D
:10C4E000BB685B19984204D03000FFF7BBFE002008
:10C4F000F8BD61423000FFF7B7FE431C0DD00122AA
:10C50000BB682D1B15435D600F4B30001A68141B70
:10C510001C60FFF7A7FE0120EAE700213000FFF7CB
:10C52000A3FEBA68831A0F2BDEDD08490968401A9A
:10C530000549086001210B435360D5E7F819002035
:10C54000EF0F0000FF0F0000501F0020F019002027
:10C55000F8B5CE464746050080B50C1E55D0FFF70E
:10C560007FFE210008394F68012438000323A043CF
:10C570000A1856689E43B146644EB368934229D068
:10C580004B465360D3189C463C4242D10F68C91BAE
:10C590008B68C019984663465F6808239C46B4447C
:10C5A0002740E0456AD04346CC68DC60A360002F9A
:10C5B00032D1012448440443A0469368544C0F18D8
:10C5C000A34200D17FE0D268DA60936043464B60BB
:10C5D000386025E003004B443C4206D10A68891AC2
:10C5E00088689B18CA68C260906001221A434A603A
:10C5F000484AB16012689A4204D8474B280019682B
:10C60000FFF756FF2800FFF72DFE0CBC9046994619
:10C61000F8BD5F682740CCD0012303434B6008502E
:10C620003E4B98421AD9430A042B33D8820914008E
:10C6300039323834D200B218083A936803279A4244
:10C6400039D05C68BC43844233D99B689A42F8D1A4
:10C65000D368CB608A609960D160D3E7C008FF3BA4
:10C660008210FF3B93407268C000134373608619C9
:10C67000B368CE608B60B160D960C3E7002F41D151
:10C68000030090684B44D2681C43C26090604C60C9
:10C69000CB50B7E7142B07D9542B1CD8020B14002E
:10C6A0006F326E34D200C6E71C005C335B34DA00B4
:10C6B000C1E71A00CCE70123A410A340706803432C
:10C6C00073601300C5E7D9609960CB608B60434607
:10C6D0004B60386096E7AA225200934205D8C20BFD
:10C6E000140078327734D200A5E70D4A934205D87A
:10C6F000820C14007D327C34D2009CE7FE227E2422
:10C70000920098E704434C6010607BE7F819002022
:10C71000001A0020F41900204C1F0020FF01000027
:10C720005405000058220120014B40421A60704716
:10C730001C2F002058220120014B40421A607047F4
:10C740001C2F0020F8B5C04601B40248844601BC45
:10C75000604700BF8903002001B40248844601BC41
:10C76000604700BFE901002001B40248844601BCD3
:10C77000604700BFD904002001B40248844601BCD0
:10C78000604700BF0903002001B40248844601BC91
:10C79000604700BFD904002001B40248844601BCB0
:10C7A000604700BF0901002001B40248844601BC73
:10C7B000604700BF8D02002001B40248844601BCDE
:10C7C000604700BF5101002001B40248844601BC0B
:10C7D000604700BF8D04002001B40248844601BCBC
:10C7E000604700BF3504002001B40248844601BC04
:10C7F000604700BFC100002001B40248844601BC6C
:08C80000604700BFC5130020D2
:10C808005A230010681500105A2300105A230010EC
:10C818005A2300105A2300100C1100105A2300103C
:10C828005A2300105A2300105A2300105A230010CC
:10C838005A2300105A2300105A2300105A230010BC
:10C848005A2300105A2300105A2300105A230010AC
:10C858005A2300105A2300105A2300105A2300109C
:10C868005A2300105A2300105A2300105A2300108C
:10C878005A2300105A2300100C100010C610001084
:10C88800741000105C1000108C1000104410001080
:10C89800A41000102210001030303030300000009A
:10C8A8004C6F52612073657474696E67733A000047
:10C8B8006C6F72614672657175656E6379202020B0
:10C8C800202020203D2025750A0000006C6F726131
:10C8D800537072656164696E67466163746F722034
:10C8E8003D2025690A0000006C6F72615072656115
:10C8F8006D626C6520202020202020203D202569A5
:10C908000A0000006C6F7261436F64696E67526160
:10C9180074652020202020203D2025690A00000081
:10C928006C6F72615478506F7765722020202020D8
:10C93800202020203D2025690A0000004C6F52610C
:10C94800506153656C6563742020202020202020CE
:10C958003D2025690A0000006C6F726142616E64B7
:10C968007769647468202020202020203D202575C8
:10C978000A0000005374617274696E67204C6F522C
:10C988006120726164696F0020205B204641494C38
:10C998004544205D0000000020205B20444F4E45A8
:10C9A800205D0000536F7572636520616464726571
:10C9B80073733A2025730A44696769706561746501
:10C9C800727320282575293A202573202573202580
:10C9D800732025730A446174613A2025730A0000A4
:10C9E8004D6573736167652066726F6D207365723C
:10C9F8007665723A2025732028636F6D6D616E64C9
:10CA0800202575290A00000041636B6E6F776C65FD
:10CA180064676520726571756573743A2025730AB9
:10CA2800000000004572726F72206465636F64696C
:10CA38006E672041505253206672616D652E00006A
:10CA48004E6F2076616C6964206461746120666F42
:10CA5800756E6420696E20464C415348206D656DA3
:10CA68006F72792E0000000045726173696E67204D
:10CA7800464C41534820726567696F6E2E2E2E0012
:10CA8800646F6E650000000057726974696E6720F4
:10CA980064656661756C742076616C756573207465
:10CAA8006F20464C4153482E2E2E0000466F756E5F
:10CAB800642076616C69642073657474696E677349
:10CAC80020696E20464C415348206D656D6F727920
:10CAD8002E000000415052532073657474696E67CC
:10CAE800733A00004D792063616C6C3A2025730A13
:10CAF800000000005365727665722063616C6C3AC1
:10CB08002025730A000000004669726D776172651E
:10CB18003A2025730A0000005265636569766564EA
:10CB2800207061636B6574202852535349203D205F
:10CB3800256964426D290A004552524F523A204EE7
:10CB48006F206F7220636F72727570746564204114
:10CB5800505253206672616D652E00004E6F20732F
:10CB680070696E6C6F636B732061726520617661AA
:10CB7800696C61626C650000486172647761726516
:10CB880020616C61726D20256420616C726561643E
:10CB98007920636C61696D656400000048617264A6
:10CBA80020617373657274000A2A2A2A2050414E44
:10CBB8004943202A2A2A0A002A550010E254001064
:10CBC800E254001022550010E2540010E254001004
:10CBD800E2540010E2540010E2540010E254001035
:10CBE800E254001012550010E25400101A550010BB
:10CBF800E2540010E2540010CC5400107455001098
:10CC0800B25C001068550010B25C0010545500105A
:10CC1800B25C0010B25C0010B25C0010B25C001094
:10CC2800B25C0010B25C0010B25C00103855001005
:10CC3800B25C0010B25C0010B25C0010B25C001074
:10CC4800B25C001038550010C05500107254001026
:10CC58007254001072540010725400107254001074
:10CC68007254001072540010725400107254001064
:10CC78007254001072540010725400107254001054
:10CC88007254001072540010725400107254001044
:10CC98007254001072540010725400107254001034
:10CCA8007254001072540010725400107254001024
:10CCB8007254001072540010725400107254001014
:10CCC8007254001072540010DA5800108655001083
:10CCD800DA58001072540010725400107254001088
:10CCE80072540010725400107254001072540010E4
:10CCF80072540010725400107254001072540010D4
:10CD080072540010725400107254001072540010C3
:10CD180072540010685700107254001072540010BA
:10CD280072540010725400107254001072540010A3
:10CD3800725400107254001072540010685700109A
:10CD4800FC56001068570010DA580010865500107D
:10CD5800DA5800107254001068570010725400100E
:10CD68007254001072540010725400107254001063
:10CD7800685700108C56001072540010725400103E
:10CD8800D0550010725400106857001072540010EB
:10CD980072540010685700106E616E00666E692D3F
:10CDA80000000000666E692B00000000666E6900D6
:10CDB800000000000000F03F0000000000002440D8
:10CDC80000000000000059400000000000408F40B3
:10CDD800000000000088C34000000000006AF8401E
:10CDE8000000000080842E4100000000D012634142
:10CDF8000000000084D797410000000065CDCD41B8
:10CE080006005250BBFF3CB64CCE001006005250F4
:10CE1800E182887F34CE001006005250D3F075426C
:10CE28002CCE001052656C6561736500626F6F747B
:10CE3800325F77323571303830000000312E332EB2
:10CE4800300000007069636F000000006D61696E5A
:10CE58000000000041707220323920323032320036
:10CE68000D0A000041780010457800105578001030
:10CE78007D78001051780010000000000600525024
:10CE880053B4F4A190CE00105553422073746469D2
:10CE98006E202F207374646F757400005261737074
:10CEA8006265727279205069000000005069636FF2
:10CEB80000000000426F6172642043444300000098
:10CEC8005265736574000000090254000301008074
:10CED8007D080B00020202000009040000010202A2
:10CEE8000004052400200105240100010424020295
:10CEF8000524060001070581030800100904010044
:10CF0800020A00000007050202400000070582022D
:10CF18004000000904020000FF00010512010002A0
:10CF2800EF0201408A2E0A000001010203010000FD
:10CF380000000000A4CE0010B4CE0010402C002049
:10CF4800BCCE0010C8CE0010556E68616E646C656A
:10CF5800642049525120307825780A0065702025D0
:10CF6800642025732077617320616C726561647930
:10CF780020617661696C61626C65000043616E27AF
:10CF88007420636F6E74696E7565207866657220AB
:10CF98006F6E20696E6163746976652065702025FF
:10CFA80064202573000000006F757400696E00002E
:10CFB800B4860010288900109A8800104488001050
:10CFC800268800100E8800105E8700100287001067
:10CFD800F6860010028C0010E88B0010428A0010C0
:10CFE800228C0010428A0010D08B0010BC8B0010DD
:10CFF800428A0010A88B00107E8B0010428A001015
:10D00800B28C0010868C00107A8C0010428A0010B6
:10D01800428A00105C8C0010868C0010428A001036
:10D02800428A0010428A0010428A0010428A001088
:10D03800428A0010428A00103C8C0010C1970010F0
:10D048003D980010699800104D990010319A001011
:10D0580000000000781E0000A0280000F03C00003E
:10D0680040510000127A0000E4A2000024F40000FD
:10D0780048E8010090D0030020A10700000000004C
:10D088000000000039A40010E9A50010CDA300108D
:10D09800D1A30010D5A300102DA5001001A70010E2
:10D0A800080052500A38A504090052500001000037
:0CD0B800BCD0001053504920435300002E
:10D0C400A0B20181ABF08001000000008014018156
:10D0D400B0B0ABF00000000080020181B0B0AB3012
:10D0E4000000000080040181B0B0AB3000000000FB
:10D0F40080010181B0B0AB10000000008006018106
:10D10400B0B0ABF00000000080030181B0B0AB70A0
:10D114000000000080080181B0B0ABF00000000006
:10D1240080060181B0B0AB300000000080030181B3
:10D13400B0B0AB7000000000800A0181B0B0ABF069
:10D144000000000080010181B0B0AB1000000000BD
:10D1540080040181B0B0AB30000000008004018184
:10D16400B0B0AB300000000080060181B0B0ABF07D
:10D174000000000080040181B0B0ABF000000000AA
:10D1840080020181B0B0AB30000000008002018158
:10D19400B0B0AB300000000080020181B0B0AB3011
:10D1A4000000000074B20181B0AB308000000000C8
:10D1B400800A0181B0B0ABF0000000003F020181A1
:10D1C400B0AB30800000000080060181B0B0ABF04D
:04D1D4000000000057
:10D1D8008431FF7FAB08B1804432FF7FAB70808021
:10D1E8004833FF7FAB108080A837FF7FD0FEFF7FDA
:10D1F800DC3BFF7F01000000FC3CFF7FCCFEFF7F93
:10D208006451FF7F01000000C4D1FF7FC8FEFF7F8B
:10D2180020D2FF7FCCFEFF7F0CD3FF7FD0FEFF7FA5
:10D22800C0D3FF7FD4FEFF7FD0D4FF7FD8FEFF7F1F
:10D23800F4D5FF7FDCFEFF7F68D9FF7FE0FEFF7F2C
:10D2480078DBFF7FE4FEFF7FC0DCFF7FE8FEFF7F27
:10D25800D8DFFF7FECFEFF7F4CE0FF7FF0FEFF7F13
:10D26800B4E1FF7FF4FEFF7F28E3FF7FF8FEFF7F36
:10D27800CCE5FF7FFCFEFF7F64E8FF7F00FFFF7FB8
:10D2880000E9FF7F04FFFF7F88E9FF7F08FFFF7F3A
:10D2980014EAFF7F01000000F032FF0FB0A90280FE
:10D2A8008433FF0FB0B0A880D033FF0F0100000017
:10D2B800DC33FF0FB0B0AA801034FF0FE4FEFF7F0D
:10D2C800D034FF0F01000000CC34FF0FAA3F398093
:10D2D8001835FF0FB0B0A8802435FF0FB0B0AA8072
:10D2E8006435FF0FB0B0A8807835FF0F010000004B
:10D2F8007435FF0FB0B0A8807C35FF0F0100000027
:10D308000436FF0FAA0FB2806C36FF0FA0FEFF7F16
:10D318004439FF0FB0B0A8806039FF0F9CFEFF7F33
:10D32800BC3BFF0F010000002C3DFF0F0084048070
:10D338003C3DFF0FB0B0A8803C3DFF0F88FEFF7F4B
:10D348002440FF0F008404804440FF0FB0B0A88041
:08D358005C40FF0F0100000022
:10D36000B4020010A80200109C02001008CE0010A9
:10D370009002001014CE001020CE0010A8D0001093
:08D38000B0D0001084CE0010B3
:10D38800D02330B500251B065D57002406E003684E
:10D39800BFF35F8F1C6081F3108820BF0268EFF332
:10D3A800108172B61368002BFCD0BFF35F8F03792E
:10D3B8007F2BECD905710368BFF35F8F00221A60D9
:10D3C80081F3108830BDC046030010B50068EFF344
:10D3D800108472B60268002AFCD0BFF35F8F042263
:10D3E8009A56002A0BDB00290FD000200A601B6820
:10D3F800BFF35F8F00221A6084F3108810BDD0221B
:10D408001206126801201A71F1E70020EFE7C04602
:10D41800F0B5C64600B50C00070001F089F9FA22FC
:10D4280005000E00920020000023002101F078F989
:10D438002C002A00350024184D41AE422FD9012472
:10D448006442E517D0231B061B68002698460BE0AC
:10D458003B68BFF35F8F1E6081F3108820002900AE
:10D4680001F076F9002818D13A68EFF3108172B606
:10D478001368002BFCD0BFF35F8F3B797F2BE7D974
:10D4880043463B713B68BFF35F8F00221A6081F30C
:10D498001088012004BC9046F0BD0020FAE7AE4297
:10D4A800D0D1A242CBD8CDE70268EFF3108172B693
:10D4B8001368002BFCD0BFF35F8FFF230371036851
:10D4C800BFF35F8F00221A6081F3108840BF704756
:10D4D80030B5094C2378002B0DD180230748084923
:10D4E8005B05F0221D6812069A18043385508B429A
:10D4F800F7D10123237030BD542C00205C24002078
:10D508000001001010B5024B0133984710BDC0460A
:10D518005C240020054B1A6880239B005340C022DE
:10D5280092001340024A13607047C0460C800140C5
:10D538000C900140034B1A68C0239B009343024A96
:10D54800136070470C8001400C900140F0B58023B7
:10D558004F464646D6464218C0B59B0306000F0004
:10D568009A4201D901F0FCF8142518242888238848
:10D578001149984723888246104928889847238864
:10D5880081460F492888984723880E49804628886D
:10D5980098470400FFF79CFFD047C847802239000E
:10D5A8003000D8235202C047A047FFF7ABFF1CBC8E
:10D5B80090469946A246F0BD4946000045580000ED
:10D5C8005245000046430000F8B54E465746DE4631
:10D5D80045468023E0B517008218060089469B035C
:10D5E8009A4201D901F0BCF8142518242888238808
:10D5F80011499847238883461049288898472388E3
:10D6080082460F492888984723880E4980462888EB
:10D6180098470400FFF75CFFD847D0473A004946CF
:10D628003000C047A047FFF76DFF3CBC90469946C5
:10D63800A246AB46F8BDC046494600004558000022
:10D648005250000046430000F0B5D6464F464646C5
:10D658001423C0B51827984681460D00188822491A
:10D668003B881400984743468246204918883B88DF
:10D67800984743461E49060018883B8898478046C5
:10D68800FFF726FFD047B047FFF744FFC02022002E
:10D6980008264005163F230013431BD03100836A38
:10D6A80019401F420BD0002C09D0131B0D2B06D894
:10D6B8004B461B78013C036601239C46E144002944
:10D6C800E9D0002AE7D0036E013A2B702300013518
:10D6D8001343E3D1FFF72EFFC047FFF713FF1CBC2E
:10D6E80090469946A246F0BD4946000045580000BC
:10D6F80046430000F0B5C6468C461D001C000221BA
:10D70800042700B526002E431BD0002D0DD0C66877
:10D7180031420AD02E000836A64206D96646367827
:10D72800013D86600126B046C444002CEAD0C66894
:10D738003742E7D08668013C1670260001322E4336
:10D74800E3D1180004BC9046F0BDC04630B50300D4
:10D75800002A09D002258818DC682542FCD00C78FC
:10D7680001319C608842F7D1D968490704D504245F
:10D778009968D9680C42FBD11024D9680C42FCD1B5
:10D78800D968490704D504249968D9680C42FBD1A3
:10D7980001211000196230BD7047C04603685A0065
:10D7A80003D45B005B08C01870478022120613433D
:10D7B800F9E7C046F0B557464E46DE464546E0B561
:10D7C800814683B09246002925D04B1E9B460027F0
:10D7D80001935B46FB18DC0FE4184B466410E50028
:10D7E8005E193000FFF7DAFF019B8046A3420BD099
:10D7F800280008304844FFF7D1FFD04506D8013843
:10D80800504509D2671CE4E7504505D9A74202D024
:10D81800631E9B46DDE70026300003B03CBC904603
:10D828009946A246AB46F0BD012809D0022805D08A
:10D83800002801D0002070470248FCE70248FAE7B8
:10D848000248F8E75D0C0020750C0020690C0020E8
:10D8580030B5234B83B005008C1E002B26D001A9C0
:10D86800200000E000BF00281CD001992200FFF72B
:10D87800A1FF041E16D0FFF791FF6368A864012B6F
:10D888002AD0201D002B23DBFFF788FF0023E86444
:10D898002B650368002B0FDBFFF780FF2861002052
:10D8A80003B030BD002309202B61F9E70D480E496C
:10D8B800091AC9100191D9E71801000FFFF7B4FF41
:10D8C8002861431E98410823404298430930E7E7FE
:10D8D8000123E8642B65DCE7002305202B61DFE7E3
:10D8E80000000000D8D1001060D30010036810B504
:10D8F8000400DA0705D448309B070ED500F06CFC0D
:10D9080023685A070ED51A0713D5DB0604D420005E
:10D91800D130FF3000F06CFC10BD00F059FC2368DA
:10D928005A07F0D42000D03000F05AFC23681A07B8
:10D93800EBD420005130FF3000F056FC2368E4E7B8
:10D948000368002B00D01B18180070470920704787
:10D958007047C04670B504000D0008E02B6C2A0023
:10D9680063612100012023699847082807D1296CA1
:10D978002000FFF76DFF0028F0D000F0F9FE07281F
:10D98800FBD10020296CFFF7E3FF281D00F00AFCFB
:10D99800F0B5CE46474680B5C3682E4C9846A54498
:10D9A8008369060014000431402205A8994600F056
:10D9B800C7FE002304AD049323E0F0222B6C520031
:10D9C800736129007CA800F0BBFE7CAA3100336992
:10D9D800200098478A9B07006B6403934B46009589
:10D9E80001933200330021000120C04700281FD1D5
:10D9F800F0227CA95200280000F0A2FE0024082F83
:10DA08001FD1296C3000FFF723FF611E8C410700EE
:10DA180009340028D1D0AB6B10216B644B462143ED
:10DA280001930095330032000120C047002800D040
:10DA380009273800F5239B009D440CBC9046994665
:10DA4800F0BD072FF4D12000296CFFF781FF05A84E
:10DA580000F0A8FB2CFCFFFF406C704770B5CB6B47
:10DA6800FAB00B6404000E004022043103A800F051
:10DA780067FE01235B42029306E002AA21002369A4
:10DA88009847050008280AD1129B20001900019325
:10DA9800FFF7DEFE0028F0D009207AB070BD02A89A
:10DAA800FFF724FF062DF7D131002000FFF752FFC2
:10DAB80010B58261DA6BC1601A6419000022FFF7A1
:10DAC80067FF10BD436970B50B64C36804000D009F
:10DAD800002B15D10A002369010002209847072866
:10DAE80007D0082803D129002000FFF733FF00F0F2
:10DAF8003FFE0020296CFFF72BFF281D00F052FB8A
:10DB08000122FFF745FF00F033FEC046C36810B599
:10DB1800002B05D0CB6B00220B64FFF739FF10BD3B
:10DB2800FFF79CFFFBE7C0467047C046836810B507
:10DB3800002B02D001000120984710BD012906D012
:10DB4800002906D003390220012900D97047012095
:10DB5800FCE7002B08D10F2A06D8920082185268D9
:10DB6800009B00201A60F1E70220EFE700B585B0BE
:10DB780003AB0A00009300210023FFF7DFFF03989F
:10DB880005B000BD012906D0002906D003390220BE
:10DB9800012900D970470120FCE7002B08D10F2A82
:10DBA80006D8009B92001B68821853600020F1E79A
:10DBB8000220EFE700B585B003AB039200930A009B
:10DBC80000230021FFF7DEFF05B000BD70B51A4C39
:10DBD800D36BA544136406000D0019A8111D40223B
:10DBE80000F0AEFD01235B42189314E00C2118A845
:10DBF80002AAFFF7DFFF290018A8B047002812D1B2
:10DC0800069B18AA02A90830019398470400052822
:10DC18000AD0092807D0289B02A819000193FFF70A
:10DC280017FE0028E2D0092418A8FFF75FFE20009D
:10DC380090239B009D4470BDC0FDFFFFF0B5DE46FC
:10DC480057464E464546E0B5160003220D00110022
:10DC58008BB01F000193EB6C01401C1D009107A9BC
:10DC68001B688B460894002F6BD01A0C1B0459466E
:10DC7800079302230B72FD3313409B004A72E4188A
:10DC8800009B022B00D1AC6B2B6DDB0747D4002324
:10DC980005930833034002932768002F00D112E14F
:10DCA800019B022B49D063882788984604340123B6
:10DCB80040469A469843AB6C0F2199468144300000
:10DCC800FFF754FF0021814506D839005346994390
:10DCD800494488428941494243465A000223134035
:10DCE800012217403B43012B3AD0002B30D0022BA6
:10DCF8001BD12368009A5F007F08002A67D100299A
:10DD080006D0029A002A00D17CE0002F00D1A9E0B9
:10DD1800002B00DA04340137BF00E419BCE7594688
:10DD2800300000F00BFB002810D009200BB03CBCE1
:10DD380090469946A246AB46F0BD636808349846BB
:10DD4800B5E71B0207935B461A8199E70820EDE7C0
:10DD5800009B002B02D0002900D08DE004349BE703
:10DD6800009B002B1AD1002916D02368DF0F6368A7
:10DD78009A1CDAD02A0058320692013300D1BDE04D
:10DD8800201DFFF7DDFD06AB01003A00280000E08A
:10DD980000BF002800D082E008347DE70D21300064
:10DDA8002F6AFFF7E3FE8742F6D1AB6A9C42F3D1B4
:10DDB8002000FFF7F3FC0F2102003000FFF7FAFE06
:10DDC80030002A000021FFF7F5FE0720AEE72B6A96
:10DDD8000D2130009846FFF7C9FE804501D0236821
:10DDE80096E7AB6A9C42FAD10023EB6204332B63BB
:10DDF800231DAF626B632368002B00DA86E00123E2
:10DE0800059388E7002F2DD058239C46AC446346E1
:10DE18000393231D99460023984606AB22000493DA
:10DE28003B004C464746B24698462E00914603E0D2
:10DE380004342F00454542D0039B20000693FFF78A
:10DE48007FFD049B0100002230007D1C00E000BF24
:10DE58000028EDD04346B84635004C4656461F00CC
:10DE68009845BCD10D213000FFF780FE069B286243
:10DE78006B62AC62062059E72000FFF78FFC043480
:10DE88000700AC63280000E000BF002800D14CE781
:10DE980030003A000F21FFF78DFE072046E7070004
:10DEA8000D213000FFF762FE2862022F2BD1069B5E
:10DEB800EB622B002C336B62AC62062036E7350030
:10DEC8004C465646CEE75946300000F037FA00284F
:10DED80000D02AE7059B002B00D137E70F2130003F
:10DEE800FFF744FE0E2102003000FFF763FE30000A
:10DEF800094A0F21FFF75EFE072017E70D213000C2
:10DF0800FFF734FE2862069B6B62D5E738000130C4
:10DF1800800020184DE7C0460000000010B500231F
:10DF2800FFF78CFE10BDC04610B50123FFF786FE33
:10DF380010BDC04610B50223FFF780FE10BDC046D5
:10DF4800F0B5CE46474680B50500C3B014001E00A4
:10DF5800012955D000294BD0032922D0042949D1C1
:10DF6800002B47D1102A45D8102203681A4200D046
:10DF7800F1E020AF380000F03DF900230120A96B43
:10DF880002009A40144203D00E689A00BE50043131
:10DF98000133042BF4D13800A96300F029F90020DB
:10DFA80029E0032B26D11404230C160C9846F318E9
:10DFB800102B1FD8082203681A4200D098E020AF1F
:10DFC800380000F013F94246AB6BF6001C00002A3B
:10DFD80008D0D400F21A1C19BA181968D1500433A1
:10DFE8009C42FAD1AC63380000F0FEF8002002E051
:10DFF800002B24D0022043B00CBC90469946F0BDBB
:10E00800130C14049846240C012E2ED0052EF1D1A1
:10E018001B19202BEED842460F2A70D9A146002C96
:10E028007ED1AA6B4346AA630F2B00D89AE04B46D1
:10E03800002BDBD0684600F0D3F80020DBE7002394
:10E048001004A96B000C013632009A40104204D02B
:10E058000F689A00AA18576004310133102BF3D1C6
:10E068000020A304C7D4A963C5E71B19102BC1D886
:10E0780043460F2BBED82B681E4206D00322280029
:10E0880093432B60483000F0A5F820AF380000F02B
:10E09800A1F8AA6B002C24D04346DB00FF1800230C
:10E0A800994664000023A400D158F95004339C42D7
:10E0B800FAD14B4612196F46002B0FD04046102854
:10E0C80000D210204B46D90000231038C000381861
:10E0D800D458C45004339942FAD15218012EA1D110
:10E0E80020AF04323800AA6300F072F8002082E7FB
:10E0F800934303605130FF3000F078F85FE7102B4E
:10E108003BD910225242914699442B68194208D0B3
:10E11800022228008B4313432B60483000F05EF83E
:10E128002B6804221A4221D143460F2B03D820AF73
:10E13800380000F053F86F46380000F053F8102408
:10E148004346AA6BE41A002CB8DD434620AFDB0037
:10E158006400FF18A6E793430360D130FF3000F056
:10E1680049F806E720A800F037F860E7280093434D
:10E178002B60D03000F036F8D6E72B680B4207D07A
:10E18800022228008B4313432B60483000F026F806
:10E1980020AF380000F022F8A146AA6B002C00D06E
:10E1A8007AE73FE7011C343138C9043B9C461D60BF
:10E1B800A646011C20313CC990469946A246AB466A
:10E1C800011C0831FCC941680068E54600BDC0462D
:10E1D8007047C0467047C0467047C0467047C04643
:10E1E8007047C0467047C0467047C0467047C04633
:10E1F8007047C0467047C04601B401A801B585B054
:10E20800FFB408A841464A4653465C4665463EC0A8
:10E2180001A83EC80F98009000230CB401A9FFF78D
:10E228001DFC109B12B0184701B401A801B585B0B8
:10E23800FFB408A841464A4653465C4665463EC078
:10E2480001A83EC80F98009000230CB401A9FFF75D
:10E2580039FC109B12B0184701B401A801B585B06C
:10E26800FFB408A841464A4653465C4665463EC048
:10E2780001A83EC80F98009000230CB401A9FFF72D
:10E2880045FC109B12B0184701B401A801B585B030
:10E29800FFB408A841464A4653465C4665463EC018
:10E2A80001A83EC80F98009000230CB401ABFFF7FB
:10E2B800FFFB109B12B0184701B401A801B585B047
:10E2C800FFB408A841464A4653465C4665463EC0E8
:10E2D80001A83EC80F98009000230CB401AAFFF7CC
:10E2E80075FC109B12B01847027A0300002A0BD164
:10E2F800427A002A0FD0013A42724268111D4160E9
:10E3080003211268017202E0013A02720268100EDB
:10E3180012021A607047B020FCE7C04600B585B00D
:10E3280003AB00930C2200230021FFF707FC03989E
:10E3380005B000BD10B5FFF7F1FF10BDF0B55746A9
:10E348004E464546DE460023E0B587B003930F33BB
:10E358009846083B994680231B0306000F009A46FF
:10E368003800FFF7C1FF0400B02800D1C3E003065E
:10E378002AD5030042469343DBB2802B00D171E0DB
:10E38800902B3DD0A02B00D185E0B02B50D0C02BD6
:10E3980000D196E003004A469343DBB2D02B0AD162
:10E3A8005346024001321A43052301213000FFF78A
:10E3B800C7FD0028D4D00924200007B03CBC9046F3
:10E3C8009946A246AB46F0BDFF23820013401D1DAF
:10E3D80005AB9B4600930D22002300213000FFF778
:10E3E800ADFB630620D4059B9C46654405955B46BA
:10E3F8000D220093002100233000FFF7C3FBAFE795
:10E40800833B03400D2BD6D005AD02400095002379
:10E4180000213000FFF792FB009500230D22002118
:10E428003000FFF7AFFB9BE7059B5D1B0595DEE71B
:10E43800B12874D0B22800D1CFE0B32800D184E04D
:10E44800FC230340B42BB6D04A465346024001325F
:10E458001A43012101233000FFF772FD002800D183
:10E468007EE7A8E704023800FFF73EFF8025204337
:10E478002D02A8429FD004010005020C00230021B0
:10E488003000FFF75DFD002895D12C4200D167E7E9
:10E498000123039364E7FF234A461B0119008243C3
:10E4A80011410A001A40030702D58023DB011A43F1
:10E4B800002300213000FFF743FD002800D14FE77B
:10E4C80079E7C6284CD0C7285ED003004A46934354
:10E4D800DBB2C02B6DD0C82872D0C92800D06AE73B
:10E4E8003800FFF701FFF02302031B0313404246E5
:10E4F8000240013257E7039B0024002B00D05BE762
:10E5080005AD00950E2200213000FFF717FB00959E
:10E5180000230F2200213000FFF734FB4CE73800BE
:10E52800FFF7E2FE002800D145E703004246934387
:10E53800DBB2002B00D03EE7020000213000FFF7DD
:10E54800FFFC002800D10BE735E73800FFF7CCFEC9
:10E55800F02302031B03134042460240013277E7CF
:10E568003800FFF7C1FEF02302031B0313404246A5
:10E57800024001321A43032303213000FFF7E0FC75
:10E58800002800D1ECE616E73800FFF7ADFE021EC2
:10E5980000D110E7030041468B43DBB2002B00D0CB
:10E5A80009E704213000FFF7CBFC002800D1D7E6AB
:10E5B80001E74346A0221C40013412032243DAE754
:10E5C8003800FFF791FE434602009A43D2B2103258
:10E5D8001840120301300243E6E605AB00939B4660
:10E5E8000D22002300213000FFF7A8FA3800FFF7BA
:10E5F8007BFE030618D57F25B03C059B2840A0402C
:10E608009C466044059038000734FFF76DFE03060A
:10E61800F3D481217F23890003408C46A340059AC7
:10E6280062449B180593E2E60224F2E7030000B572
:10E63800DB6C85B05A680800120201921A0001A921
:10E6480008324A6003220A72DB794B72FFF776FEC2
:10E6580005B000BD10B5FFF76DFE806C10BDC0465B
:10E6680010B5FFF767FEC26CD3799B000833D0184A
:10E6780010BDC04610B500F07BF8C04610B5FFF7D6
:10E68800F9FFC046F0B588420AD98B18984207D2DC
:10E69800531E002A03D0CA5CC254013BFBD2F0BD12
:10E6A8000F2A09D80500002AF9D00023CC5CEC54C5
:10E6B80001339342FAD1F2E70D0005430C00030041
:10E6C800AD0729D11500103D2D092F013F1810372E
:10E6D80026681E6066685E60A6689E60E6681034FC
:10E6E800DE601033BB42F3D10F2401352D014919E7
:10E6F80014404519032C11D90023CE58EE50043389
:10E70800E61A032EF9D80323043CA4080134A40014
:10E718002D1909191A40C6E70500C6E72200C2E705
:10E7280001B40248844601BC604700BF4173001031
:10E7380001B40248844601BC604700BF352F001071
:10E7480001B40248844601BC604700BF257400102C
:10E7580001B40248844601BC604700BFB92C0010D0
:10E7680001B40248844601BC604700BF79380010F4
:10E7780001B40248844601BC604700BFE1BC0010F8
:10E78800010000000000081048E801000500000032
:10E7980098E1DA19080000000C00000011000000E0
:10E7A80010000000FC14002000000000281E0020BB
:10E7B80088250020000000000000000098250020A7
:10E7C8000000000000000000100000000000000031
:10E7D800000001000000000000000000000002002E
:10E7E800000000000000000000000300000000001E
:10E7F800000000000000FF000000000000B54868AD
:10E8080001318E460047704609380149884700BDE6
:10E81800B13D0010000000000000000000000000F2
:10E82800503300004C3300005433000052330000D2
:10E838004D5300004D4300005334000043340000A2
:10E84800B9790010000000002179001000000000D4
:10E8580000010000B0CF0010B4CF00105C2E0020E3
:10E8680010000C000000E0FF1F0000000000000086
:10E878000000000000000000000000000000000090
:10E88800C81500200000000000000000B418002097
:10E898001C1900208419002000000000000000005E
:10E8A8000000000000000000000000000000000060
:10E8B8000000000000000000000000000000000050
:10E8C8000000000000000000000000000000000040
:10E8D8000000000000000000000000000000000030
:10E8E8000000000000000000000000000000000020
:10E8F8000000000000000000000000000000000010
:10E9080000000000000000000000000000000000FF
:10E9180000000000000000000000000000000000EF
:10E9280000000000000000000000000000000000DF
:10E9380001000000000000000E33CDAB34126DE67C
:10E94800ECDE05000B0000000000000000000000E5
:10E9580000000000000000000000000000000000AF
:10E96800000000000000000000000000000000009F
:10E97800000000000000000000000000000000008F
:10E98800000000000000000000000000000000007F
:10ECB800FFFFFFFF0000020000000000000000004E
:10ECC800F8190020F8190020001A0020001A002066
:10ECD800081A0020081A0020101A0020101A002014
:10ECE800181A0020181A0020201A0020201A0020C4
:10ECF800281A0020281A0020301A0020301A002074
:10ED0800381A0020381A0020401A0020401A002023
:10ED1800481A0020481A0020501A0020501A0020D3
:10ED2800581A0020581A0020601A0020601A002083
:10ED3800681A0020681A0020701A0020701A002033
:10ED4800781A0020781A0020801A0020801A0020E3
:10ED5800881A0020881A0020901A0020901A002093
:10ED6800981A0020981A0020A01A0020A01A002043
:10ED7800A81A0020A81A0020B01A0020B01A0020F3
:10ED8800B81A0020B81A0020C01A0020C01A0020A3
:10ED9800C81A0020C81A0020D01A0020D01A002053
:10EDA800D81A0020D81A0020E01A0020E01A002003
:10EDB800E81A0020E81A0020F01A0020F01A0020B3
:10EDC800F81A0020F81A0020001B0020001B002061
:10EDD800081B0020081B0020101B0020101B00200F
:10EDE800181B0020181B0020201B0020201B0020BF
:10EDF800281B0020281B0020301B0020301B00206F
:10EE0800381B0020381B0020401B0020401B00201E
:10EE1800481B0020481B0020501B0020501B0020CE
:10EE2800581B0020581B0020601B0020601B00207E
:10EE3800681B0020681B0020701B0020701B00202E
:10EE4800781B0020781B0020801B0020801B0020DE
:10EE5800881B0020881B0020901B0020901B00208E
:10EE6800981B0020981B0020A01B0020A01B00203E
:10EE7800A81B0020A81B0020B01B0020B01B0020EE
:10EE8800B81B0020B81B0020C01B0020C01B00209E
:10EE9800C81B0020C81B0020D01B0020D01B00204E
:10EEA800D81B0020D81B0020E01B0020E01B0020FE
:10EEB800E81B0020E81B0020F01B0020F01B0020AE
:10EEC800F81B0020F81B0020001C0020001C00205C
:10EED800081C0020081C0020101C0020101C00200A
:10EEE800181C0020181C0020201C0020201C0020BA
:10EEF800281C0020281C0020301C0020301C00206A
:10EF0800381C0020381C0020401C0020401C002019
:10EF1800481C0020481C0020501C0020501C0020C9
:10EF2800581C0020581C0020601C0020601C002079
:10EF3800681C0020681C0020701C0020701C002029
:10EF4800781C0020781C0020801C0020801C0020D9
:10EF5800881C0020881C0020901C0020901C002089
:10EF6800981C0020981C0020A01C0020A01C002039
:10EF7800A81C0020A81C0020B01C0020B01C0020E9
:10EF8800B81C0020B81C0020C01C0020C01C002099
:10EF9800C81C0020C81C0020D01C0020D01C002049
:10EFA800D81C0020D81C0020E01C0020E01C0020F9
:10EFB800E81C0020E81C0020F01C0020F01C0020A9
:10EFC800F81C0020F81C0020001D0020001D002057
:10EFD800081D0020081D0020101D0020101D002005
:10EFE800181D0020181D0020201D0020201D0020B5
:10EFF800281D0020281D0020301D0020301D002065
:10F00800381D0020381D0020401D0020401D002014
:10F01800481D0020481D0020501D0020501D0020C4
:10F02800581D0020581D0020601D0020601D002074
:10F03800681D0020681D0020701D0020701D002024
:10F04800781D0020781D0020801D0020801D0020D4
:10F05800881D0020881D0020901D0020901D002084
:10F06800981D0020981D0020A01D0020A01D002034
:10F07800A81D0020A81D0020B01D0020B01D0020E4
:10F08800B81D0020B81D0020C01D0020C01D002094
:10F09800C81D0020C81D0020D01D0020D01D002044
:10F0A800D81D0020D81D0020E01D0020E01D0020F4
:10F0B800E81D0020E81D0020F01D0020F01D0020A4
:10F0C8000000000000000000097400106D660010C8
:10F0D800816D00107573001039030010D50D0010F4
:08F0E800C9A00010ADBC00102E
:04000005100001E9FD
:00000001FF
